:100000000C94080A0C94270A0C94270A0C94E20B0F
:100010000C941C0C0C94270A0C94270A0C94270AA5
:100020000C94270A0C94270A0C94270A0C94270A8C
:100030000C94270A0C94270A0C94270A0C944B0F53
:100040000C94270A0C94270A0C94270A0C94270A6C
:100050000C9475730C94286B0C94270A0C94270A43
:100060000C94270A0C94FD6B0C94270A0C94F16BEA
:100070000C94270A0C94270A0C94270A0C94270A3C
:100080000C94A87E0C94270A0C94270A0C94270A37
:100090000C943B6C0C94270A0C942F6C0C94270A3C
:1000A0000C94270A0C94270A0C94270A0C94270A0C
:1000B0000C94270A0C94270A0C94270A0C94270AFC
:1000C0000C94270A0C94270A0C94270A0C94270AEC
:1000D0000C94270A0C94270A0C94270A0C94270ADC
:1000E0000C94270A0C942E730C9438730C9424737C
:1000F0000C94E4720C9469730C945A730C944E73C0
:100100000C9442730C94270A0C94270A0C94270A27
:100110000C94270A0C94270A0C94270A0C94270A9B
:10012000DF87FE877D886C898C89AC89B489618979
:10013000084AD73B3BCE016E84BCBFFDC12F3D6C4E
:1001400074319ABD56833DDA3D00C77F11BED9E4B4
:10015000BB4C3E916BAAAABE000000803F076342E1
:1001600036B79BD8A71A39685618AEBAAB558C1D4E
:100170003CB7CC5763BD6DEDFD753EF6177231BFD0
:10018000000000803F08000000BE922449123EABF0
:10019000AAAA2ABECDCCCC4C3E00000080BEABAAA1
:1001A000AAAA3E00000000BF000000803F0000003F
:1001B0000000084178D3BB4387D1133D190E3CC3DF
:1001C000BD4282AD2B3E68EC8276BED98FE1A93E5E
:1001D0004C80EFFFBE01C4FF7F3F00000000000025
:1001E00025630025630025730A005854414C5F5471
:1001F00052494D3D25640025730A0025730A0054B9
:1002000065737420362025730A0054657374203595
:100210002025730A005465737420342025730A0066
:100220005465737420332025730A00546573742059
:10023000322025730A005465737420312025730A17
:10024000006368616E3D25640A0074787077723DC2
:1002500025640A003530306B0A003235306B0A00F5
:100260003131356B0A0035366B0A0033386B0A00C2
:1002700025730A00765F6C6F773D252D332E32662D
:100280000A0025730A0073656E743D252D75206480
:1002900075703D252D752069676E6F7265643D250B
:1002A0002D752074746C5F7A65726F3D252D750A0B
:1002B0000025372E33662025372E33660025352E50
:1002C000326620004572726F72203020566F6C7457
:1002D000004E6F7420737570706F727465640A00DD
:1002E0004572726F72203020566F6C7400457272C6
:1002F0006F72203020566F6C740062756C6B5F6497
:10030000656C61793D252D750062756C6B3D252D01
:10031000750056616C7565206E6F7420616C6C6F32
:100320007765640062756C6B3A206D61783D257568
:100330002073746172743D25752C20656E643D25B3
:10034000752C20696E5F7573653D25750A007062B6
:10035000323D25730A007062313D25730A00256C19
:100360007500416C6C6F77656420737065656420FF
:10037000312F31302F3130302F343030206B6269E3
:10038000742F730025630074746C3D252D64200068
:1003900074746C3D252D6420004E65772074746C58
:1003A0003D252D6420002563004D53353631312025
:1003B000503D252D372E326620252D372E32666D85
:1003C0000A00424D5030383520256C6420506120A1
:1003D00020252D372E32666D00256300545F484579
:1003E00041545F4944583D252D352E326620005436
:1003F0005F4445573D252D352E3266200041483D4E
:10040000252D352E32662000545F53485432583D16
:10041000252D352E3266200052485F5348543258FD
:100420003D252D352E32662000545F52483D252D46
:10043000342E3166200052483D252D342E31662061
:100440000025630025630025630025630025630004
:100450007265706F72745F616C6C3D007265706F75
:1004600072743D0025630025630025630025630049
:10047000204F534343414C3D256420002046757373
:10048000653A2065653D253032782068663D253027
:100490003278206C663D25303278206C623D253004
:1004A0003278004D43553D2530366C780025630089
:1004B00074785F6C656E3D252D6C752C765F6C6F66
:1004C000773D252D6C752C73687432783D252D6C25
:1004D000752C62756C6B3D252D6C75002563004F86
:1004E0004B0A002563002563002563002563002572
:1004F00063002563002563002563006465627567FA
:100500005F616C6C3D0064656275673D00646562A7
:1005100075673D0025730A00646565700A006E6F9B
:100520006E650A00707772733D007062323D25730C
:100530000A007062313D25730A00696E74725F7340
:1005400065635F70313D252D372E33660A00696E75
:1005500074725F70313D252D6C640A00696E74728F
:100560005F7365635F70303D252D372E33660A005B
:10057000696E74725F70303D252D6C640A00765F81
:100580006D63753D252D352E32660A00745F6D63EF
:10059000753D252D352E32660A00707077723D2527
:1005A000730A0064656275673D0072636D643D2582
:1005B000730A0025730A006175746F0A006C6F6717
:1005C0005F6D6F64653D007573625F7077723D2586
:1005D000730A0072656C61793D25730A0074746C4E
:1005E0003D252D640A0052494D455F616464723DAA
:1005F000252D642E252D640A006E65696768626F7B
:10060000725F7461626C655F73697A653D25640A27
:1006100000765F6C6F773D252D332E32660A0074AD
:100620007870773D25640A006368616E3D25640A31
:100630000069643D006932635F6275733D00693231
:10064000635F73706565643D252D6C750A00747871
:10065000743D25730A0053797374656D2053756D6D
:100660006D6172790A002530366C780041744D65F1
:100670006761323536524652320041744D656761CA
:10068000313238524652320041744D65676136341A
:10069000524652320041744D6567613132385246DC
:1006A0004131004D43553D006D61736B3D002C00A1
:1006B000696E74657276616C3D252D750023252D5C
:1006C000642C00745F686561745F69647800745FAE
:1006D00064657700616800705F6D73353631310095
:1006E00072685F736874327800745F73687432780C
:1006F0000070610070006164340061643300616403
:100700003200616431006133006132006131007692
:100710005F696E0072680065727200757074696D51
:10072000650070315F6C73740070315F74007031FC
:100730000070305F6C73740070305F740070300054
:10074000765F6D637500745F6D637500743100745E
:100750000069640065363400747874002D002B0045
:100760006175746F006E6F6E650062756C6B007002
:100770006F7765725F736176655F6C65647279002F
:1007800072656C61795F6C65647900636F6D70612F
:10079000737300616363656C007072657300705FF2
:1007A000707772006165730070315F6C6564790009
:1007B00070305F6C656472006576656E74006C65A0
:1007C00064006F7700706B740074785F6C65647997
:1007D0000072785F6C656472006F706572006E6F96
:1007E0006E65002530327800765F6164343D252DDA
:1007F000382E3666002000765F6164333D252D3843
:100800002E3666002000765F6164323D252D382E3D
:100810003666002000765F6164313D252D382E3626
:1008200066002000765F6C696768743D252D382E60
:100830003666002000765F61323D252D372E336607
:10084000002000765F61313D252D372E3366002074
:1008500000765F696E3D252D352E326600204E658F
:100860007665722D7573656420737461636B203EC9
:100870002025642062797465730A00757074696D4F
:10088000653D252D642D646179732D253032643AE0
:10089000253032643A253032642D686F7572730AE0
:1008A0000074657374205B6F66667C317C327C33C8
:1008B0007C347C355D20202020202020202D2074B9
:1008C000657374206D6F6465730A0D007478205B26
:1008D000706B74207061796C6F61645D20202020E2
:1008E00020202020202020202D2073656E6420727F
:1008F0006164696F20706B74206B6579626F6172DF
:10090000640A0D00776474205B6F6E7C6F66667C92
:10091000746573745D20202020202020202020205A
:100920002D207761746368646F670A0D00765F6CD1
:100930006F77205B765F6C6F775D20202020202012
:100940002020202020202020202D206C6F77657310
:1009500074207265706F727420766F6C7461676555
:100960000A0D007570677220202020202020202092
:100970002020202020202020202020202020202D6A
:10098000207265626F6F742076696120626F6F7488
:100990006C6F616465720A0D0075617274205B335F
:1009A000386B7C35366B7C3131356B7C3235306B56
:1009B0007C3530306B5D202D20736574207465723A
:1009C0006D2F756172742073706565640A0D006225
:1009D0006F6F742020202020202020202020202025
:1009E00020202020202020202020202D2072656221
:1009F0006F6F740A0D0070777273205B64656570A9
:100A00007C6E6F6E655D202020202020202020201D
:100A100020202D206D637520736C656570206D6FCF
:100A200064650A0D007265737420656570726F6D80
:100A300020202020202020202020202020202020B6
:100A4000202D20726573746F726520656570726FFA
:100A50006D0A0D0070707772205B6F6E7C6F66663A
:100A60005D20202020202020202020202020202049
:100A70002D2070726F6772616D6D61626C652070A0
:100A800077720A0D0070623220205B6F6E7C6F6699
:100A9000665D2020202020202020202020202020D3
:100AA000202D2070726F6772616D6D61626C6520C0
:100AB00070696E2062320A0D0070623120205B6F17
:100AC0006E7C6F66665D2020202020202020202064
:100AD00020202020202D2062756C6B204750494F2C
:100AE0002070696E0A0D00747874205B73747269EB
:100AF0006E675D2020202020202020202020202024
:100B00002020202D20536574207265706F72742030
:100B10007465787420737472696E670A0D00747856
:100B20007077205B31352D305D2020202020202063
:100B3000202020202020202020202D20545820500C
:100B400077722E20486967686573742030202833D7
:100B500064426D290A0D0074746C205B302D3135B0
:100B60005D20202020202020202020202020202048
:100B70002020202D2074696D652D746F2D6C697691
:100B80006520666F72207061636B6574730A0D0077
:100B900073732020202020202020202020202020AF
:100BA0002020202020202020202020202D2073798C
:100BB0007374656D2073756D6D6172790A0D0072C5
:100BC00073202020202020202020202020202020D2
:100BD00020202020202020202020202D2072616431
:100BE000696F2073746174730A0D007269205B234E
:100BF0006E5D205B696E745D202020202020202007
:100C0000202020202020202D207265706F727420FB
:100C1000696E74657276616C0A0D0072636D642092
:100C20005B6F6E7C6F66665D202020202020202078
:100C3000202020202020202D20616C6C6F772063E5
:100C40006D642066726F6D206E65746F726B0A0D35
:100C5000007265205B236E5D205B2B7C2D5D205B2D
:100C60006D61736B7C6175746F2C6D61736B5D204E
:100C70002D206D6F7465207265706F7274207365BE
:100C8000742F6D6F646966790A0D006F77202020DC
:100C90002020202020202020202020202020202054
:100CA000202020202020202D206F6E652D77697256
:100CB000652073656E736F72730A0D006C6F672029
:100CC0005B6175746F7C6F6E7C6F66665D20202043
:100CD00020202020202020202D206D6F746573207F
:100CE00064617461206F6E205553420A0D006E6579
:100CF000205B666C7573685D2020202020202020FA
:100D0000202020202020202020202D206E656967B3
:100D100068626F72207461626C650A0D00657272A0
:100D200020202020202020202020202020202020C3
:100D30002020202020202020202D206572726F721C
:100D40002073746174730A0D006D63752020202078
:100D50002020202020202020202020202020202093
:100D600020202020202D206D637520696E666F0A7B
:100D70000D00693263205B70726F62657C73706511
:100D8000656420236E5D20202020202020202D203F
:100D90006932632070726F6265206275737C73655F
:100DA00074206275732073706565640A0D00696450
:100DB000205B72657365745D202020202020202038
:100DC000202020202020202020202D206964206841
:100DD000616E646C696E670A0D0068756D20202075
:100DE0002020202020202020202020202020202003
:100DF0002020202020202D2068756D696469747979
:100E00002073656E736F720A0D0072656C617920D4
:100E10005B6F6E7C6F66667C73746174735D20209B
:100E20002020202020202D2072656C6179206E65A5
:100E300074776F726B207265706F7274730A0D0035
:100E40006465205B6D61736B5D2020202020202075
:100E50002020202020202020202020202D206465FC
:100E60006275670A0D006368616E205B31312D3257
:100E7000365D20202020202020202020202020201F
:100E800020202D206368616E2031312D32362028DC
:100E9000322E3430352D32343830204D687A290ADC
:100EA0000D0063616C69205B5B765F696E7C61310C
:100EB0007C61325D20766F6C747C72657365747CC6
:100EC0006E6F6E655D202D2063616C696272617466
:100ED000650A0D0062756C6B205B5B73686F777CD5
:100EE000666C7573685D205B7365742074687273DB
:100EF000682064656C61795D5D20202D2062756CD1
:100F00006B696E67207061636B657473200A0D00F6
:100F10006164632020202020202020202020202009
:100F20002020202020202020202020202D20736819
:100F30006F7720765F696E2C2061312C2061322022
:100F4000766F6C74616765730A0D00752020202030
:100F50002020202020202020202020202020202091
:100F6000202020202020202D20757074696D650AB6
:100F70000D0076202020202020202020202020204E
:100F800020202020202020202020202020202D2054
:100F900076657273696F6E0A0D006820202020202C
:100FA0002020202020202020202020202020202041
:100FB0002020202020202D2068656C700A0D00253F
:100FC0006300756E6B6E6F776E20636D640A004808
:100FD0004D433538383300257300257300202573C1
:100FE000002025362E3266200025303278007465C8
:100FF0006D705F65787465726E3D252D362E326694
:1010000000202573002025362E3266204F6E2D429B
:101010006F61726400253032780074656D705F62B4
:101020006F6172643D252D362E3266000A004275CE
:101030006C6B2072656D3A2073746172743D257516
:101040002C20656E643D25752C20696E5F75736577
:101050003D25750A0042756C6B206164643A20730B
:10106000746172743D25752C20656E643D25752C68
:1010700020696E5F7573653D25750A0042756C6B5E
:10108000207468726573683A2074696D65723D25D5
:10109000750A00503A20256C642050612020252DCF
:1010A000372E3266206D0A004932433A200045202F
:1010B00025642E256420636C6F636B20256C75207E
:1010C00063707520256C75206C706D20256C752003
:1010D00069727120256C7520676C656420256C75BC
:1010E00020796C656420256C7520726C6564202500
:1010F0006C7520747820256C75206C697374656E2E
:1011000020256C752073656E736F727320256C7566
:101110002073657269616C20256C750A0053202567
:10112000642E256420636C6F636B20256C752074BE
:101130007820256C7520727820256C752072747863
:1011400020256C752072727820256C752072657868
:101150006D697420256C752061636B747820256C33
:1011600075206E6F61636B747820256C75206163E8
:101170006B727820256C752074696D65646F757469
:1011800020256C752062616461636B727820256C28
:101190007520746F6F6C6F6E6720256C7520746F8F
:1011A0006F73686F727420256C7520626164737947
:1011B0006E636820256C752062616463726320250C
:1011C0006C7520636F6E74656E74696F6E64726F98
:1011D0007020256C752073656E64696E6764726F2C
:1011E0007020256C75206C6C747820256C75206CD3
:1011F0006C727820256C750A00257325730A004FE0
:101200006E6C696E650A000A002C20636865636B6A
:10121000207261746520257520487A002573202589
:10122000732C206368616E6E656C20257520706F6D
:10123000776572202575000A0025783A004D4143F4
:101240002061646472657373200052616E646F6D17
:101250002045554936342061646472657373206794
:10126000656E6572617465640A000A2A2A2A2A2A50
:101270002A2A426F6F74696E672025732A2A2A2AE8
:101280002A2A2A0A00454550524F4D20697320638F
:101290006F72727570742C20726577726974696EE2
:1012A0006720776974682064656661756C74732E55
:1012B0000A006C6F63616C686F73740041544D4534
:1012C00047413132387266613100020000FFFE0092
:1012D00000016E616E00696E660000407A10F35A7C
:1012E00000A0724E18090010A5D4E80000E8764866
:1012F000170000E40B54020000CA9A3B000000E112
:10130000F505000080969800000040420F000000A4
:10131000A08601000000102700000000E803000084
:1013200000006400000000000A000000000001004E
:10133000000000002C76D888DC674F0823DFC1DF6F
:10134000AE59E1B1B796E5E3E453C63AE651997672
:1013500096E8E6C28426EB898C9B62ED407C6FFCAC
:10136000EFBC9C9F40F2BAA56FA5F490055A2AF7EE
:101370005C936B6CF9676DC11BFCE0E40D47FEF5F7
:1013800020E6B500D0ED902E03009435770500805F
:10139000841E080000204E0A000000C80C333333BE
:1013A000330F986E12831141EF8D2114893BE6555E
:1013B00016CFFEE6DB18D1844B381BF77C1D901D41
:1013C000A4BBE424203284725E228100C9F124ECA3
:1013D000A1E53D274E414E494E495459494E46CD0F
:1013E000CCCC3D0AD7233C17B7D13877CC2B3295DC
:1013F00095E6241FB14F0A000020410000C84200BA
:10140000401C4620BCBE4CCA1B0E5AAEC59D740083
:1014100011241FBECFEFD1E4DEBFCDBF1AE0A0E0A4
:10142000B2E0EEE4F9E301E00BBF02C007900D92D9
:10143000A633B107D9F72DE3A6E3BAE001C01D92A8
:10144000A436B207E1F70E94838A0C94A59C0C9401
:1014500000008115910511F00197F1F7089584E2DC
:1014600095E09F938F930E948A9980916202909158
:101470006302A0916402B09165020F900F9093FFF8
:1014800003C08EE195E002C088E195E09F938F93C1
:101490000E948A990F900F900895E091FD1BEF73C1
:1014A000F0E0E25BF34E80838091FD1B8F5F8093C1
:1014B000FD1B80919E34886080939E3448E452E006
:1014C00061E1CA010E94085B80E090E00895CF933B
:1014D000DF93EC014091410A5091420A6091430A26
:1014E0007091440A46FF1DC08E811F928F938D819B
:1014F0001F928F938C811F928F938B811F928F935A
:101500008A811F928F9381E793E09F938F930E942C
:1015100078998DB79EB70C960FB6F8949EBF0FBE04
:101520008DBFBE0182E89AE00E943A5CBE0184E071
:1015300092E0DF91CF910C94AF5B1092B41C1092AB
:10154000B51C1092B31C0895CF92DF92EF92FF92D8
:101550000F931F93CF93DF93EC01FB018091B31C9A
:10156000843108F0B7C08091B51C64E10E948D926F
:101570009093B51CC090D02FD090D12FE090D22F57
:10158000F090D32F092F10E06DE8969F9001112461
:101590002D54334ED9011396CD92DD92ED92FC92EB
:1015A00016974115510569F0DA018C91D901AA57B6
:1015B000BF4F8C93DA0111968C91D901A957BF4F77
:1015C0008C932097A1F029813DE8309FC001319F85
:1015D000900D11248D54934EDC01A657BF4F2C93D0
:1015E000119688818F708C9388818F708C9330973F
:1015F000B9F186819DE8909F9001919F300D112453
:101600002D54334ED901A757BF4F8C938581119725
:101610008C93A90144575F4F83859485A585B68532
:10162000C92EDA2EEB2EFF24DA01CD92DC9279015D
:10163000BEE8EB0EF11C2385348545855685A4E66E
:10164000B0E00E942D93672F782F892F992724E6E9
:1016500030E040E050E00E94C192F7017183608366
:101660008DE8809FD001819FB00D1124A654B34E08
:10167000FE0132968FE701900D928A95E1F7209155
:10168000B51C2F5F2093B51C3091B31C3F5F309386
:10169000B31C8091410A9091420AA091430AB091F3
:1016A000440AA0FF2DC01F923F931F922F93809159
:1016B000B41C1F928F9385E590E19F938F930E94B6
:1016C0008A998DB79EB708960FB6F8949EBF0FBE45
:1016D0008DBF16C08091E02F9091E12FA091E22F55
:1016E000B091E32F0196A11DB11D8093E02F90933F
:1016F000E12FA093E22FB093E32F80E090E002C0AF
:1017000081E090E0DF91CF911F910F91FF90EF90DA
:10171000DF90CF9008952091B31C222369F180912E
:10172000B41C8F5F21502093B31C64E10E948D9202
:10173000392F9093B41C8091410A9091420AA09154
:10174000430AB091440AA0FF1AC01F922F938091C0
:10175000B51C1F928F931F923F938EE290E19F934F
:101760008F930E948A998DB79EB708960FB6F8940A
:101770009EBF0FBE8DBF03C080E090E0089581E062
:1017800090E008958823B9F052985A981DBA809134
:101790006900806280936900EA9A53985B98EB9A9B
:1017A0008091690080688093690080916800816001
:1017B000809368000895109269005A9AEA985B9A9B
:1017C000EB9808951F920F920FB60F9211248F93EA
:1017D0009F93AF93BF938091680080FF24C0809156
:1017E000793490917A34A0917B34B0917C34019615
:1017F000A11DB11D8093793490937A34A0937B34EA
:10180000B0937C348091410A9091420AA091430A9E
:10181000B091440A87FF07C0749882E090E09093EB
:101820008F0280938E02BF91AF919F918F910F9005
:101830000FBE0F901F9018951F920F920FB60F9228
:1018400011248F939F93AF93BF938091680080FF83
:1018500024C080917D3490917E34A0917F34B091EA
:1018600080340196A11DB11D80937D3490937E3408
:10187000A0937F34B09380348091410A9091420AC2
:10188000A091430AB091440A90FF07C0739882E088
:1018900090E090938F0280938E02BF91AF919F91C1
:1018A0008F910F900FBE0F901F90189580937C0022
:1018B00080917B00877F80937B0080917C00806C8F
:1018C00080937C0085E080937A0080917A00806824
:1018D00080937A0080917B0087FFFCCF80917B0012
:1018E00085FFFCCF80917A00806480937A0080919C
:1018F0007A0086FDFCCF109279001092780084E087
:1019000090E060E070E020917A00206420937A00FB
:1019100020917A0026FDFCCF20917800309179004B
:10192000620F731F0197009771F710927C008091EE
:101930007A008F7780937A0076956795769567958C
:1019400080E090E00E94D98F089580E00E94560CBC
:10195000209186023091870240918802509189023D
:101960000E94BD9121EE3AE744E95EE30E94728E47
:1019700008950F931F93CF93DF93CFE1D0E00BE552
:101980001EE0C093510187EC90E00E94290A8091EB
:10199000510185FD0DC0C031D10521F02CF00B5453
:1019A000110904C004EC19E0025311092197E9CF91
:1019B000B80180E090E00E94D98F20E030E04AE753
:1019C00054E40E943C8FDF91CF911F910F910895B5
:1019D000CF93DF93EC0188819981009799F08B3D3B
:1019E000914121F01982188283E011C0623171F4B3
:1019F0000E94B90C6093CC2F7093CD2F8093CE2F83
:101A00009093CF2F8BED91E19983888381E0DF91D3
:101A1000CF91089580917B00886080937B0089EC52
:101A200080937C0085E080937A0080917A008068C2
:101A300080937A0080917B0087FFFCCF80917B00B0
:101A400085FFFCCF80917A00806480937A0080913A
:101A50007A0086FDFCCF80917A00806480937A00C2
:101A600080917A0086FDFCCF6091780070917900BA
:101A700080917A008F7780937A0080E090E00E94D6
:101A8000D98F27ED33EA40E95FE30E94BD9126E656
:101A900036E648E853E40E94718E0895BF92CF92D3
:101AA000DF92EF92FF920F931F93CF93DF93CDB707
:101AB000DEB729970FB6F894DEBF0FBECDBF6C011D
:101AC00010923A0A8FEF89870EE01CE1B12C7E015B
:101AD00089E0E80EF11C89858823E9F1E8E0BE166B
:101AE000E1F1BE016F5F7F4FC7010E94A36489854A
:101AF0008F3F11F08E3F19F480933A0A2CC0CE012B
:101B00000196C114D10471F40E94BC6480939B348B
:101B1000FE013196A3E9B4E381918D93EE15FF05A3
:101B2000D9F71DC00E94BC64F8018083FE01319684
:101B300020E030E0A801485051098191DA01A20F5C
:101B4000B31F8C932F5F3F4F28303105B1F7B3940B
:101B5000075F1F4FC0CF8B2D03C088E001C081E01D
:101B600029960FB6F894DEBF0FBECDBFDF91CF919F
:101B70001F910F91FF90EF90DF90CF90BF9008954D
:101B80008CE290E19F938F930E948A990F900F901F
:101B900008952F923F924F925F926F927F928F9211
:101BA0009F92AF92BF92CF92DF92EF92FF920F93EC
:101BB0001F93CF93DF93EC014B01009711F427E0C3
:101BC00004C08130910549F426E04AE250E06BE21E
:101BD00070E089E290E00E948363CE010E944E0D86
:101BE0009E01255C354F5901D9018C93CD2B69F0AD
:101BF000AEE0CA2EACE1DA2EC6E0DCE1E12CF12C3D
:101C0000BDED2B2EBFE03B2EA6C083E994E30E94DE
:101C1000F165BC01882777FD8095982F0E94DB8FA6
:101C20006B017C01892869F020E030E048EC52E447
:101C30000E943C8F9F938F937F936F938AE190E1F3
:101C4000ACC0C3E9D4E305E110E189911F928F9301
:101C50001F930F930E948A990F900F900F900F90EF
:101C6000B4E3CB39DB0789F720E030E048EC52E4FD
:101C7000C701B6010E943C8F9F938F937F936F9310
:101C800085E090E19F938F930E948A990F900F9027
:101C90000F900F900F900F9080919B34882319F034
:101CA00080EA93E002C084E194E09F938F9381E007
:101CB00090E19F938F930E948A990F900F900F90BD
:101CC0000F9075C000E010E0FE01E00FF11F808171
:101CD0001F928F93A9EEBFE0BF93AF930E948A99A2
:101CE0000F5F1F4F0F900F900F900F90083011054E
:101CF00059F720E030E048EC52E4C301B2010E9401
:101D00003C8F9F938F937F936F93A1EEBFE0BF9320
:101D1000AF930E948A990F900F900F900F900F90A1
:101D20000F90D6018C91882309F455C080EA93E086
:101D30009F938F933F922F920E948A990E94C00D89
:101D4000BFEFEB1AFB0AE9E0CE0ED11C29960F90EB
:101D50000F900F900F90D5018C9190E0E816F90646
:101D6000ECF5CE010E94F165BC01882777FD8095D6
:101D7000982F0E94DB8F2B013C018114910409F400
:101D8000A1CF20E030E048EC52E40E943C8F9F93CA
:101D90008F937F936F938EEE9FE09F938F930E941C
:101DA0008A990F900F900F900F900F900F90DF91E6
:101DB000CF911F910F91FF90EF90DF90CF90BF9048
:101DC000AF909F908F907F906F905F904F903F90DB
:101DD0002F900C94C00D84E194E0AACFDF91CF91B5
:101DE0001F910F91FF90EF90DF90CF90BF90AF9039
:101DF0009F908F907F906F905F904F903F902F902B
:101E00000895CF93DF9300D0CDB7DEB7809194349F
:101E1000898380919A348A83CE0101960E94FC586E
:101E20000F900F90DF91CF910895CF93DF93EC0146
:101E3000209193343091943440919534509196345C
:101E400060919734709198348091993490919A343C
:101E5000AFEF0E94F994E1F427E04AE250E06BE230
:101E600070E089E290E00E94836380E090E00E944D
:101E70004E0DC55CD54F888349E050E06EE070E0C0
:101E800083E994E30E94FC9ADF91CF910C94010FB7
:101E9000DF91CF9108951F920F920FB60F921124E8
:101EA0000BB60F92FF920F931F932F933F934F9375
:101EB0005F936F937F938F939F93AF93BF93CF93D2
:101EC000DF93EF93FF9380919E34826080939E34E2
:101ED0008091620286FD2B9A8091620287FD2B9A87
:101EE00080918E0290918F021816190614F4749A3C
:101EF000739A8091410A9091420AA091430AB0914D
:101F0000440A85FF02C074987398809102029091F0
:101F1000030201979093030280930202892B09F038
:101F20004BC18091510A9091520A01969093520AA6
:101F30008093510A8091D02F9091D12FA091D22FD0
:101F4000B091D32F0196A11DB11D8093D02F9093F6
:101F5000D12FA093D22FB093D32F80E190E0909314
:101F60000302809302028091620280FD02C01D9BE9
:101F700005C010923F0A10923E0A06C081E090E030
:101F800090933F0A80933E0A8091410A9091420AC1
:101F9000A091430AB091440A97FF08C080913E0A7D
:101FA00090913F0A892B49F0749A7398CDEADBE14E
:101FB00005EE1FE2FF24F3941FC0739A7498F6CFC6
:101FC0008091510A9091520A01960E949992892B10
:101FD000C9F0688579856115710591F56885798500
:101FE0006115710509F03FC02A960B5F1F4FFBE199
:101FF000C53DDF0709F44DC0688579856115710518
:1020000041F3DECF4A81417020E030E050E060E0F3
:1020100070E080E090E0A0E00E94F994D1F277981F
:102020008091410A9091420AA091430AB091440ADA
:1020300092FFCFCF749810928F0210928E02C9CF68
:102040008091510A9091520A01960E949992892B8F
:1020500029F6F80114821382A80162E180E292E07D
:102060000E94085BBBCF8091510A9091520A0E9456
:102070009992892B09F0B8CFF801F082D283C183FD
:1020800014821382A80162E18EE392E00E94085B51
:10209000ABCF609168027091690261157105A1F181
:1020A0008091510A9091520A0E949992892B61F570
:1020B0008091793490917A34A0917B34B0917C34C2
:1020C0004091C2275091C3276091C4277091C527C2
:1020D000841B950BA60BB70B8093D51B9093D61B37
:1020E000A093D71BB093D81B8091793490917A3408
:1020F000A0917B34B0917C348093C2279093C32706
:10210000A093C427B093C5276091660270916702BF
:1021100061157105A1F18091510A9091520A0E94B6
:102120009992892B61F580917D3490917E34A091B4
:102130007F34B09180344091C6275091C727609179
:10214000C8277091C927841B950BA60BB70B8093EA
:10215000D91B9093DA1BA093DB1BB093DC1B8091FF
:102160007D3490917E34A0917F34B09180348093FF
:10217000C6279093C727A093C827B093C9278091FB
:10218000620286FD2B988091620290916302A09179
:102190006402B091650291FF0FC00E94A26F8A3164
:1021A00019F0C1E0C80F01C0CBE00E945E6E8C2F19
:1021B0000E94BA6F0E94A66E40E050E060E080E9A5
:1021C00092E00E94085BFF91EF91DF91CF91BF9168
:1021D000AF919F918F917F916F915F914F913F91BF
:1021E0002F911F910F91FF900F900BBE0F900FBE7C
:1021F0000F901F9018958091FD1B9091E42F891BE3
:1022000008950E94FB10882371F0E091E42FEF7392
:10221000F0E0E25BF34E808190E02091E42F2F5FAD
:102220002093E42F08958FEF9FEF0895CF93DF93CE
:10223000EC011092760A1092750A888199810097B4
:10224000B1F0843E934021F01982188283E0B6C039
:10225000613109F0B2C00E94011199279093710A6F
:102260008093700A8D3009F443C08F3F49F40E9477
:10227000FB108111F0CF84EE93E0998388839DC099
:102280008231910509F45AC08F37910509F052C087
:1022900080916E0A90916F0A181619060CF56091DC
:1022A0005E3D70915F3D88E090E00E9446996091AC
:1022B0005E3D70915F3D80E290E00E9446996091A2
:1022C0005E3D70915F3D88E090E00E94469980916C
:1022D0006E0A90916F0A019790936F0A80936E0A2D
:1022E00080916E0A90916F0A8F37910509F0BFCFE8
:1022F0001092E42F1092FD1B80916E0A90916F0A4C
:10230000FC01E750F04D10829093760A8093750A95
:1023100010926F0A10926E0A80919C3490919D34B5
:10232000009709F4A4CF40E050E0609184120E942D
:10233000085B9DCF8830910571F5AACF60915E3D15
:1023400070915F3D8DE090E00E94469910926D0A79
:1023500010926C0A80916C0A90916D0A20916E0A1D
:1023600030916F0A821793070CF0BACFFC01E75047
:10237000F04D808160915E3D70915F3D90E00E94E4
:10238000469980916C0A90916D0A019690936D0A1E
:1023900080936C0ADFCF60915E3D70915F3D0E943B
:1023A000469980916E0A90916F0A2091700AFC0103
:1023B000E750F04D208301968FCF81E0DF91CF91E0
:1023C000089580913E0A90913F0A892BD1F0809127
:1023D000620290916302A0916402B091650293FD44
:1023E00010C00E945E6E83B7817F866083BFF894C1
:1023F00083B7816083BF7894889583B78E7F83BFCE
:1024000078940895CF93DF93EC01888199810097A8
:1024100019F08E30924199F40E941B6D0E94E111D7
:1024200040E050E065E880918812909189120E9406
:10243000085B8EE092E19983888381E003C0198272
:10244000188283E0DF91CF910895CF93DF9300D07E
:10245000CDB7DEB7892B81F05F934F938AED9FE074
:102460009F938F9369837A830E948A990F900F902C
:102470000F900F907A8169817F936F9387ED9FE032
:102480009F938F930E948A990F900F900F900F90B7
:102490000F900F90DF91CF910895FF920F931F93AC
:1024A000CF93DF930E941B6D80EB0E947E668111AB
:1024B0001CC00E94E2668091CA2B9091CB2B816058
:1024C0009093CB2B8093CA2B89EA93E09F938F93B1
:1024D00087ED9FE09F938F930E948A990F900F90B2
:1024E0000F900F90C1E0D0E002C0C0E0D0E0FEB09D
:1024F0008F2D8470F82E729A0E941B6D8EE40E94BC
:102500007E66811116C00E94E2668091CA2B90916E
:10251000CB2B82609093CB2B8093CA2B8E010F5FC5
:102520001F4F4BE959E061EB73E0CE010E94251289
:10253000E801F11001C072980E941B6D8EEE0E949E
:102540007E66811116C00E94E2668091CA2B90912E
:10255000CB2B84609093CB2B8093CA2B8E010F5F83
:102560001F4F4BE959E069EB73E0CE010E94251241
:10257000E8010E941B6D86EA0E947E66811116C0EA
:102580000E94E2668091CA2B9091CB2B8860909339
:10259000CB2B8093CA2B8E010F5F1F4F4BE959E065
:1025A00060EC73E0CE010E942512E8010E941B6DD1
:1025B0008CE30E947E6681111EC00E94E2668091BB
:1025C000CA2B9091CB2B80619093CB2B8093CA2BFD
:1025D0008E010F5F1F4F4BE959E068EC73E0CE01AD
:1025E0000E9425128FEC9FE09F938F930E948A99FF
:1025F0000F900F90E8010E941B6D82ED0E947E6695
:10260000811116C00E94E2668091CA2B9091CB2B5B
:1026100080629093CB2B8093CA2B8E010F5F1F4F4C
:102620004BE959E060ED73E0CE010E942512E8010C
:102630000E941B6D80E80E947E66811116C00E9478
:10264000E2668091CA2B9091CB2B91609093CB2B1B
:102650008093CA2B8E010F5F1F4F4BE959E069ED44
:1026600073E0CE010E942512E8010E941B6D80EDEF
:102670000E947E66811116C00E94E2668091CA2B7C
:102680009091CB2B80689093CB2B8093CA2B8E019B
:102690000F5F1F4F4BE959E06FED73E0CE010E94D1
:1026A0002512E8010E941B6D8CEE0E947E6681114E
:1026B00016C00E94E2668091CA2B9091CB2B92604B
:1026C0009093CB2B8093CA2B8E010F5F1F4F4BE94A
:1026D00059E067EE73E0CE010E942512E80107E0A1
:1026E00010E00E941B6D8CE70E947E66811113C072
:1026F0000E94E2668091CA2B9091CB2B80649093CC
:10270000CB2B8093CA2B4BE959E06EEE73E0CE01E0
:102710000E94251205C0015011090115110509F784
:102720000E94E266DF91CF911F910F91FF900C9470
:10273000C00DCF93DF9300D0CDB7DEB74A83698356
:102740000E94B9666981862F0E94EA664A81842FB9
:102750000E94EA660F900F90DF91CF910C94E26691
:10276000AF92BF92DF92EF92FF920F931F93CF939E
:10277000DF9300D01F92CDB7DEB7182FD22E4A8339
:102780005B8369830E94B9666981862F0E94EA662D
:10279000812F81600E94E0664A81A42E5B81B52E64
:1027A00000E010E0ED2CF12C81E0E81AF1080D15A5
:1027B00080F40E151F0519F40E94056702C00E94DF
:1027C000FB66F50180830F5F1F4FFFEFAF1ABF0A53
:1027D000EECF0F900F900F90DF91CF911F910F913F
:1027E000FF90EF90DF90BF90AF900C94E266AF92B5
:1027F000BF92CF92DF92EF92FF920F931F93CF93EE
:10280000DF93CDB7DEB760970FB6F894DEBF0FBE8B
:10281000CDBFB82EA42E6623E9F18E010F5F1F4FA6
:1028200080E1F80111928A95E9F728E0A80168E9AA
:1028300080EB0E94B013BB2041F027EF33E03F93C1
:102840002F930E9478990F900F906E01F8E0CF0EB1
:10285000D11C9EEFE92E93E0F92EF80181918F01B2
:102860001F928F93FF92EF920E9478990F900F9092
:102870000F900F900C151D0581F788851F928F937F
:1028800023E534E03F932F930E9478990F900F90A7
:102890000F900F90AA20E9F18E010F5F1F4F80E18A
:1028A000F80111928A95E9F720E1A80160E880EB30
:1028B0000E94B013BB2041F083E094E09F938F937C
:1028C0000E9478990F900F906E01F0E1CF0ED11C0D
:1028D0008EEFE82E83E0F82EF80181918F011F9290
:1028E0008F93FF92EF920E9478990F900F900F9024
:1028F0000F900C151D0581F788891F928F9383E532
:1029000094E09F938F930E9478990F900F900F906F
:102910000F9060960FB6F894DEBF0FBECDBFDF916B
:10292000CF911F910F91FF90EF90DF90CF90BF90CC
:10293000AF900895CF93DF9300D0CDB7DEB71A8262
:10294000198222E0AE014F5F5F4F6AEA8EEE0E946D
:10295000B013898190E0982F88272A81822B909349
:102960008F1C80938E1C22E0AE014F5F5F4F6CEA9C
:102970008EEE0E94B013898190E0982F88272A81DB
:10298000822B9093911C8093901C22E0AE014F5FAC
:102990005F4F6EEA8EEE0E94B013898190E0982F0F
:1029A00088272A81822B9093931C8093921C22E08B
:1029B000AE014F5F5F4F60EB8EEE0E94B0138981D6
:1029C00090E0982F88272A81822B9093A11C8093D6
:1029D000A01C22E0AE014F5F5F4F62EB8EEE0E94C3
:1029E000B013898190E0982F88272A81822B9093B9
:1029F000A31C8093A21C22E0AE014F5F5F4F64EBEB
:102A00008EEE0E94B013898190E0982F88272A814A
:102A1000822B9093A51C8093A41C22E0AE014F5FF3
:102A20005F4F66EB8EEE0E94B013898190E0982F85
:102A300088272A81822B9093951C8093941C22E0F6
:102A4000AE014F5F5F4F68EB8EEE0E94B01389813D
:102A500090E0982F88272A81822B9093971C80934F
:102A6000961C22E0AE014F5F5F4F6AEB8EEE0E9434
:102A7000B013898190E0982F88272A81822B909328
:102A80009B1C80939A1C22E0AE014F5F5F4F6CEB62
:102A90008EEE0E94B013898190E0982F88272A81BA
:102AA000822B90939D1C80939C1C22E0AE014F5F73
:102AB0005F4F6EEB8EEE0E94B013898190E0982FED
:102AC00088272A81822B90939F1C80939E1C0F90B5
:102AD0000F90DF91CF9108952F923F924F925F9286
:102AE0006F927F928F929F92AF92BF92CF92DF921E
:102AF000EF92FF920F931F93CF93DF93CDB7DEB783
:102B00006A970FB6F894DEBF0FBECDBF182F488F5F
:102B1000298F19821A821B828091B21C811107C0F1
:102B20006A8F0E949A1481E08093B21C6A8D66239A
:102B300009F46CC04EE264EF8EEE0E94991369E0D6
:102B40007AE180E090E00E945C6622E0AE014F5F97
:102B50005F4F66EF8EEE0E94B0132981822F90E0C6
:102B6000A0E0B0E02227382F492F5A2F8A81282B46
:102B70008091A41C9091A51C281B390B4109510977
:102B8000A091A21CB091A31C0E942D936B017C010B
:102B90008FE0F594E794D794C7948A95D1F7609124
:102BA0009C1C70919D1C882777FD8095982F2BE0A9
:102BB000660F771F881F991F2A95D1F720919E1CB9
:102BC00030919F1C442737FD4095542F2C0D3D1DFF
:102BD0004E1D5F1D0E94E392C20ED31ED092991C1F
:102BE000C092981C88E0C80ED11C34E0D594C794DC
:102BF0003A95E1F7EE24D7FCE094FE2CC092A61C97
:102C0000D092A71CE092A81CF092A91C012F02955B
:102C1000000F000F007C0C5CA12FB0E0BD8BAC8BD3
:102C2000A3E0B0E0012E02C0AA0FBB1F0A94E2F796
:102C300025E335E00E942693DC01CB010296A11D1D
:102C4000B11D8C879D87AE87BF8780E593ECA0E0A0
:102C5000B0E004C0B595A795979587951A95D2F7DA
:102C6000888B998BAA8BBB8B10E0188619861A86E5
:102C70001B86A8E02A2E312CAC89BD892A1A3B0A72
:102C8000988D191709F436C1402F64EF8EEE0E941B
:102C900099136C857D858E859F850E945C6623E0F7
:102CA000AE014F5F5F4F66EF8EEE0E94B013E09172
:102CB000981CF091991CE05AFF409F01DF010E948F
:102CC0000F936B017C018091901C9091911C9F8BC4
:102CD0008E8BA0908E1CB0908F1C2091921C3091F6
:102CE000931C0E940F932B013C01ADE075946794F7
:102CF00057944794AA95D1F7A091941CB091951C34
:102D0000A70196018CE055954795379527958A95AB
:102D1000D1F70E943893BB2797FDB095AB2F480E93
:102D2000591E6A1E7B1E92E0490E511C611C711CCB
:102D300032E075946794579447943A95D1F7A0E898
:102D40005A0E611C711CA091A01CB091A11CA30182
:102D500092010E942D93DC01CB014FE0B695A7951F
:102D6000979587954A95D1F78C839D83AE83BF83D2
:102D700029818A8190E0A0E0B0E04424582E692E99
:102D80007A2E622A8B81482A022C04C0759467949B
:102D9000579447940A94D2F74501AA2497FCA0942B
:102DA000BA2C62E0880C991CAA1CBB1C6A95D1F74E
:102DB000A091961CB091971CA70196010E94389390
:102DC0006B017C0177E1F594E794D794C7947A95E9
:102DD000D1F72E893F89DF010E940F93EBE0959593
:102DE000879577956795EA95D1F7C60ED71EE81EA9
:102DF000F91E8C0C9D1CAE1CBF1C0C8804C0880CDA
:102E0000991CAA1CBB1C0A94D2F792E0890E911C53
:102E1000A11CB11CF2E0B594A79497948794FA95FD
:102E2000D1F7481859086A087B08A30192016889FC
:102E300079898A899B890E947D9297FD0DC0660FD2
:102E4000771F881F991F2C813D814E815F810E94D1
:102E5000C19249015A010CC02C813D814E815F8194
:102E60000E94C19249015A01880C991CAA1CBB1CE2
:102E70009927B7FC9A958B2D7A2D692D9B01AC0172
:102E80000E947D929B01AC01AEEDBBE00E942D93B0
:102E90006C01FF24D7FCF094EF2CA3E4B3EEA50162
:102EA00094010E943B93BB2797FDB095AB2FC80EB2
:102EB000D91EEA1EFB1EAFECCA0EAEE0DA1EE11C04
:102EC000F11C64E0F594E794D794C7946A95D1F720
:102ED000C80CD91CEA1CFB1C88859985AA85BB8572
:102EE0008C0D9D1DAE1DBF1D88879987AA87BB8746
:102EF0001F5FC6CE112391F0212F30E040E050E05B
:102F0000688579858A859B850E94C1922093AA1C39
:102F10003093AB1C4093AC1C5093AD1CA98DAA23DD
:102F200089F16091AA1C7091AB1C8091AC1C9091AE
:102F3000AD1C611571058105910521F10E94DB8FA2
:102F400020E836EE45EC57E40E943C8F21E03EED50
:102F500042E45EE30E9420929B01AC0160E070E0DD
:102F600080E89FE30E94718E2BE43AE34DEB57E338
:102F70000E943C8F6093AE1C7093AF1C8093B01C7A
:102F80009093B11C6A960FB6F894DEBF0FBECDBF0A
:102F9000DF91CF911F910F91FF90EF90DF90CF9035
:102FA000BF90AF909F908F907F906F905F904F9069
:102FB0003F902F9008950F931F93CF93DF9300D0EE
:102FC00000D000D0CDB7DEB78E010F5F1F4F86E077
:102FD000F80111928A95E9F78091A41B811113C021
:102FE00040E061E386EA0E9499134AE06CE286EAD7
:102FF0000E94991381E08093A41B6CE77EE380E03C
:1030000090E00E945C6648E06DE286EA0E949913B7
:103010006CE77EE380E090E00E945C6626E0A80119
:1030200062E386EA0E94B01347E06DE286EA0E94FE
:1030300099138A8190E0982F88272981822B909379
:103040009F1B80939E1B2C8130E0322F22274B81C7
:10305000242B3093A11B2093A01B4E8150E0542FB2
:1030600044276D81462B5093A31B4093A21B5F9373
:103070004F933F932F939F938F9387E094E09F9379
:103080008F930E9478990FB6F894DEBF0FBECDBF24
:1030900026960FB6F894DEBF0FBECDBFDF91CF915D
:1030A0001F910F910895CF92DF92EF92FF920F93AD
:1030B0001F93CF93DF93CDB7DEB72A970FB6F8945F
:1030C000DEBF0FBECDBF8E010F5F1F4F86E0F80140
:1030D00011928A95E9F741E062E08CE30E9499132E
:1030E00048E560E08CE30E94991362E174E380E0BC
:1030F00090E00E945C6626E0A80163E08CE30E94F9
:10310000B01343E062E08CE30E949913098110E060
:10311000102F00278A81082B10937F1B00937E1BA2
:10312000EB80F12CFE2CEE248C81E82AF092811B9E
:10313000E092801BCD80D12CDC2CCC248E81C82A3F
:10314000D092831BC092821BB801882777FD80959F
:10315000982F0E94DB8F9B01AC01B701882777FD78
:103160008095982F2F83388749875A870E94DB8F55
:103170002F81388549855A850E94E58E20EE3EE2F2
:1031800045E652E40E94BD9120E030E044E353E480
:103190000E94728E9F938F937F936F93DF92CF9253
:1031A000FF92EF921F930F9385E194E09F938F938B
:1031B0000E9478990FB6F894DEBF0FBECDBF2A9655
:1031C0000FB6F894DEBF0FBECDBFDF91CF911F9138
:1031D0000F91FF90EF90DF90CF900895CF93DF9302
:1031E000EC0188819981009759F1873F914121F045
:1031F0001982188283E06FC08BE59AE00E94AE5D71
:10320000892B41F18091410A9091420AA091430A91
:10321000B091440A93FD20C04091410A5091420A66
:103220006091430A7091440A54FD47C04091410A9D
:103230005091420A6091430A7091440A55FD44C07E
:1032400060E870E08BE59AE00E94875D87EF91E18E
:103250009983888381E03FC08091CA2B82FFDCCFB5
:1032600021E048E061E083E00E946C158091B11C90
:103270008F938091B01C8F938091AF1C8F9380911E
:10328000AE1C8F938091AD1C8F938091AC1C8F935B
:103290008091AB1C8F938091AA1C8F9383E990E15E
:1032A0009F938F930E948A998DB79EB70A960FB607
:1032B000F8949EBF0FBE8DBFAFCF8091CA2B83FF06
:1032C000B5CF0E94DB17B2CF8091CA2B84FFB8CF55
:1032D0000E945318B5CFDF91CF910895CF93C82F97
:1032E0008CEE0E94E0668C2F0E94EA6665E375E032
:1032F00080E090E00E945C668DEE0E94E0660E9495
:10330000FB66C82F0E9405672C2F30E0322F222742
:10331000A901482BCA01CF910895CF93DF93C82FFD
:103320008CEE0E94E0668C2F0E94EA6662E174E3F4
:1033300080E090E00E945C668CEE0E94E06680E097
:103340000E94EA6665E375E080E090E00E945C66BA
:103350008DEE0E94E0660E94FB66C82F0E94FB660D
:10336000D82F0E9405674D2F50E060E070E0762F67
:10337000652F542F44276C2B482BCB01BA01DF91CA
:10338000CF9108952F923F924F925F926F927F92CA
:103390008F929F92AF92BF92CF92DF92EF92FF9265
:1033A0000F931F93CF93DF93CDB7DEB7CD54D109E1
:1033B0000FB6F894DEBF0FBECDBF80910002909192
:1033C0000102892BD1F110920102109200028CEEC1
:1033D0000E94E0668EE10E94EA666BE17EE480E096
:1033E00090E00E945C6682EA0E946E199093500AF7
:1033F00080934F0A84EA0E946E1990934E0A80933C
:103400004D0A86EA0E946E1990934C0A80934B0AEB
:1034100088EA0E946E1990934A0A8093490A8AEAC0
:103420000E946E199093480A8093470A8CEA0E9482
:103430006E199093460A8093450A88E40E948D197C
:103440006FAB78AF89AF9AAF88E50E948D194B01B9
:103450005C018091470A9091480A20E030E040E00A
:1034600050E0BA0126962FAF269727963FAF2797B1
:1034700028964FAF289729965FAF29972A966FAF66
:103480002A972B967FAF2B979C0140E050E060E09D
:1034900070E080E090E008E00E949B940E945494C9
:1034A0003901B42FA52FF62FE72F8C019401A50128
:1034B00060E070E080E090E05301CB2EDA2EEF2E3A
:1034C000FE2E0E94D29429833A832A011B014C01CB
:1034D000B101C401315041095F4F6F4F7F4F8F4F92
:1034E0009F4FA1E0B0E02596BFAFAEAF2597211565
:1034F0003F4F4F4F5140610571058105910509F01E
:1035000020F425961FAE1EAE259725966EAC7FAC97
:1035100025978091450A9091460A5C01C12CD12CD7
:10352000E12CF12C00E010E029813A81A201B101E7
:10353000C4010E944093D22EE32EF42E052F162FA5
:10354000B72FF82FE92FA0E00E94F99484F42150BE
:10355000310940485F4F6F4F7F4F8F4F9F4FD22EA3
:10356000E32EF42E052F162FB72FF82FE92F2D2D30
:103570003E2D4F2D502F612F7B2F8F2F9E2F07E138
:103580000E94B4942B8F3C8F4D8F5E8F6F8F78A3EA
:1035900089A39AA32053384F4F4F5F4F6F4F7F4FF0
:1035A0008F4F9F4F2B8B3C8B4D8B5E8B6F8B788F10
:1035B000898F9A8F2056304F4F4F5F4F6F4F7F4FFD
:1035C0008F4F9F4F243D30434105510561057105E3
:1035D0008105910541F038F025966EAC7FAC2597BA
:1035E000FFEF6F1A7F0A80914D0A90914E0A9C015D
:1035F00040E050E060E070E080E090E000E10E9498
:103600009B942B833C834D835E836A8779878F836A
:1036100098874091490A50914A0AA980BA8062016C
:10362000710184019A0140E050E060E070E080E0C8
:1036300090E00E944093D22EE32EF42E052F162FF9
:10364000B72FF82FE92FA0E00E94F9945CF4AFE7C0
:103650000E94DB94D22EE32EF42E052F162FB72FC7
:10366000F82FE92F2D2D3E2D4F2D502F612F7B2F21
:103670008F2F9E2F07E00E94B49459016A017B01AD
:103680008C012B813C814D815E816A8579858F819A
:1036900098850E94D2942B833C834D835E836F83F5
:1036A00078878F87988B2E5F3F4F434051096E4F2D
:1036B0007F4F8F4F9F4F22303105494F5F4F6440FE
:1036C00071058105910521F018F01FEF611A710A4B
:1036D00080914F0A9091500ABC0180E090E020E078
:1036E00030E840E050E00E94999329873A874B8761
:1036F0005C876A8B798B8D879E8740914B0A5091AE
:103700004C0AA980BA806201710184019A0140E0EB
:1037100050E060E070E080E090E00E944093D22EA4
:10372000E32EF42E052F162FB72FF82FE92FA0E048
:103730000E94F99484F421503F4F4F4F5F4F6F4FD9
:103740007F4F8F4F9F4FD22EE32EF42E052F162F33
:10375000B72FF82FE92F2D2D3E2D4F2D502F612FF4
:103760007B2F8F2F9E2F08E00E94B49459016A018D
:103770007B018C0129853A854B855C856A8979892D
:103780008D859E850E94D29429873A874B875C87D6
:103790006D877E87898B9A8B2F5F3F4F4140510900
:1037A0006109710981099109213030484C4F5F4707
:1037B000614071058105910521F018F0BFEF6B1A8A
:1037C0007B0A2B893C894D895E896F89788D898D2B
:1037D0009A8D2F3C374041055105610571058105E2
:1037E000910511F00CF0A5C1A980BA8062017101A8
:1037F00084019501A201B101C4010E944093A12C52
:10380000B12CC12C10E8D12EE12CF12C00E010E0FD
:103810000E94C6932BAF3CAF4DAF5EAF6FAF21960A
:103820007FAF219722968FAF229723969FAF239742
:10383000AB8CBC8CCD8CDE8CEF8CF8A009A11AA1CE
:103840009501A601B701C8010E94409359016A0180
:103850007B01E82F192F02E00E949B940E2F0E94FB
:10386000D29469017A01162F272EF82FE92F322ED4
:103870008D2C942EAF2CB62E072F582EB92FA0E0EA
:103880000E94F9945CF4A1E00E94DB94322E832E16
:10389000942EA52EB62E072F582EB92F232D382D56
:1038A000492D5A2D6B2D702F852D9B2F01E00E94E5
:1038B000B4942E962FAF2E972D963FAF2D9749A7F4
:1038C0005AA76BA77CA78DA79EA7522E432E4BA36A
:1038D0005CA36DA37EA38FA398A7B22D9601A70129
:1038E000612F722D8F2F9E2FA0E00E94F9944CF42F
:1038F000A3E00E94DB9469017A01162FB72FF82FFD
:10390000E92F9601A701612F7B2F8F2F9E2F02E0B9
:103910000E94B4942FA738AB49AB5AAB6BAB7CABCE
:103920008DAB9EAB19014A01B62FA72F24968FAFFE
:103930002497F92F2B893C894D895E896F89788D71
:10394000898D9A8D24323A4F4F4F5F4F6F4F7F4F83
:103950008F4F9F4F0CF08CC02B8D3C8D4D8D5E8D0D
:103960006F8D78A189A19AA12455324F4F4F5F4F97
:103970006F4F7F4F8F4F9F4F59016A017B018C0121
:103980000E94409319014A01B62FA72FFC0103E0C2
:103990000E949B9451016401EB2EFA2E8F010E942C
:1039A000E79459016A017B018C012E962FAD2E9769
:1039B0002D963FAD2D9749A55AA56BA57CA58DA544
:1039C0009EA50E94D294522E432E4BA35CA36DA3BE
:1039D0007EA38FA398A79101A4016B2F7A2FCF010B
:1039E00002E00E949B9451016401EB2EFA2E8F019C
:1039F0000E94E79402E00E949B940E2F0E94E7949D
:103A0000F22E032F142FD52EE62EB72FF82FE92FE5
:103A1000A0E00E94F9945CF4A1E00E94DB94F22EF5
:103A2000032F142FD52EE62EB72FF82FE92F2F2D89
:103A3000302F412F5D2D6E2D7B2F8F2F9E2F01E07C
:103A40000E94B49459016A017B018C012FA538A909
:103A500049A95AA96BA97CA98DA99EA90E94D294B3
:103A600019014A01B62FA72F24968FAF2497F92F5B
:103A70002B813C814D815E816F8178858F8598890E
:103A8000A52CB42CCBA0DCA0EDA0FEA00FA118A506
:103A90000E94E7942B833C834D835E836F837887FA
:103AA0008F87988B29853A854B855C856D857E85CA
:103AB00089899A8951016401EB2EFA2E24960FAD63
:103AC00024971F2F0E94E79429873A874B875C87AA
:103AD0006D877E87898B9A8B2B893C894D895E897E
:103AE0006F89788D898D9A8DABACBCACCDACDEACDA
:103AF000EFAC2196FFAC219722960FAD229723962B
:103B00001FAD23970E94E7942056304F4F4F5F4FD1
:103B10006F4F7F4F8F4F9F4F243D304341055105DD
:103B2000610571058105910521F018F02FEF621AEA
:103B3000720A6FA978AD89AD9AADAB01BC0180E086
:103B400090E0DC0124964FAF249725965FAF259730
:103B500026966FAF269727967FAF279728968FAF29
:103B6000289729969FAF29972A96AFAF2A972B9629
:103B7000BFAF2B97A984BA84CB84DC84ED84FE8408
:103B800009891A899A01AB0160E070E080E090E059
:103B90000E944093F22E032F142FD52EE62EB72F1E
:103BA000F82FE92FA0E00E94F99484F42150310904
:103BB000404E5F4F6F4F7F4F8F4F9F4FF22E032F1F
:103BC000142FD52EE62EB72FF82FE92F2F2D302FBB
:103BD000412F5D2D6E2D7B2F8F2F9E2F05E10E9493
:103BE000B494AB80BC80CD80DE80EF80F8840F85FC
:103BF00018890E94E794F22E032F142FD52EE62E5B
:103C0000B72FF82FE92FA0E00E94F99484F42150F7
:103C100030484F4F5F4F6F4F7F4F8F4F9F4FF22E68
:103C2000032F142FD52EE62EB72FF82FE92F2F2D87
:103C3000302F412F5D2D6E2D7B2F8F2F9E2F0FE06C
:103C40000E94B49469017A018B018A8399832901C6
:103C50001A014B015C01285E334041095109610999
:103C6000710981099109283D304D41405105610597
:103C700071058105910521F018F0BFEF6B1A7B0AE1
:103C80000E94E266672859F09601A701B8018A816F
:103C900099810E94549429011A014B015C019201FF
:103CA000A101B401C5010E94D58F20E030E048ECAD
:103CB00052E40E943C8FC35BDF4F0FB6F894DEBF27
:103CC0000FBECDBFDF91CF911F910F91FF90EF906D
:103CD000DF90CF90BF90AF909F908F907F906F902C
:103CE0005F904F903F902F9008954F925F926F9208
:103CF0007F928F929F92AF92BF92CF92DF92EF927C
:103D0000FF922B013C0169017A0123EC35EF4CE86D
:103D100051E4C701B6010E94BD914B015C0128EB43
:103D20003EE143E753E4C701B6010E94728E9B0156
:103D3000AC01C501B4010E943C8F0E94A98F4B01C8
:103D40005C0120E030E048EC52E4C301B2010E9483
:103D50003C8F21E835E943EC50E40E94BD91A50178
:103D600094010E94BD914B015C0123E333E948E8D3
:103D700053E4C701B6010E94728E9B01AC01C501DC
:103D8000B4010E943C8F23E333EB48E553E40E94E7
:103D9000BD91FF90EF90DF90CF90BF90AF909F903C
:103DA0008F907F906F905F904F9008954F925F92A9
:103DB0006F927F928F929F92AF92BF92CF92DF923B
:103DC000EF92FF9269017A010E943F9120E030E07A
:103DD00040E050E40E94718E22E93CE54EED5EE346
:103DE0000E943C8F4B015C0123EC35EF4CE851E421
:103DF000C701B6010E94BD912B013C0128EB3EE1B9
:103E000043E753E4C701B6010E94728E9B01AC01E7
:103E1000C301B2010E943C8F9B01AC01C501B401FA
:103E20000E94728E6B017C0128EB3EE143E753E474
:103E30000E94BD914B015C01A701960163EC75EFF7
:103E40008CE891E40E94718E9B01AC01C501B40124
:103E50000E943C8FFF90EF90DF90CF90BF90AF908B
:103E60009F908F907F906F905F904F9008954F92AA
:103E70005F926F927F928F929F92AF92BF92CF92FA
:103E8000DF92EF92FF922B013C0169017A0123EC52
:103E900035EF4CE851E4C701B6010E94BD914B01DA
:103EA0005C0128EB3EE143E753E4C701B6010E9401
:103EB000728E9B01AC01C501B4010E943C8F0E942F
:103EC000A98F4B015C0120E030E048EC52E4C301D3
:103ED000B2010E943C8FA50194010E94BD9120E097
:103EE00030E040E251E40E94718E24EE38E34EE06F
:103EF0005FE30E94BD919B01AC01C701B6010E9426
:103F0000728EFF90EF90DF90CF90BF90AF909F9018
:103F10008F907F906F905F904F90089580E80E94FF
:103F2000E06681110DC08EEF0E94EA66811108C023
:103F30006BE17EE480E090E00E945C660C94E266B7
:103F40000E94E2668091DC2F9091DD2FA091DE2F00
:103F5000B091DF2F0196A11DB11D8093DC2F9093AE
:103F6000DD2FA093DE2FB093DF2F0895FC01DC013D
:103F700082E020E041E39D91292798E0322F330F22
:103F800027FF03C0232F242701C0232F9150B1F70F
:103F9000815089F781E090E03281231711F080E0B1
:103FA00090E00895DF92EF92FF920F931F93CF93CB
:103FB000DF930E948E1F80E80E94E06681116DC031
:103FC0008AEF0E94EA66811168C08FE00E94EA666B
:103FD000811163C065E375E080E090E00E945C665B
:103FE00081E80E94E066811158C00E94FB66C82FDC
:103FF0000E94FB660E94FB66D82F0E94FB660E940F
:10400000FB66182F0E94FB660E940567082F80E858
:104010000E94E066811141C08CEF0E94EA66811126
:104020003CC089EC0E94EA66811137C065E375E007
:1040300080E090E00E945C6681E80E94E0660E9459
:10404000FB66E82E0E94FB66D82E0E94FB660E944B
:10405000FB66F82E0E9405671F92DF921F92EF9277
:104060001F920F931F921F931F92DF931F92CF9364
:104070001F928F931F92FF928AE294E09F938F93F7
:104080000E9478990E94E2668DB79EB742960FB65D
:10409000F8949EBF0FBE8DBF17C00E94E26680914C
:1040A000DC2F9091DD2FA091DE2FB091DF2F0196B4
:1040B000A11DB11D8093DC2F9093DD2FA093DE2FE7
:1040C000B093DF2F0E948E1F20E030E040E050E0F0
:1040D00060E070E080E090E0DF91CF911F910F9160
:1040E000FF90EF90DF900895EF92FF920F931F9350
:1040F000CF93DF9300D01F92CDB7DEB78C0180E85D
:104100000E94E066811154C00115110551F085EE41
:104110000E94EA6681114CC061E077E980E090E09E
:1041200009C083EE0E94EA66811142C069E97AEB18
:1041300081E090E00E945C6681E80E94E066811167
:1041400037C00E94FB66F82E89830E94FB66E82E2A
:104150008A830E9405678B830E94E266CE010196E6
:104160000E94B61F892B21F16E2D70E07F296C7F94
:1041700080E090E0012B69F00E94D98F20E030E0D0
:104180004AEF5AE30E94BD9120E030E040EC50E459
:104190000CC00E94D98F22E538EB4FE25BE30E940E
:1041A000BD9126E636E64BE352E40E94718E1BC0B9
:1041B0000E94E2668091DC2F9091DD2FA091DE2F8E
:1041C000B091DF2F0196A11DB11D8093DC2F90933C
:1041D000DD2FA093DE2FB093DF2F0E948E1F60EFA4
:1041E0007FEF89E794E40F900F900F90DF91CF91CC
:1041F0001F910F91FF90EF9008950F931F93CF930E
:10420000DF93729A8091620283FF08C08EE40E945D
:104210007E66811167C0C0E5D0E00AC0C0E5D0E08D
:1042200087EE93E00E94290A21972097C9F7EECFE5
:1042300087EE93E00E94290A21972097C9F78FE41F
:104240000E947E660E94FB66082F0F730E94FB6629
:10425000182F0E94FB66D82F0E940567C82F0E9466
:10426000E2668091620283FF7298602F70E0762F81
:104270006627610F711D80E090E00E94D98F20E1D8
:1042800034E048EC5BE30E94BD916093BE277093DD
:10429000BF278093C0279093C1276D2F70E0762FA2
:1042A00066276C0F711D769567957695679580E00A
:1042B00090E00E94D98F24EA3CEF44E25CE30E9444
:1042C000BD9120E030E040E252E40E94718E6093A4
:1042D0009F347093A0348093A1349093A23480E0F3
:1042E00090E002C081E090E0DF91CF911F910F91AB
:1042F00008957298729A8EE40E947E6680EA0E9407
:10430000EA6680E00E94EA6680E00E94EA668FE446
:104310000E947E660E94FB668EE40E947E6680E8B4
:104320000E94EA6680E00E94EA6680E00E94EA66F7
:104330000E94E26680E090E0089582EC9FE09F9307
:104340008F930E948A9980917D020F900F9088230D
:1043500061F01F928F938FEB9FE09F938F930E944A
:104360008A990F900F900F900F9008958AE99FE01F
:104370009F938F930E948A9982E79FE09F938F93E8
:104380000E948A998BE49FE09F938F930E948A9961
:1043900080E19FE09F938F930E948A9984ED9EE035
:1043A0009F938F930E948A9982EA9EE09F938F93B6
:1043B0000E948A9986E69EE09F938F930E948A9935
:1043C00080E49EE09F938F930E948A998AE09EE00A
:1043D0009F938F930E948A998091CA2B9091CB2BA7
:1043E000827091702DB73EB72E5E3F4F0FB6F89496
:1043F0003EBF0FBE2DBF892B41F08AED9DE09F93FC
:104400008F930E948A990F900F908EEA9DE09F9360
:104410008F930E948A9982E79DE09F938F930E94D9
:104420008A9989E49DE09F938F930E948A998DE1F8
:104430009DE09F938F930E948A998EEE9CE09F93BC
:104440008F930E948A998CEB9CE09F938F930E949C
:104450008A998BE89CE09F938F930E948A9981E5CB
:104460009CE09F938F930E948A998BE19CE09F939D
:104470008F930E948A998BEE9BE09F938F930E946B
:104480008A998FEB9BE09F938F930E948A9980E992
:104490009BE09F938F930E948A9987E59BE09F936F
:1044A0008F930E948A998EE19BE09F938F930E9445
:1044B0008A9987EE9AE09F938F930E948A9989EB5D
:1044C0009AE09F938F930E948A998DB79EB78096AA
:1044D0000FB6F8949EBF0FBE8DBF85E89AE09F93FC
:1044E0008F930E948A9984E59AE09F938F930E940C
:1044F0008A9985E29AE09F938F930E948A9986EF2A
:1045000099E09F938F930E948A998FEC99E09F93F3
:104510008F930E948A9989E999E09F938F930E94D3
:104520008A9983E699E09F938F930E948A998DE2FE
:1045300099E09F938F930E948A9984E099E09F93DA
:104540008F930E948A998CEC98E09F938F930E949E
:104550008A9981EA98E09F938F930E948A992DB758
:104560003EB72A5E3F4F0FB6F8943EBF0FBE2DBF39
:10457000089589E594E00C94AE994F925F926F9202
:104580007F928F929F92AF92BF92CF92DF92EF92E3
:10459000FF92CF93DF93CDB7DEB728970FB6F8948D
:1045A000DEBF0FBECDBF8091D02F9091D12FA091B3
:1045B000D22FB091D32F89839A83AB83BC83409051
:1045C000D02F5090D12F6090D22F7090D32F809108
:1045D000D02F9091D12FA091D22FB091D32F8D8336
:1045E0009E83AF83B8876091D02F7091D12F809137
:1045F000D22F9091D32F2CE3822E912CA12CB12C71
:10460000A50194010E94C1927F936F9330E1C32E64
:104610003EE0D32EE12CF12C6D817E818F81988537
:10462000A70196010E94C192A50194010E94C19226
:104630003F932F9340E8842E41E5942EAA24A3941F
:10464000B12CC301B201A50194010E94C192A7013E
:1046500096010E94C1923F932F9369817A818B8149
:104660009C81A50194010E94C1923F932F938BE7F7
:1046700098E09F938F930E948A990FB6F894DEBFBB
:104680000FBECDBF28960FB6F894DEBF0FBECDBFCC
:10469000DF91CF91FF90EF90DF90CF90BF90AF90E0
:1046A0009F908F907F906F905F904F900895E4E679
:1046B000FDE3808191818234924479F0E456FD4398
:1046C000FF93EF938DE598E09F938F930E948A99D3
:1046D0000F900F900F900F9008953A96E53F81E468
:1046E000F80738F30895CF93DF93EC018C9A0E947A
:1046F000A50C9F938F937F936F9381E598E09F9391
:104700008F930E948A990F900F900F900F900F90A7
:104710000F90209719F00E94C00D08C08FE498E018
:104720009F938F930E948A990F900F9081E00E942F
:10473000560C209182023091830240918402509164
:1047400085020E94BD919F938F937F936F9383E423
:1047500098E09F938F930E948A990F900F900F90EB
:104760000F900F900F90209719F00E94C00D08C075
:1047700081E498E09F938F930E948A990F900F9005
:1047800082E00E94560C20917E0230917F0240917F
:104790008002509181020E94BD919F938F937F93DD
:1047A0006F9385E398E09F938F930E948A990F906F
:1047B0000F900F900F900F900F90209719F00E947C
:1047C000C00D08C083E398E09F938F930E948A995D
:1047D0000F900F9083E00E94560C9F938F937F93CE
:1047E0006F9384E298E09F938F930E948A998C98AC
:1047F0000F900F900F900F900F900F90209719F03F
:104800000E94C00D08C082E298E09F938F930E949F
:104810008A990F900F908091CA2B87FF83C021E067
:1048200042E161E080ED0E9442689F938F937F9305
:104830006F9385E198E09F938F930E948A990F90E0
:104840000F900F900F900F900F90209719F00E94EB
:10485000C00D08C083E198E09F938F930E948A99CE
:104860000F900F9021E042E162E080ED0E944268EB
:104870009F938F937F936F9386E098E09F938F939E
:104880000E948A990F900F900F900F900F900F90A9
:10489000209719F00E94C00D08C084E098E09F9313
:1048A0008F930E948A990F900F9021E042E163E07C
:1048B00080ED0E9442689F938F937F936F9387EF61
:1048C00097E09F938F930E948A990F900F900F907B
:1048D0000F900F900F90CD2B19F00E94C00D08C0C3
:1048E00085EF97E09F938F930E948A990F900F9086
:1048F00021E042E164E080ED0E9442689F938F9343
:104900007F936F9388EE97E09F938F930E948A998D
:104910000F900F900F900F900F900F90DF91CF910D
:104920000C94C00DCD2BD1F3DF91CF9108950F934F
:104930001F93CF93DF93882389F049E050E06FEF16
:1049400070E083E994E30E94CC9849E050E06EE087
:1049500070E083E994E30E94FC9A13C0C3E9D4E3B6
:1049600003EE17E089911F928F931F930F930E947C
:104970008A990F900F900F900F9084E3CB39D8074E
:1049800089F7DF91CF911F910F910C94C00D88236F
:1049900011F0299A089529980895882311F02A9AE8
:1049A00008952A980895882311F02B9A08952B983A
:1049B0000895CF92DF92EF92FF92CF93DF936B0136
:1049C0007C0160FF11C086E994E09F938F9387ED8F
:1049D0009FE09F938F930E948A990F900F900F9062
:1049E0000F9081E090E002C080E090E0C1FE09C03D
:1049F000EC0121964BE959E06BE974E00E94251225
:104A0000CE01C2FE09C0EC0121964BE959E063EAF0
:104A100074E00E942512CE01C3FE09C0EC0121966C
:104A20004BE959E06BEA74E00E942512CE01C4FE06
:104A300009C0EC0121964BE959E066E176E00E945D
:104A40002512CE01C5FE09C0EC0121964BE959E0C3
:104A50006FEA74E00E942512CE01C6FE09C0EC0187
:104A600021964BE959E063EB74E00E942512CE01D8
:104A7000C7FE09C0EC0121964BE959E069EB74E0EF
:104A80000E942512CE01D0FE09C0EC0121964BE90F
:104A900059E061EC74E00E942512CE01D1FE09C0FC
:104AA000EC0121964BE959E069EC74E00E94251273
:104AB000CE01D2FE09C0EC0121964BE959E06DEC24
:104AC00074E00E942512CE012091CA2B3091CB2B8D
:104AD00024703270232B59F0D3FE09C0EC012196CB
:104AE0004BE959E063ED74E00E942512CE0120915C
:104AF000CA2B23FF0BC0D4FE09C0EC0121964BE961
:104B000059E068ED74E00E942512CE012091CA2B75
:104B100024FF0BC0D5FE09C0EC0121964BE959E0FA
:104B20006EED74E00E942512CE01D6FE09C0EC01A4
:104B300021964BE959E066EE74E00E942512CE0101
:104B4000D7FE09C0EC0121964BE959E061EF74E012
:104B50000E942512CE01E0FE0CC04BE959E062E054
:104B600075E0DF91CF91FF90EF90DF90CF900C94A4
:104B70002512CD28CE28CF2841F48EED97E09F93C3
:104B80008F930E948A990F900F90DF91CF91FF90A1
:104B9000EF90DF90CF900895CF92DF92EF92FF9247
:104BA000CF93DF93EC01C12CD12C7601209709F42F
:104BB000A3C069ED77E0CE010E94AB98892B11F478
:104BC0006894C0F861ED77E0CE010E94AB98892B24
:104BD00011F46894C1F869EC77E0CE010E94AB98BB
:104BE000892B11F46894C2F865EC77E0CE010E943D
:104BF000AB98892B11F46894C3F862EC77E0CE018E
:104C00000E94AB98892B11F46894C4F86EEB77E09E
:104C1000CE010E94AB98892B11F46894C5F868EB1B
:104C200077E0CE010E94AB98892B11F46894C6F806
:104C300060EB77E0CE010E94AB98892B11F4689469
:104C4000C7F868EA77E0CE010E94AB98892B11F48F
:104C50006894D0F864EA77E0CE010E94AB98892B83
:104C600011F46894D1F86EE977E0CE010E94AB9818
:104C7000892B11F46894D2F869E977E0CE010E949B
:104C8000AB98892B11F46894D3F863E977E0CE01EF
:104C90000E94AB98892B11F46894D4F86BE877E004
:104CA000CE010E94AB98892B11F46894D5F860E886
:104CB00077E0CE010E94AB98892B11F46894D6F866
:104CC0006FE677E0CE010E94AB98892B11F46894CF
:104CD000D7F86AE677E0CE010E94AB98892B11F4F1
:104CE0006894E0F860917B0270917C0280E090E033
:104CF0000E94BF98EC015ACFC701B601DF91CF9156
:104D0000FF90EF90DF90CF900895AF92BF92CF9237
:104D1000DF92EF92FF920F931F93CF93DF93F22EC8
:104D2000032F142FE52ED62EA72EB82EC92E2170B4
:104D300030E040E050E060E070E080E090E0A0E033
:104D40000E94F99489F0E7E0F5E0FF93EF93E7ED37
:104D5000FFE0FF93EF930E948A990F900F900F90BE
:104D60000F90E1E0F0E002C0E0E0F0E08091CA2BBB
:104D700080FF17C02F2D247030E040E050E060E04D
:104D800070E080E090E0A0E00E94F99451F0EF0123
:104D900021964BE959E06BE075E0CF010E942512A6
:104DA000FE012F2D227030E040E050E060E070E026
:104DB00080E090E0A0E00E94F99451F0EF0121968C
:104DC0004BE959E06FE075E0CF010E942512FE012A
:104DD0002F2D287030E040E050E060E070E080E08F
:104DE00090E0A0E00E94F99451F0EF0121964BE988
:104DF00059E067E275E0CF010E942512FE012F2DD8
:104E0000207130E040E050E060E070E080E090E051
:104E1000A0E00E94F99451F0EF0121964BE959E08E
:104E200062E175E0CF010E942512FE012F2D207254
:104E300030E040E050E060E070E080E090E0A0E032
:104E40000E94F99451F0EF0121964BE959E065E198
:104E500075E0CF010E942512FE012F2D207430E055
:104E600040E050E060E070E080E090E0A0E00E9470
:104E7000F99451F0EF0121964BE959E06BE175E0AF
:104E8000CF010E942512FE012F2D207830E040E056
:104E900050E060E070E080E090E0A0E00E94F994D3
:104EA00051F0EF0121964BE959E061E275E0CF0145
:104EB0000E942512FE0120E0302F317040E050E0CA
:104EC00060E070E080E090E0A0E00E94F99451F092
:104ED000EF0121964BE959E064E275E0CF010E94B1
:104EE0002512FE0120E0302F327040E050E060E0FB
:104EF00070E080E090E0A0E00E94F99451F0EF01B2
:104F000021964BE959E069E275E0CF010E94251234
:104F1000FE0120E0302F347040E050E060E070E0AF
:104F200080E090E0A0E00E94F99451F0EF0121961A
:104F30004BE959E060E375E0CF010E942512FE01C4
:104F400020E0302F387040E050E060E070E080E01A
:104F500090E0A0E00E94F99451F0EF0121964BE916
:104F600059E063E375E0CF010E942512FE0120E0C5
:104F7000302F307140E050E060E070E080E090E081
:104F8000A0E00E94F99451F0EF0121964BE959E01D
:104F900068E375E0CF010E942512FE0120E0302F6A
:104FA000307240E050E060E070E080E090E0A0E02F
:104FB0000E94F99451F0EF0121964BE959E06FE31B
:104FC00075E0CF010E942512FE0120E030E040E0B4
:104FD00050E06D2D647070E080E090E0A0E00E94F1
:104FE000F99451F0EF0121964BE959E066E475E040
:104FF000CF010E942512FE018091CA2B81FF17C0AC
:1050000020E0302F307440E050E060E070E080E05D
:1050100090E0A0E00E94F99451F0EF0121964BE955
:1050200059E06AE475E0CF010E942512FE018091EB
:10503000CA2B9091CB2B90FF17C020E030E040E0CE
:105040005E2D507160E070E080E090E0A0E00E9492
:10505000F99451F0EF0121964BE959E06DE475E0C8
:10506000CF010E942512FE018091CA2B9091CB2B7B
:1050700090FF17C020E030E040E05E2D507260E00D
:1050800070E080E090E0A0E00E94F99451F0EF0120
:1050900021964BE959E060E575E0CF010E942512A9
:1050A000FE018091CA2B9091CB2B90FF17C020E07E
:1050B00030E040E05E2D507460E070E080E090E011
:1050C000A0E00E94F99451F0EF0121964BE959E0DC
:1050D00066E575E0CF010E942512FE0120E0302F29
:1050E000307840E050E060E070E080E090E0A0E0E8
:1050F0000E94F99451F0EF0121964BE959E061E6E5
:1051000075E0CF010E942512FE0120E030E0412F22
:10511000417050E060E070E080E090E0A0E00E942C
:10512000F99451F0EF0121964BE959E066E675E0FC
:10513000CF010E942512FE0120E030E0412F427095
:1051400050E060E070E080E090E0A0E00E94F99420
:1051500051F0EF0121964BE959E069E675E0CF0186
:105160000E942512FE0120E030E0412F447050E003
:1051700060E070E080E090E0A0E00E94F99451F0DF
:10518000EF0121964BE959E06CE675E0CF010E94F2
:105190002512FE018091CA2B87FF17C020E030E066
:1051A000412F487050E060E070E080E090E0A0E0C7
:1051B0000E94F99451F0EF0121964BE959E06FE616
:1051C00075E0CF010E942512FE018091CA2B87FF56
:1051D00017C020E030E0412F407150E060E070E007
:1051E00080E090E0A0E00E94F99451F0EF01219658
:1051F0004BE959E063E775E0CF010E942512FE01FB
:105200008091CA2B87FF17C020E030E0412F407209
:1052100050E060E070E080E090E0A0E00E94F9944F
:1052200051F0EF0121964BE959E067E775E0CF01B6
:105230000E942512FE018091CA2B87FF17C020E033
:1052400030E0412F407450E060E070E080E090E09A
:10525000A0E00E94F99451F0EF0121964BE959E04A
:105260006BE775E0CF010E942512FE018091CA2BE9
:1052700082FF17C020E030E0412F407850E060E02E
:1052800070E080E090E0A0E00E94F99451F0EF011E
:1052900021964BE959E069EA76E0CF010E94251298
:1052A000FE018091CA2B82FF17C020E030E040E071
:1052B0005E2D517060E070E080E090E0A0E00E9420
:1052C000F99451F0EF0121964BE959E06FE775E051
:1052D000CF010E942512FE018091CA2B9091CB2B09
:1052E00090FF17C020E030E040E05E2D527060E09B
:1052F00070E080E090E0A0E00E94F99451F0EF01AE
:1053000021964BE959E062E875E0CF010E94251231
:10531000FE018091CA2B9091CB2B90FF17C020E00B
:1053200030E040E05E2D547060E070E080E090E09E
:10533000A0E00E94F99451F0EF0121964BE959E069
:105340006AE875E0CF010E942512FE018091CA2B08
:105350009091CB2B91FF1EC020E030E040E05E2D0D
:10536000587060E070E080E090E0A0E00E94F99466
:1053700089F04BE959E063E975E0CF01DF91CF9106
:105380001F910F91FF90EF90DF90CF90BF90AF9063
:105390000C9425122F2D302F412F5E2D6D2D7A2D3F
:1053A0008B2D9C2DA0E00E94F99441F485E697E0B6
:1053B0009F938F930E948A990F900F90DF91CF91C6
:1053C0001F910F91FF90EF90DF90CF90BF90AF9023
:1053D00008958F929F92BF92DF92EF920F931F9347
:1053E000CF93DF93EC014B01FB01108260E677E085
:1053F0000E94AB98892B61F58091CA2B7DE4D72E52
:10540000E0E8EE2E82FD02C004E001C004E810E0F6
:10541000B12C81FF02C060ECE62E26E04AE250E0AB
:105420006BE270E089E290E00E94836381E090E0AB
:105430000E944E0D882311F05DE5D52E8091CA2B78
:105440009091CB2B90FD16E091FF07C0186005C02E
:10545000D12CE12C00E010E0B12C6EE577E0CE011C
:105460000E94AB98892B61F481E0F4018083609104
:105470007B0270917C0280E090E00E94BF98EC017A
:105480006CE577E0CE010E94AB98892B61F48FEF39
:10549000F401808360917B0270917C0280E090E057
:1054A0000E94BF98EC01209709F424C168E577E0D9
:1054B000CE010E94AB98892B19F4FD2DF160DF2EEF
:1054C00064E577E0CE010E94AB98892B19F48D2D0D
:1054D0008460D82E61E577E0CE010E94AB98892BDD
:1054E00019F4ED2DE260DE2E6FE477E0CE010E942C
:1054F000AB98892B19F4FD2DF860DF2E6CE477E072
:10550000CE010E94AB98892B19F48D2D8061D82E85
:1055100066E477E0CE010E94AB98892B19F4ED2D5B
:10552000E062DE2E60E477E0CE010E94AB98892B2A
:1055300019F4FD2DF064DF2E6DE377E0CE010E94BB
:10554000AB98892B19F48D2D8068D82E68E377E00D
:10555000CE010E94AB98892B19F4EE2DE160EE2E5E
:1055600061E377E0CE010E94AB98892B19F4FE2D00
:10557000F260EF2E6EE277E0CE010E94AB98892BAD
:1055800019F48E2D8460E82E69E277E0CE010E9446
:10559000AB98892B19F4EE2DE860EE2E62E277E0ED
:1055A000CE010E94AB98892B19F4FE2DF061EF2EED
:1055B0006BE177E0CE010E94AB98892B19F48E2D18
:1055C0008062E82E67E177E0CE010E94AB98892BDC
:1055D00019F4EB2DE460BE2E64E177E0CE010E9469
:1055E000AB98892B19F4FE2DF064EF2E6FE077E075
:1055F000CE010E94AB98892B19F48E2D8068E82E7D
:105600006CE077E0CE010E94AB98892B09F4016031
:1056100069E077E0CE010E94AB98892B09F4026023
:1056200066E077E0CE010E94AB98892B09F4046014
:1056300062E077E0CE010E94AB98892B09F4086004
:105640006EEF76E0CE010E94AB98892B09F40061E1
:105650006AEF76E0CE010E94AB98892B09F40062D4
:1056600066EF76E0CE010E94AB98892B09F40064C6
:1056700064EF76E0CE010E94AB98892B09F40068B4
:1056800061EF76E0CE010E94AB98892B09F411609E
:1056900069EE76E0CE010E94AB98892B09F4126086
:1056A00060EE76E0CE010E94AB98892B09F414607D
:1056B00067ED76E0CE010E94AB98892B09F4186063
:1056C00064ED76E0CE010E94AB98892B09F410615D
:1056D0006EEC76E0CE010E94AB98892B09F4106243
:1056E00063EC76E0CE010E94AB98892B09F0D2CE14
:1056F0001064D0CE2D2D3E2DA8016B2D70E080E0E2
:1057000090E0DF91CF911F910F91EF90DF90BF90CC
:105710009F908F9008955F926F927F928F929F9249
:10572000AF92BF92CF92DF92EF92FF920F931F93AF
:10573000CF93DF93782ECDEADBE100E010E0FDEBC4
:10574000EF2EF6E0FF2E8170582E872D8270682E86
:10575000A8EACA2EA6E0DA2EB0EBAB2EB6E0BB2E3E
:105760008EEA882E86E0982E772051F01F930F93B3
:10577000FF92EF920E948A990F900F900F900F90D6
:105780005520A1F089858F9388858F93BF92AF9222
:105790000E948A990F900F900F900F906620C1F091
:1057A0009F928F920E948A990F900F90662081F0AD
:1057B000DF92CF920E948A99288139814A815B8148
:1057C0006C817D818E819F810E9485260F900F9034
:1057D0000E94C00D0F5F1F4F2A960430110521F65D
:1057E000DF91CF911F910F91FF90EF90DF90CF90BD
:1057F000BF90AF909F908F907F906F905F90089533
:1058000083EA96E09F938F930E948A998091BA27AA
:105810009091BB27A091BC27B091BD270F900F900E
:10582000813027EA92072EE1A207B10519F485E934
:1058300096E01DC0823026EA92072EE1A207B1054C
:1058400019F488E896E013C0823027EA92072EE127
:10585000A207B10519F48AE796E009C0823028EA68
:1058600092072EE1A207B10549F48CE696E09F93DA
:105870008F930E948A990F900F900895BF93AF93D2
:105880009F938F9386E696E09F938F930E948A99C9
:105890000F900F900F900F900F900F90089586E546
:1058A00096E09F938F930E948A990E94B9220E944A
:1058B000002C0E94C00D84E99BE19F938F938EE49E
:1058C00096E09F938F930E948A9960915C027091F9
:1058D0005D0280915E0290915F0228EE33E040E02D
:1058E00050E00E94C1925F934F933F932F938EE3BA
:1058F00096E09F938F930E948A9985E396E09F9309
:105900008F930E948A990E944D128091CA2B2DB7C5
:105910003EB7225F3F4F0FB6F8943EBF0FBE2DBF7C
:1059200080FF05C041E061E081E00E94F71381E360
:1059300096E09F938F930E948A9980E00E9497241B
:105940000E94BD22809161021F928F9388E296E0AF
:105950009F938F930E948A9980913D0A1F928F9303
:105960008FE196E09F938F930E948A9980918D0298
:105970008F9380918C028F9380918B028F93809173
:105980008A028F9381E196E09F938F930E948A9978
:105990001F9280E48F9389EF95E09F938F930E94ED
:1059A0008A998091A4341F928F938091A3341F927F
:1059B0008F9386EE95E09F938F930E948A998091B2
:1059C00060021F928F938DED95E09F938F930E94BD
:1059D0008A998091620290916302A0916402B091D1
:1059E00065022DB73EB7225E3F4F0FB6F8943EBF1B
:1059F0000FBE2DBF96FF03C08CE995E002C08FE972
:105A000095E09F938F9383ED95E09F938F930E94F2
:105A10008A9983E00E948B2B0F900F900F900F902C
:105A20001D9B03C08CE995E002C08FE995E09F9330
:105A30008F9387EC95E09F938F930E948A998DEBCB
:105A400095E09F938F930E948A99809162020F90B4
:105A50000F900F900F900F900F9081FF09C087EB70
:105A600095E09F938F930E948A990F900F9013C097
:105A700080FF03C08CE995E002C08FE995E09F9319
:105A80008F9383EB95E09F938F930E948A990F9059
:105A90000F900F900F908091620290916302A091FD
:105AA0006402B091650297FF03C08CE995E002C0E3
:105AB0008FE995E09F938F938AEA95E09F938F9368
:105AC0000E948A9983EA95E09F938F930E948A9916
:105AD0006091410A7091420A8091430A9091440A70
:105AE0000E94D9240E94C00D0F900F900F900F902C
:105AF0000F900F90779903C08CE995E002C08FE971
:105B000095E09F938F938AE995E09F938F930E94EE
:105B10008A990E942F0A0E940A0D9F938F937F9368
:105B20006F938CE895E09F938F930E948A990E94CF
:105B3000B90C9F938F937F936F938EE795E09F931C
:105B40008F930E948A9981E090E00E947323809154
:105B5000793490917A34A0917B34B0917C34BF93A6
:105B6000AF939F938F9380E795E09F938F930E94CD
:105B70008A9980918E348F9380918D348F93809108
:105B80008C348F9380918B348F938CE595E09F9329
:105B90008F930E948A9980917D3490917E34A09158
:105BA0007F34B0918034BF93AF939F938F938EE4F3
:105BB00095E09F938F930E948A998DB79EB78296A6
:105BC0000FB6F8949EBF0FBE8DBF809192348F9315
:105BD000809191348F93809190348F9380918F3402
:105BE0008F938AE395E09F938F930E948A9961E057
:105BF00070E080E090E00E94C90D61E070E081E01B
:105C000090E00E94C90D0F900F900F900F900F9091
:105C10000F90299B03C08CE995E002C08FE995E0C5
:105C20009F938F9382E395E09F938F930E948A992D
:105C30000F900F900F900F902A9B03C08CE995E076
:105C400002C08FE995E09F938F938AE295E09F933E
:105C50008F930E948A990F900F900F900F90089544
:105C6000F894E0E0F0E081E2809357008491E2E074
:105C7000F0E041E2409357004491E4E0F0E091E22B
:105C800090935700E49190E0A0E0B0E0DC01992708
:105C9000882750E060E070E0762F652F542F44276E
:105CA000840F951FA61FB71F8E0F911DA11DB11D3B
:105CB0008093BA279093BB27A093BC27B093BD27AE
:105CC00078940895CF93DF93CDB7DEB761970FB681
:105CD000F894DEBF0FBECDBF48E250E062E270E054
:105CE0008DEA9BE10E94DE9A2091AD1B3091AE1BA4
:105CF0004091AF1B5091B01B6091B11B7091B21BD2
:105D00008091B31B9091B41BAFEF0E94F99409F0FE
:105D10005DC08DE48093AD1B80E88093AE1B84E072
:105D20008093AF1B1092B01B1092B11B1092B21B4C
:105D30001092B31B1092B41B8CE390E09093B61BAF
:105D40008093B51B1092B71B1092B81B1092B91B11
:105D50001092BA1B1092BB1B1092BC1B1092BD1B61
:105D60001092BE1B1092C01B1092BF1B1092C11B41
:105D70001092C21B1092C31B1092C41B1092C51B21
:105D80001092C61B1092C71B1092C81B1092CA1B00
:105D90001092C91B1092CB1B1092CC1B1092CD1BE2
:105DA0001092CE1B1092CF1B1092D01B1092D11BC1
:105DB0001092D21B1092D41B1092D31B48E250E0D9
:105DC00062E270E08DEA9BE10E94FC9A44E050E0C0
:105DD0006EE170E0CE010B960E94DE9A8B859C8569
:105DE000AD85BE858F3F2FEF9207A207B207A9F4BA
:105DF0008AE090E4A0E0B0E08093620290936302B6
:105E0000A0936402B093650244E050E06EE170E05C
:105E100082E692E00E94FC9A08C08093620290930E
:105E20006302A0936402B093650280916202909134
:105E30006302A0916402B0916502A2FF02C02A9A97
:105E400003C080E00E94CD2444E050E06AE570E0A9
:105E5000CE010B960E94DE9A8B859C85AD85BE8512
:105E60008F3F2FEF9207A207B20789F41092410AE1
:105E70001092420A1092430A1092440A44E050E001
:105E80006AE570E081E49AE00E94FC9A08C0809381
:105E9000410A9093420AA093430AB093440A49E00E
:105EA00050E06EE070E083E994E30E94DE9A0E9485
:105EB000010F44E050E06EE470E0CE010B960E94CA
:105EC000DE9A8B859C85AD85BE8544E050E06EE40E
:105ED00070E08F3F9F4FAF4FBF4F29F482E892E0B1
:105EE0000E94FC9A04C082E892E00E94DE9A44E09C
:105EF00050E06AE470E0CE010B960E94DE9A8B853A
:105F00009C85AD85BE8544E050E06AE470E08F3F3B
:105F10009F4FAF4FBF4F29F48EE792E00E94FC9A4B
:105F200004C08EE792E00E94DE9A44E050E062E511
:105F300070E0CE010B960E94DE9A8B859C85AD8524
:105F4000BE8544E050E062E570E08F3F9F4FAF4F69
:105F5000BF4F29F486E892E00E94FC9A04C086E8CC
:105F600092E00E94DE9A41E050E06DE170E0CE01E7
:105F700041960E94DE9A898941E050E06DE170E02F
:105F80008F3F29F48DE39AE00E94FC9A04C08DE3D0
:105F90009AE00E94DE9A41E050E06CE170E0CE01B0
:105FA00041960E94DE9A898941E050E06CE170E000
:105FB0008F3F29F481E692E00E94FC9A04C081E6BA
:105FC00092E00E94DE9A41E050E06BE170E0CE0189
:105FD00041960E94DE9A898941E050E06BE170E0D1
:105FE0008F3F29F480E692E00E94FC9A04C080E68C
:105FF00092E00E94DE9A4AE050E064E070E0CE0158
:1060000001960E94DE9A89814AE050E064E070E0E7
:106010008F3F29F484E99BE10E94FC9A04C084E943
:106020009BE10E94DE9A44E050E066E570E0CE011C
:106030000B960E94DE9A8B859C85AD85BE8544E0DB
:1060400050E066E570E08F3F9F4FAF4FBF4F29F4A0
:106050008AE892E00E94FC9A04C08AE892E00E94DA
:10606000DE9A44E050E067E170E0CE010B960E94BA
:10607000DE9A8B859C85AD85BE8544E050E067E166
:1060800070E08F3F9F4FAF4FBF4F29F48CE592E0F8
:106090000E94FC9A04C08CE592E00E94DE9A42E0E5
:1060A00050E062E070E0CE010F960E94DE9A8F858C
:1060B000988942E050E062E070E08F3F910529F45A
:1060C00088E39AE00E94FC9A04C088E39AE00E9468
:1060D000DE9A42E050E060E070E0CE010F960E9450
:1060E000DE9A8F85988942E050E060E070E08F3F53
:1060F000910529F486E39AE00E94FC9A04C086E3A5
:106100009AE00E94DE9A61960FB6F894DEBF0FBE49
:10611000CDBFDF91CF910895CF92DF92EF92FF92A2
:1061200060917B0270917C0280E090E00E94BF98B9
:1061300063EA75E00E94D398892B09F03BC18DE496
:106140008093AD1B80E88093AE1B84E08093AF1BEF
:106150001092B01B1092B11B1092B21B1092B31B85
:106160001092B41B8CE390E09093B61B8093B51B08
:106170001092B71B1092B81B1092B91B1092BA1B49
:106180001092BB1B1092BC1B1092BD1B1092BE1B29
:106190001092C01B1092BF1B1092C11B1092C21B09
:1061A0001092C31B1092C41B1092C51B1092C61BE9
:1061B0001092C71B1092C81B1092CA1B1092C91BC9
:1061C0001092CB1B1092CC1B1092CD1B1092CE1BA9
:1061D0001092CF1B1092D01B1092D11B1092D21B89
:1061E0001092D41B1092D31B48E250E062E270E0A0
:1061F0008DEA9BE10E94FC9A8AE090E4A0E0B0E086
:106200008093620290936302A0936402B09365024C
:1062100044E050E06EE170E082E692E00E94FC9A79
:106220001092410A1092420A1092430A1092440AB4
:1062300044E050E06AE570E081E49AE00E94FC9A54
:1062400042E2C42EDD24DA944CECE42E4BE3F42E2F
:10625000C0928202D0928302E0928402F092850280
:1062600044E050E06EE470E082E892E00E94FC9A24
:10627000C0927E02D0927F02E0928002F092810270
:1062800044E050E06AE470E08EE792E00E94FC9AFD
:1062900087ED94E3AFEEBCE3809386029093870290
:1062A000A0938802B093890244E050E062E570E078
:1062B00086E892E00E94FC9A8AE999E9A9E1B0E4B3
:1062C00080938A0290938B02A0938C02B0938D02EC
:1062D00044E050E066E570E08AE892E00E94FC9AB3
:1062E00010923D0A80E00E94FE7041E050E06DE1B6
:1062F00070E08DE39AE00E94FC9A8AE1809361024B
:106300000E94A56F41E050E06CE170E081E692E010
:106310000E94FC9A8FE08093600241E050E06BE1C4
:1063200070E080E692E00E94FC9A8AE0E4E9FBE1FA
:10633000DF011D928A95E9F74AE050E064E070E0E1
:10634000CF010E94FC9A80EA96E8A1E0B0E0809339
:106350005C0290935D02A0935E02B0935F0244E002
:1063600050E067E170E08CE592E00E94FC9A1092A8
:10637000390A1092380A42E050E062E070E088E3A7
:106380009AE00E94FC9A1092370A1092360A42E074
:1063900050E060E070E086E39AE00E94FC9A81E0C1
:1063A0000E94972480E090E0FF90EF90DF90CF90E4
:1063B0000C94150FFF90EF90DF90CF9008950E94FE
:1063C000036D6C9A6B9A6A9A6F9A729A749A739A1E
:1063D000779A809880B3897F80BB8398849887E080
:1063E00080937E00549A0E94302E0E94622E81E09B
:1063F0000E94C20B80E090E00E94150F60915C0249
:1064000070915D0280915E0290915F020E946966C8
:106410000E94B90C6093CC2F7093CD2F8093CE2F18
:106420009093CF2F8091620286FD239A219A229A1F
:10643000239A0E949D0A1D9B05C010923F0A10924C
:106440003E0A089581E090E090933F0A80933E0ACF
:1064500008950F931F93CF93DF939DE8899FE001E9
:106460001124CA54D34E4091410A5091420A60917E
:10647000430A7091440A41FD08C08091620280FD88
:1064800004C081FF89C01D9B87C0CE0104969F93E5
:106490008F938AEA95E09F938F930E947899FE01EB
:1064A000ED57FF4F80810F900F900F900F90088154
:1064B00019812A813B81882309F440C04091D02F63
:1064C0005091D12F6091D22F7091D32F401B510B3F
:1064D000620B730B7F936F935F934F933896918109
:1064E0009F9390819F93329791819F9390819F93E7
:1064F000339790811F929F93319790811F929F9322
:10650000339690811F929F93319790811F929F9312
:10651000CC57DF4F98811F929F931F928F9380EBF0
:1065200095E09F938F930E9478998DB79EB746967A
:106530000FB6F8949EBF0FBE8DBF1CC08091D02FA8
:106540009091D12FA091D22FB091D32F801B910B7E
:10655000A20BB30BBF93AF939F938F9387EF95E0FD
:106560009F938F930E9478990F900F900F900F90A8
:106570000F900F900E94C00D80917D02882361F0E2
:106580001F928F9383EE91E09F938F930E948A993D
:106590000F900F900F900F90DF91CF911F910F915F
:1065A00008958091B31C882341F08091B41C90E041
:1065B0000E9429320E948B0BF4CF0895CF93DF9372
:1065C000EC0188819981823D2EE09207E9F018F470
:1065D000892BB9F048C08A3D2EE0920709F449C0E2
:1065E0008E3D9E4009F03FC083E59AE00E94AE5D7B
:1065F000892BE9F183E59AE00E94915D80E00E9499
:10660000C72482ED9EE02CC0623189F5299A609101
:10661000360A7091370A7695762F662777956795B3
:1066200083E59AE00E94875D4091410A5091420AB9
:106630006091430A7091440A60FF10C08091370A4C
:106640008F938091360A8F938CE790E19F938F937D
:106650000E948A990F900F900F900F908AED9EE004
:106660009983888304C01982188283E017C081E06F
:1066700015C083E59AE00E94AE5D892BC1F383E5E6
:106680009AE00E94915D0E94D13260E270E083E561
:106690009AE00E94875D8EED9EE0E2CFDF91CF9180
:1066A00008952F923F924F925F926F927F928F92B6
:1066B0009F92AF92BF92CF92DF92EF92FF920F9391
:1066C0001F93CF93DF93CDB7DEB72B970FB6F89418
:1066D000DEBF0FBECDBF9B878A874A01FC01808148
:1066E0009181892B11F00C94AA4760917B027091E3
:1066F0007C02CA010E94BF9860E870E0C4010E9459
:10670000F298009759F460915E3D70915F3D8AE088
:1067100090E00E94469981E00C94AF47813091054A
:1067200061F4F401B0801B2D110F110B012F412ECC
:10673000512E612E712EA12EBCC082309105B9F46C
:10674000F4018081992787FD9095982F88272181D2
:10675000820F911D27FD9A95B82E192F092F000F32
:10676000000B402E502E602E702EA02EA2C0833023
:106770009105B1F5F4012081922F990F990B392FD2
:10678000492F592F692F792F892F00E10E949B945F
:1067900019012A013B01B82FA92F2181922F990FAE
:1067A000990B392F492F592F692F792F892F08E0FD
:1067B0000E949B9459016A017B018C019101A20105
:1067C000B3018B2F9A2F0E94D294A2801A2D110F01
:1067D000110BB12EC12ED12EE12EF12E012F55C05D
:1067E00004970CF45DC0F4012081922F990F990B4E
:1067F000392F492F592F692F792F892F08E10E94AE
:106800009B9419012A013B01B82FA92F2181922FB6
:10681000990F990B392F492F592F692F792F892FCC
:1068200000E10E949B9459016A017B018C01910156
:10683000A201B3018B2F9A2F0E94D294A3801A2D0C
:10684000110F110BB12EC12ED12EE12EF12E012FE1
:106850000E94D29419012A013B01B82FA92F22814D
:10686000922F990F990B392F492F592F692F792F73
:10687000892F08E00E949B9459016A017B018C01D9
:106880009101A201B3018B2F9A2F0E94D294B22EB4
:10689000132F042F452E562E672E782EA92E09C0B1
:1068A000EAE0BE2E10E000E0412C512C612C712C4E
:1068B000A12C0E94C00D2B2D312F402F542D652D62
:1068C000762D872D9A2D2537F3E63F07FDE64F07F6
:1068D0005105610571058105910511F40C949242F1
:1068E0002537E3E63E07EDE64E07510561057105E4
:1068F0008105910511F008F0C0C12337F2E73F0789
:1069000041055105610571058105910511F40C944E
:1069100025452337E2E73E0741055105610571052D
:106920008105910511F008F0BFC02536F4E63F0758
:1069300041055105610571058105910509F4F9C706
:106940002536E4E63E0741055105610571058105DF
:10695000910511F008F043C0A6E70E94F99411F4E4
:106960000C941B3F0E94F99409F070F4A8E60E9471
:10697000F99411F40C94EA3CA5E70E94F99411F4FF
:106980000C94053F0C94A8472B2D312F402F542DEC
:10699000652D762D872D9A2D2436F1E63F0741058A
:1069A0005105610571058105910511F40C944D4562
:1069B0002537E2E63E074105510561057105810570
:1069C000910509F44DC52A3336424105510561054B
:1069D00071058105910509F44CC30C94A8472B2D32
:1069E000312F402F542D652D762D872D9A2D273749
:1069F000EFE63E07410551056105710581059105E9
:106A000011F40C94F8422737FFE63F074105510582
:106A1000610571058105910509F0C8F42436E9E6A0
:106A20003E0741055105610571058105910511F488
:106A30000C94DE3E25363E46410551056105710543
:106A40008105910511F40C942C430C94A8472B2D2F
:106A5000312F402F542D652D762D872D9A2D2536DB
:106A6000E2E73E0741055105610571058105910584
:106A700011F40C94F6432936F2E73F07410551051E
:106A8000610571058105910511F40C94D4442333FB
:106A9000314741055105610571058105910511F0E9
:106AA0000C94A8470C944D452B2D312F402F542D7D
:106AB000652D762D872D9A2D2236F5E63F07F4E6D3
:106AC0004F075105610571058105910509F431C72D
:106AD0002236E5E63E07E4E64E07510561057105FD
:106AE0008105910511F008F05DC02133F4E63F0700
:106AF000F1E64F075105610571058105910509F41E
:106B0000CCC22133E4E63E07E1E64E0751056105BC
:106B100071058105910509F0C0F42337F3E73F07BC
:106B200041055105610571058105910511F40C942C
:106B300039452837344741055105610571058105FF
:106B4000910509F496C20C94A8472B2D312F402FA4
:106B5000542D652D762D872D9A2D2837F4E63F0785
:106B6000F1E64F075105610571058105910509F4AD
:106B700090C22C36E5E73E07E2E64E075105610577
:106B800071058105910509F46BC4233634464146ED
:106B90005105610571058105910511F00C94A84717
:106BA0000C944D452B2D312F402F542D652D762DD6
:106BB000872D9A2D2D36E5E73E07E8E64E0751056D
:106BC000610571058105910511F40C9463452D361D
:106BD000F5E73F07F8E64F075105610571058105A7
:106BE000910509F0E0F42237E2E73E07E5E64E07BB
:106BF0005105610571058105910511F40C9443421D
:106C000023363D46484651056105710581059105CC
:106C100011F00C94A8470E9453180C94AA472B2DEE
:106C2000312F402F542D652D762D872D9A2D24360A
:106C3000E3E63E07ECE64E07510561057105810567
:106C4000910511F40C94A6412736FFE63F07FCE6B8
:106C50004F075105610571058105910511F40C94EB
:106C6000A941233632434946510561057105810525
:106C7000910511F00C94A84730C22B2D312F402FD5
:106C8000542D652D762D872D9A2D2037FCE63F0754
:106C9000F5E64F07F8E65F07610571058105910587
:106CA00009F498C62037ECE63E07E5E64E07E8E62D
:106CB0005E07610571058105910511F008F0E6C0D8
:106CC0002437F8E73F07F4E74F07510561057105E1
:106CD0008105910511F40C94873F2437E8E73E07BE
:106CE000E4E74E075105610571058105910511F035
:106CF00008F05FC02033F1E33F07F1E74F0751058C
:106D0000610571058105910511F40C94434220330E
:106D1000E1E33E07E1E74E07510561057105810595
:106D2000910509F0C0F42133F2E63F07F0E74F0781
:106D30005105610571058105910509F4A6C222334B
:106D4000324640475105610571058105910509F4F9
:106D5000F1C20C94A8472B2D312F402F542D652DB7
:106D6000762D872D9A2D2037F5E63F07F2E74F075E
:106D70005105610571058105910511F40C94F643E7
:106D80002C36E4E73E074E07510561057105810584
:106D9000910511F40C94D1462133314341475105FB
:106DA000610571058105910511F00C94A8470C94BB
:106DB00092422B2D312F402F542D652D762D872D6E
:106DC0009A2D2B36ECE63E07E5E74E07E2E65E0736
:106DD000610571058105910509F442C32B36FCE676
:106DE0003F07F5E74F07F2E65F076105710581058B
:106DF000910509F0E0F42437E4E63E07E7E74E07A3
:106E00005105610571058105910511F40C941F4729
:106E100024373F464F46524661057105810591056D
:106E200011F00C94A8470C9400000C94AA472B2D49
:106E3000312F402F542D652D762D872D9A2D2E36EE
:106E4000E1E63E07E8E64E07E3E65E076105710509
:106E50008105910511F40C945B3F2633F9E63F0759
:106E6000F5E74F07F5E65F076105710581059105B7
:106E700009F4B4C529363C464146534661057105BF
:106E80008105910511F00C94A84791C32B2D312F4A
:106E9000402F542D652D762D872D9A2D2437F3E71D
:106EA0003F07F5E64F07F2E75F07610571058105CA
:106EB000910511F40C94A6432437E3E73E07E5E679
:106EC0004E07E2E75E07610571058105910511F046
:106ED00008F064C02337F5E63F07F2E74F07F0E715
:106EE0005F07610571058105910511F40C94134646
:106EF0002337E5E63E07E2E74E07E0E75E07610578
:106F000071058105910509F0D0F42136FDE63F07B2
:106F1000F5E74F07F8E65F07610571058105910503
:106F200011F40C9416432237374740475047610508
:106F300071058105910509F462C20C94A8472B2DB7
:106F4000312F402F542D652D762D872D9A2D2436E7
:106F5000FDE63F07F3E64F07F2E75F0761057105BE
:106F60008105910509F445C62136ECE63E07E5E6C4
:106F70004E07E2E75E07610571058105910509F499
:106F80004AC5233732474747504761057105810598
:106F9000910511F00C94A8470C94A9432B2D312F87
:106FA000402F542D652D762D872D9A2D2437E2E71D
:106FB0003E07E1E64E07E5E75E07610571058105DD
:106FC000910509F471C62437F2E73F07F1E64F0750
:106FD000F5E75F07610571058105910509F0C8F4C2
:106FE0002437E3E73E07E5E64E07E4E75E07610581
:106FF00071058105910509F4B5C727373047484722
:107000005447610571058105910509F42AC70C945F
:10701000A8472B2D312F402F542D652D762D872DF0
:107020009A2D2F36ECE63E07EFE54E07E6E75E07C2
:10703000610571058105910509F486C52C36F1E6D7
:107040003F07F4E74F07F8E75F0761057105810522
:10705000910511F40C949B4622373746404755471B
:10706000610571058105910511F00C94A8470C94F8
:10707000814183E080938134109283341092823472
:1070800041E854E362E18EE392E00E94085B0C94D5
:10709000AA470E94DB170C94AA4721E042E161E075
:1070A00080ED0E94426821E042E161E080ED0E94B3
:1070B000426821E042E161E080ED0E94426821E007
:1070C00042E161E080ED0E94426821E042E161E03E
:1070D00080ED0E9442680C94AA4760917B027091F7
:1070E0007C0280E090E00E94BF9863E076E00E941E
:1070F000D398892B09F0C5C060917B0270917C0206
:1071000080E090E00E94BF985C01009709F497C06E
:107110006CEE73E00E94D398892BE1F488EE93E043
:10712000A0E0B0E080935C0290935D02A0935E02C9
:10713000B0935F0268EE73E080E090E00E946966C1
:1071400044E050E067E170E08CE592E00E94FC9A38
:107150000C94AA4769E076E0C5010E94D398892B78
:10716000E1F480E197E2A0E0B0E080935C029093CC
:107170005D02A0935E02B0935F0260E177E280E07F
:1071800090E00E94696644E050E067E170E08CE5C1
:1071900092E00E94FC9A0C94AA476CE076E0C5014C
:1071A0000E94D398892BE1F480EA96E8A1E0B0E050
:1071B00080935C0290935D02A0935E02B0935F02A5
:1071C00060EA76E881E090E00E94696644E050E081
:1071D00067E170E08CE592E00E94FC9A0C94AA476B
:1071E00060E176E0C5010E94D398892BE1F480E844
:1071F0009AE1A6E0B0E080935C0290935D02A093D8
:107200005E02B0935F0260E87AE186E090E00E945F
:10721000696644E050E067E170E08CE592E00E942E
:10722000FC9A0C94AA4782E693E09F938F930E9466
:107230008A990E94C00D0F900F900C94AA476091FC
:107240005C0270915D0280915E0290915F0228EE77
:1072500033E040E050E00E94C1925F934F933F9330
:107260002F938EE593E09F938F930E948A990E94BB
:10727000C00D0F900F900F900F900F900F900C94E7
:10728000AA470E944D120C94AA4760917B0270910C
:107290007C0280E090E00E94BF988C016CE975E070
:1072A0000E94D398892BA1F480916202909163028D
:1072B000A0916402B0916502A260809362029093F3
:1072C0006302A0936402B0936502299A0C94AA47C2
:1072D0006FE975E0C8010E94D398892BB1F48091C1
:1072E000620290916302A0916402B0916502AD7F49
:1072F0008093620290936302A0936402B09365024C
:1073000080E00E94C7240C94AA47299B03C08CE903
:1073100095E002C08FE995E09F938F9386E593E017
:107320009F938F930E948A990F900F900F900F90C8
:107330000C94AA4760917B0270917C0280E090E0FF
:107340000E94BF988C016CE975E00E94D398892B4C
:10735000E1F48091620290916302A0916402B09185
:107360006502A4608093620290936302A09364021A
:10737000B09365022A9A44E050E06EE170E082E644
:1073800092E00E94FC9A0C94AA476FE975E0C8014C
:107390000E94D398892BF1F480916202909163024C
:1073A000A0916402B0916502AB7F809362029093DA
:1073B0006302A0936402B093650280E00E94CD2432
:1073C00044E050E06EE170E082E692E00E94FC9AB8
:1073D0000C94AA472A9B03C08CE995E002C08FE970
:1073E00095E09F938F938EE493E09F938F930E94F9
:1073F0008A990F900F900F900F900C94AA4760916C
:107400007B0270917C0280E090E00E94BF988C012A
:107410006CE975E00E94D398892B19F477980C9445
:10742000AA476FE975E0C8010E94D398892B19F427
:10743000779A0C94AA47779903C08CE995E002C02B
:107440008FE995E09F938F9384E195E09F938F93CD
:107450000E948A990F900F900F900F900C94AA475A
:1074600060917B0270917C0280E090E00E94BF9866
:107470008C0164E176E00E94D398892BD1F480914D
:10748000B31C1F928F938091B51C1F928F93809194
:10749000B41C1F928F931F9284E18F9384E293E038
:1074A0009F938F930E948A990FB6F894DEBF0FBE08
:1074B000CDBF69E176E0C8010E94D398892B19F409
:1074C0000E94D13270C061E276E0C8010E94D39878
:1074D000892B09F047C060917B0270917C0280E0AB
:1074E00090E00E94BF98009709F45DC00E94AD979C
:1074F0008531910570F59093390A8093380A42E0FE
:1075000050E062E070E088E39AE00E94FC9A6091AB
:107510007B0270917C0280E090E00E94BF9800970F
:1075200009F441C00E94AD979093370A8093360AC0
:1075300042E050E060E070E086E39AE00E94FC9A4E
:1075400060917B0270917C0280E090E00E94BF9885
:107550002AC082E193E09F938F930E948A990F90B3
:107560000F9021C08091390A8F938091380A8F93B0
:1075700089E093E09F938F930E948A990E94C00DA7
:107580008091370A8F938091360A8F938AEF92E029
:107590009F938F930E948A990E94C00D0FB6F89412
:1075A000DEBF0FBECDBF0E94C00D0C94AA476091F4
:1075B0007B0270917C0280E090E00E94BF988C0179
:1075C00066E675E00E94D398892B09F077C0609138
:1075D0007B0270917C0280E090E00E94BF988C0159
:1075E000009711F40C94AA476FE176E00E94D398BB
:1075F000892BB1F482E29FEFACECBBE38093820273
:1076000090938302A0938402B093850244E050E0FB
:107610006EE470E082E892E00E94FC9A0C94AA4723
:1076200065E276E0C8010E94D398892BB1F482E22A
:107630009FEFACECBAE38093820290938302A09315
:107640008402B093850244E050E06EE470E082E88A
:1076500092E00E94FC9A0C94AA47C8010E94A99744
:107660002B013C0120E030E0A9010E94388F8823E3
:10767000D9F081E00E94560C9B01AC01C301B2011C
:107680000E943C8F609382027093830280938402F5
:107690009093850244E050E06EE470E082E892E06E
:1076A0000E94FC9A0C94AA478DEE92E09F938F93D0
:1076B0000E948A990F900F900C94AA4769E675E092
:1076C000C8010E94D398892B09F077C060917B0292
:1076D00070917C0280E090E00E94BF988C0100973E
:1076E00011F40C94AA476FE176E00E94D398892B9D
:1076F000B1F482E29FEFACECBBE380937E02909307
:107700007F02A0938002B093810244E050E06AE4DB
:1077100070E08EE792E00E94FC9A0C94AA4765E222
:1077200076E0C8010E94D398892BB1F482E29FEFE2
:10773000ACECBAE380937E0290937F02A093800228
:10774000B093810244E050E06AE470E08EE792E09A
:107750000E94FC9A0C94AA47C8010E94A9972B0189
:107760003C0120E030E0A9010E94388F8823D9F045
:1077700082E00E94560C9B01AC01C301B2010E9441
:107780003C8F60937E0270937F028093800290937F
:10779000810244E050E06AE470E08EE792E00E94EB
:1077A000FC9A0C94AA4780EE92E09F938F930E94DC
:1077B0008A990F900F900C94AA4761E675E0C80172
:1077C0000E94D398892B09F073C060917B0270915D
:1077D0007C0280E090E00E94BF988C01009711F439
:1077E0000C94AA476FE176E00E94D398892BB1F4FC
:1077F00087ED94E3AFEEBCE380938602909387021B
:10780000A0938802B093890244E050E062E570E002
:1078100086E892E00E94FC9A0C94AA4765E276E022
:10782000C8010E94D398892B51F481ED92E09F9377
:107830008F930E948A990F900F900C94AA47C801C9
:107840000E94A9972B013C0120E030E0A9010E9491
:10785000388F882319F180E00E94560C4B015C019F
:1078600021EE3AE744E95EE3C301B2010E94718E62
:10787000A50194010E943C8F609386027093870259
:10788000809388029093890244E050E062E570E0C2
:1078900086E892E00E94FC9A0C94AA4784EC92E05D
:1078A0009F938F930E948A990F900F900C94AA47F0
:1078B0000E94A50C9F938F937F936F938DEB92E023
:1078C0009F938F930E948A9982E00E94560C209188
:1078D0007E0230917F0240918002509181020E948D
:1078E000BD91162F072FF82EE92E81E00E94560C2D
:1078F000EF92FF920F931F932091820230918302A7
:1079000040918402509185020E94BD919F938F9374
:107910007F936F9381EB92E09F938F930E948A995C
:107920000E94C00D0FB6F894DEBF0FBECDBF0C9401
:10793000AA4760917B0270917C0280E090E00E94F7
:10794000BF98009711F10E94CC258090410A909039
:10795000420AA090430AB090440A681579058A0546
:107960009B0539F16093410A7093420A8093430A60
:107970009093440A44E050E06AE570E081E49AE0C4
:107980000E94FC9A8DE095E002C086E095E09F930E
:107990008F930E948A996091410A7091420A809166
:1079A000430A9091440A0E94D9240E94C00D0F906E
:1079B0000F908BEF94E09F938F930E948A996FEFC3
:1079C0007FEFCB010E94D9240E94C00D0F900F9031
:1079D0000C94AA470E94B6210C94AA47F401848112
:1079E000843329F440E061E080E00E94F713809145
:1079F0007D02882311F40C94AA471F928F9388EF7D
:107A000094E09F938F930E948A990F900F900F900C
:107A10000F900C94AA47F4018481893709F080C043
:107A200060917B0270917C0280E090E00E94BF98A0
:107A30008C016CE975E00E94D398892B51F48091F8
:107A4000620290916302A0916402B0916502906419
:107A500010C06FE975E0C8010E94D398892BD1F45A
:107A60008091620290916302A0916402B0916502DC
:107A70009F7B8093620290936302A0936402B09311
:107A8000650244E050E06EE170E082E692E00E9420
:107A9000FC9A46C06AE276E0C8010E94D398892B1E
:107AA00021F58091AC1B8F938091AB1B8F938091BC
:107AB000AA1B8F938091A91B8F938091A81B8F93F2
:107AC0008091A71B8F938091A61B8F938091A51BFC
:107AD0008F9386E892E09F938F930E948A990FB6C6
:107AE000F894DEBF0FBECDBF1BC0809162029091A3
:107AF0006302A0916402B091650296FF03C08CE915
:107B000095E002C08FE995E09F938F9382E892E021
:107B10009F938F930E948A990F900F900F900F90D0
:107B200080917D02882311F40C94AA471F928F93B1
:107B300085EF94E09F938F930E948A990F900F9006
:107B40000F900F900C94AA47F40184818737E9F5D0
:107B500060917B0270917C0280E090E00E94BF986F
:107B60000097D9F00E94A9972B013C0120E030E05A
:107B7000A9010E94388F882381F040928A02509296
:107B80008B0260928C0270928D0244E050E066E5B8
:107B900070E08AE892E00E94FC9A80918D028F93B7
:107BA00080918C028F9380918B028F9380918A02B7
:107BB0008F9384E792E09F938F930E948A990F900E
:107BC0000F900F900F900F900F9080917D0288235F
:107BD00011F40C94AA471F928F9382EF94E09F9325
:107BE0008F930E948A990F900F900F900F900C9492
:107BF000AA4760917B0270917C0280E090E00E9435
:107C0000BF988C016CE975E00E94D39840906202A5
:107C1000509063026090640270906502892B19F4A1
:107C2000689457F809C06FE975E0C8010E94D398BD
:107C3000892B99F4E89457F84092620250926302BB
:107C4000609264027092650244E050E06EE170E080
:107C500082E692E00E94FC9A13C057FE03C08CE9B2
:107C600095E002C08FE995E09F938F9380E792E0C3
:107C70009F938F930E948A990F900F900F900F906F
:107C800080917D02882311F40C94AA471F928F9350
:107C90008FEE94E09F938F930E948A990F900F909C
:107CA0000F900F900C94AA4760917B0270917C0218
:107CB00080E090E00E94BF985C0160E376E00E9463
:107CC000D398892B11F489E108C064E376E0C501FB
:107CD0000E94D398892B49F480E18093C4001092CC
:107CE000C50082E08093C00055C068E376E0C5011E
:107CF0000E94D398892B11F488E0EFCF6DE376E0F2
:107D0000C5010E94D398892B39F062E476E0C50161
:107D10000E94D398892B11F483E0DFCF8091C400B7
:107D2000893141F48BE692E09F938F930E948A9968
:107D30000F900F908091C400803141F486E692E06C
:107D40009F938F930E948A990F900F908091C40007
:107D5000883041F480E692E09F938F930E948A9945
:107D60000F900F908091C400833041F48AE592E037
:107D70009F938F930E948A990F900F908091C400D7
:107D8000883041F484E592E09F938F930E948A9912
:107D90000F900F9080917D02882311F40C94AA47D4
:107DA0001F928F938CEE94E09F938F930E948A99F9
:107DB0000F900F900F900F900C94AA4760917B0248
:107DC00070917C0280E090E00E94BF986FE176E0C5
:107DD0000E94D398892B11F481E001C080E00E94B9
:107DE000972480917D02882311F40C94AA471F9256
:107DF0008F9389EE94E09F938F930E948A990F90BE
:107E00000F900F900F900C94AA470E94BD22809172
:107E10007D02882311F40C94AA471F928F9386EE5B
:107E200094E09F938F930E948A990F900F900F90E8
:107E30000F900C94AA470E94B92280917D0288235A
:107E400011F40C94AA471F928F9383EE94E09F93B2
:107E50008F930E948A990F900F900F900F900C941F
:107E6000AA4760917B0270917C0280E090E00E94C2
:107E7000BF980E94AD97803170F480933D0A0E94B4
:107E8000FE7041E050E06DE170E08DE39AE00E9409
:107E9000FC9A0C94AA4780913D0A1F928F938AE422
:107EA00092E09F938F930E948A990F900F900F906A
:107EB0000F900C94AA4760917B0270917C0280E045
:107EC00090E00E94BF980E94AD9795EF980F903177
:107ED00070F4809361020E94A56F41E050E06CE174
:107EE00070E081E692E00E94FC9A0C94AA4780918F
:107EF00061021F928F9381E492E09F938F930E947F
:107F00008A990F900F900F900F900C94AA47609150
:107F10007B0270917C0280E090E00E94BF98009705
:107F200089F04AE050E0BC0184E99BE10E94E398BB
:107F30004AE050E064E070E084E99BE10E94FC9A32
:107F40000C94AA4784E99BE19F938F9387E496E082
:107F50009F938F930E9478990F900F900F900F909E
:107F60000C94AA4760917B0270917C0280E090E0C3
:107F70000E94BF985C016CEE73E00E94D398892B3D
:107F8000D9F4219A8091620290916302A0916402D7
:107F9000B091650280618093620290936302A09326
:107FA0006402B093650244E050E06EE170E082E666
:107FB00092E00E94FC9ACEC76AE675E0C5010E9475
:107FC000D398892BD9F4229A80916202909163020E
:107FD000A0916402B09165028062809362029093E6
:107FE0006302A0936402B093650244E050E06EE146
:107FF00070E082E692E00E94FC9AACC76EEC73E0FF
:10800000C5010E94D398892BD9F4239A80916202EA
:1080100090916302A0916402B091650280648093A4
:10802000620290936302A0936402B093650244E0FD
:1080300050E06EE170E082E692E00E94FC9A8AC70E
:108040006DE075E0C5010E94D398892BD9F4239A7D
:108050008091620290916302A0916402B0916502E6
:1080600080688093620290936302A0936402B0934D
:10807000650244E050E06EE170E082E692E00E942A
:10808000FC9A68C764EE79E0C5010E94D398892BF9
:1080900071F581E08093E52F8DEA9BE19093E72FC6
:1080A0008093E62F1092E92F1092E82F80916202C0
:1080B00090916302A0916402B091650291608093F7
:1080C000620290936302A0936402B093650244E05D
:1080D00050E06EE170E082E692E00E94FC9A45EE8C
:1080E0005FE262E18EE392E00E94085B33C765EFD6
:1080F00073E0C5010E94D398892B11F5EDEDFBE1EA
:10810000119211922BE1ED3FF207D1F780916202BB
:1081100090916302A0916402B09165029260809395
:10812000620290936302A0936402B093650244E0FC
:1081300050E06EE170E082E692E00E94FC9A0AC78D
:108140006FE975E0C5010E94D39840916202509199
:1081500063026091640270916502892BC1F44F70D3
:108160005C7F409362025093630260936402709359
:1081700065022B9A44E050E06EE170E082E692E006
:108180000E94FC9A80918A340E94BA6FE3C644FF31
:1081900003C08CE995E002C08FE995E09F938F932F
:1081A00086E392E09F938F930E948A998091620266
:1081B0000F900F900F900F9085FF03C08CE995E012
:1081C00002C08FE995E09F938F938BE292E09F939B
:1081D0008F930E948A99809162020F900F900F9066
:1081E0000F9086FF03C08CE995E002C08FE995E00F
:1081F0009F938F9380E292E09F938F930E948A993E
:10820000809162020F900F900F900F9087FF03C034
:108210008CE995E002C08FE995E09F938F9385E10B
:1082200092E09F938F930E948A998091620290912D
:108230006302A0916402B09165020F900F900F90BD
:108240000F9090FF03C08CE995E002C08FE995E0A4
:108250009F938F938AE092E09F938F930E948A99D5
:108260008091620290916302A0916402B0916502D4
:108270000F900F900F900F9091FF03C08CE995E045
:1082800002C08FE995E09F938F938FEF91E09F93CA
:108290008F930E948A998091620290916302A091CB
:1082A0006402B09165020F900F900F900F9091FFB4
:1082B00051C68FE496E00E94AE996DEDA62E6BE15B
:1082C000B62E0BE010E077E5872E76E0972EF501CD
:1082D00080819181F2E0AF0EB11C9F938F931F9329
:1082E0000F939F928F920E9478990F5F1F4F0F906C
:1082F0000F900F900F900F900F900B31110539F7E1
:1083000029C68FED94E09F938F930E948A99809164
:108310007D020F900F90882361F01F928F938CED58
:1083200094E09F938F930E948A990F900F900F90E3
:108330000F90F89428E088E190E00FB6F894A895A3
:10834000809360000FBE20936000FFCF0E94F36710
:1083500001C660917B0270917C0280E090E00E94F7
:10836000BF988C016CE975E00E94D398892BE9F4E1
:108370000E94A66E8091620290916302A0916402B5
:10838000B09165028D7F8160809362029093630259
:10839000A0936402B093650244E050E06EE170E0A7
:1083A00082E692E00E94FC9AD5C56FE975E0C801AB
:1083B0000E94D398892BE1F40E945E6E8091620244
:1083C00090916302A0916402B09165028C7F8093CA
:1083D000620290936302A0936402B093650244E04A
:1083E00050E06EE170E082E692E00E94FC9AB2C535
:1083F00062E676E0C8010E94D398892BE9F40E94D6
:108400005E6E8091620290916302A0916402B091CD
:1084100065028E7F82608093620290936302A093D4
:108420006402B093650244E050E06EE170E082E6E1
:1084300092E00E94FC9A8EC58091620281FF0FC07B
:1084400082E696E09F938F938BEF91E09F938F93BB
:108450000E948A990F900F900F900F907BC580FF1C
:1084600003C08CE995E002C08FE995E09F938F935C
:1084700087EF91E09F938F930E948A990F900F90BE
:108480000F900F9067C58091E32F8F938091E22F1B
:108490008F938091E12F8F938091E02F8F93809124
:1084A000DF2F8F938091DE2F8F938091DD2F8F931D
:1084B0008091DC2F8F938091DB2F8F938091DA2F27
:1084C0008F938091D92F8F938091D82F8F93809104
:1084D000D72F8F938091D62F8F938091D52F8F9305
:1084E0008091D42F8F9380EB94E09F938F930E9481
:1084F0008A990E94C00D80917D020FB6F894DEBF6C
:108500000FBECDBF882309F425C51F928F938DEA36
:1085100094E09F938F930E948A990F900F900F90F1
:108520000F9018C5F89481E090E029E0FC012093B9
:108530005700C895E02C80E090E0FC0120935700A4
:10854000C895F02C7894F89483E090E0FC01209397
:108550005700C895002D82E090E0FC012093570061
:10856000C895102D78948091BD278F938091BC275A
:108570008F938091BB278F938091BA278F9323EAA3
:1085800034E03F932F930E948A991F92EF921F929B
:10859000FF921F920F931F921F938CE794E09F937B
:1085A0008F930E948A990E945723809166001F92A0
:1085B0008F9380E794E09F938F930E948A990E9403
:1085C000C00D80917D020FB6F894DEBF0FBECDBF07
:1085D000882309F4BFC41F928F938DE694E09F9384
:1085E0008F930E948A990F900F900F900F90B2C4B2
:1085F00060E070E080E090E00E94C90D60E070E013
:1086000081E090E00E94C90D80917D02882309F4E9
:10861000A1C41F928F938AE694E09F938F930E9448
:108620008A990F900F900F900F9094C40E94792117
:108630000E94C00D80917D02882309F48BC41F9293
:108640008F9387E694E09F938F930E948A990F906F
:108650000F900F900F907EC460917B0270917C020E
:1086600080E090E00E94BF9869E176E00E94D39894
:10867000892B31F5F89482E89AE00E94F55B5C0161
:10868000009769F0C5010F960E94F95EB50184E07C
:1086900092E00E94AF5BC5010E949D5CF0CF82E832
:1086A0009AE00E94825C892B29F082E89AE00E947D
:1086B0002E5CF5CF82E89AE00E94F15B789434C09A
:1086C00082E89AE00E94F55B5C0107E616E0A114DF
:1086D000B10451F1F50186811F928F9380851F921D
:1086E0008F9385811F928F9381851F928F938781AE
:1086F0001F928F9384811F928F9383811F928F93F8
:1087000082811F928F9382851F928F931F930F9365
:108710000E947899C5010E949D5C5C010FB6F89497
:10872000DEBF0FBECDBFD3CF80917D02882309F479
:1087300011C41F928F9384E694E09F938F930E94BD
:108740008A990F900F900F900F9004C40E948C3064
:1087500001C460917B0270917C0280E090E00E94F5
:10876000BF988C0166EA76E00E94D398892BD1F4F9
:108770008091620290916302A0916402B0916502BF
:10878000977F8093620290936302A0936402B093F8
:10879000650244E050E06EE170E082E692E00E9403
:1087A000FC9AD8C365E276E0C8010E94D398892B71
:1087B000D1F48091620290916302A0916402B09121
:1087C000650298608093620290936302A0936402B2
:1087D000B093650244E050E06EE170E082E692E022
:1087E0000E94FC9AB7C30E942F0AB4C360917B0217
:1087F00070917C0280E090E00E94BF98FC01208193
:108800002332B1F44AE050E060E070E001960E944B
:1088100061951B0160917B0270917C0280E090E089
:108820000E94BF98F4E02F1631040CF094C002C0EF
:10883000212C312C009709F48EC01982BE016F5F84
:108840007F4F0E94E92929013A014B01B82FA92F36
:108850008AE0829DF001839DF00D1124E355F44ED2
:1088600020812A8331813B8382818C8393819D8304
:1088700024812E8335813F838681888797819987DC
:108880009201A301B4018B2F9A2FAA80BB80CC80C8
:10889000DD80EE80FF80088519850E94F09409F440
:1088A0005DC08981882351F18CF02A81422A3B8165
:1088B000532A8C81682A9D81792A2E81822A3F81C0
:1088C000932A8885B82B9985A92B18C04094509479
:1088D0006094709480949094B095A0952A814222DF
:1088E0003B8153228C8168229D8179222E818222B4
:1088F0003F8193228885B8239985A923408251829C
:108900006282738284829582B683A78348E250E0B4
:1089100062E270E08DEA9BE10E94FC9A8CE594E0B3
:108920009F938F930E948A998AE0829DF001839D94
:10893000F00D1124E355F44E2081318142815381A1
:1089400064817581868197810E9485260E94C00D71
:108950000F900F9003C082E00E948B2B80E594E083
:108960009F938F930E948A992FEF3FEF4FEF5FEF16
:108970006FEF7FEF8FEF9FEF0E9485260E94C00D63
:1089800080917D020F900F90882309F4E3C21F921B
:108990008F938DE494E09F938F930E948A990F9018
:1089A0000F900F900F90D6C260917B0270917C0265
:1089B00080E090E00E94BF98FC0120812332A1F466
:1089C0004AE050E060E070E001960E9461958B0102
:1089D00060917B0270917C0280E090E00E94BF98E1
:1089E00004301105ECF402C000E010E00097C1F083
:1089F0004AE050E060E070E00E9495962AE0209FF7
:108A0000F001219FF00D1124E355F44E718760872A
:108A100048E250E062E270E08DEA9BE10E94FC9A3D
:108A200081E00E948B2B80917D02882309F492C201
:108A30001F928F938AE494E09F938F930E948A9968
:108A40000F900F900F900F9085C20E94325F80911F
:108A50007D02882309F47EC21F928F9387E494E0FD
:108A60009F938F930E948A990F900F900F900F9071
:108A700071C20E944F2C80917D02882309F46AC242
:108A80001F928F9384E494E09F938F930E948A991E
:108A90000F900F900F900F905DC280E090E00E94C9
:108AA000732380917D02882309F454C21F928F930F
:108AB00081E494E09F938F930E948A990F900F9086
:108AC0000F900F9047C28091CA2B81FF2DC00E944A
:108AD000FD20892B49F58091C1278F938091C02774
:108AE0008F938091BF278F938091BE278F9386E3CA
:108AF00094E09F938F930E948A998091A2348F93E0
:108B00008091A1348F938091A0348F9380919F3472
:108B10008F9389E294E09F938F930E948A990FB676
:108B2000F894DEBF0FBECDBF0E94C00D8091CA2B4E
:108B30009091CB2B90FF63C081E090E00E94742065
:108B40003B014C0180E090E00E9474201B012C014D
:108B50000E94D21F9F928F927F926F9288E194E041
:108B60009F938F930E948A995F924F923F922F9288
:108B700088E094E09F938F930E948A99222D332D51
:108B8000442D552D662D772D882D992D0E94751E0B
:108B90009F938F937F936F938DEF93E09F938F932A
:108BA0000E948A99222D332D442D552D662D772D27
:108BB000882D992D0E94D61E9F938F937F936F933C
:108BC0008FEE93E09F938F930E948A99222D332DED
:108BD000442D552D662D772D882D992D0E94371FF8
:108BE0009F938F937F936F938CED93E09F938F93DD
:108BF0000E948A990FB6F894DEBF0FBECDBF0E94C7
:108C0000C00D80917D02882309F4A4C11F928F9327
:108C100089ED93E09F938F930E948A990F900F9014
:108C20000F900F9097C18091CA2B82FF2BC021E03B
:108C300048E061E083E00E946C158091B11C8F9345
:108C40008091B01C8F938091AF1C8F938091AE1C4C
:108C50008F938091AD1C8F938091AC1C8F938091EA
:108C6000AB1C8F938091AA1C8F9382EC93E09F930F
:108C70008F930E948A990E94C00D0FB6F894DEBFB0
:108C80000FBECDBF8091CA2B9091CB2B91FF41C0DD
:108C90000E94C219B62EA72E982E892E20E030E011
:108CA00048EC52E4D501F4016B2F7A2F8F2F9E2FC1
:108CB0000E94BD9120E836EE45EC57E40E943C8FBF
:108CC00021E03EED42E45EE30E9420929B01AC0174
:108CD00060E070E080E89FE30E94718E2BE43AE34D
:108CE0004DEB57E30E943C8F9F938F937F936F933D
:108CF0008F929F92AF92BF9289EA93E09F938F9356
:108D00000E948A990E94C00D0FB6F894DEBF0FBE74
:108D1000CDBF80917D02882309F41CC11F928F93DF
:108D200086EA93E09F938F930E948A990F900F9009
:108D30000F900F900FC160917B0270917C0280E0D8
:108D400090E00E94BF986BEA76E00E94D398892B4E
:108D5000B1F460917B0270917C0280E090E00E940F
:108D6000BF98009709F4F6C00E94AD97803108F0D3
:108D7000F1C090915201982B90935201EBC08091D9
:108D800052018F701F928F938AEE91E09F938F9381
:108D90000E948A990E94C00D0F900F900F900F9023
:108DA000D9C060917B0270917C0280E090E00E94CB
:108DB000BF98009711F14AE050E060E070E00E9437
:108DC0006195603198F4609360021F926F9389E916
:108DD00093E09F938F930E948A9941E050E06BE16A
:108DE00070E080E692E00E94FC9A11C080916002DF
:108DF0001F928F9380E993E006C0809160021F92DA
:108E00008F9387E893E09F938F930E948A990F90A6
:108E10000F900F900F900E94C00D80917D028823CB
:108E200009F498C01F928F9384E893E09F938F93E7
:108E30000E948A990F900F900F900F908BC06091B5
:108E40007B0270917C0280E090E00E94BF988C01D0
:108E50006CE975E00E94D398892BE1F40E940F6DB4
:108E60008091620290916302A0916402B0916502C8
:108E700090618093620290936302A0936402B09326
:108E8000650244E050E06EE170E082E692E00E940C
:108E9000FC9A60C06FE975E0C8010E94D398892BE5
:108EA00081F5F8940E941D6D88E10FB6F8948093C7
:108EB0006000109260000FBE84B7877F84BF8091EE
:108EC00060008861809360001092600078948091C7
:108ED000620290916302A0916402B09165029F7E4C
:108EE0008093620290936302A0936402B093650240
:108EF00044E050E06EE170E082E692E00E94FC9A6D
:108F000029C060EB76E0C8010E94D39840916202CC
:108F1000509163026091640270916502892B21F483
:108F200054FF18C0F894FFCF54FF03C08CE995E0BC
:108F300002C08FE995E09F938F9386EE91E09F9317
:108F40008F930E948A990F900F900F900F9002C0FC
:108F50000E949D21EA85FB851182108283E02B9679
:108F60000FB6F894DEBF0FBECDBFDF91CF911F913A
:108F70000F91FF90EF90DF90CF90BF90AF909F90B8
:108F80008F907F906F905F904F903F902F900895BB
:108F9000CF93DF93EC0188819981009741F0803D68
:108FA000914109F48CC01982188283E093C00E9419
:108FB000DF318091620280FD05C081FF01C01D9BF1
:108FC0000E945E6E809170008C7F80937000809113
:108FD000B60080628093B6001092B20082E0809367
:108FE000B1008091B6008770E1F7809170008160D8
:108FF000809370006DE47AE080E090E00E94ED6C78
:109000000E94B92280E00E94972488EA90E19F9311
:109010008F930E948A990E944D128091CA2B0F90C3
:109020000F9086FD0E949F678091CA2B9091CB2B59
:1090300090FD0E948E1F8091CA2B87FF06C021E001
:109040004CE061E080ED0E94426880913D0A0E9400
:10905000FE70809161020E94A56F0E94A26F8093B2
:10906000720A809161020E94A56F80913D0A1F9251
:109070008F938091720A1F928F9385EB96E09F9356
:109080008F930E9478991092740A1092730A0F902D
:109090000F900F900F900F900F9082E592E09093B9
:1090A0009D3480939C3483E290E09093851280936A
:1090B000841280ED91E19983888381E00BC0633253
:1090C000E1F749EF5FE260E070E083E79AE00E9439
:1090D0005133E3CFDF91CF9108950F931F93CF9337
:1090E000DF93EC018A0188819981009711F1853E17
:1090F000914121F01982188283E020C06231E9F4A5
:10910000A80162E170E083E79AE00E94513384E0B5
:10911000809381341092833410928234109385347A
:109120000093843441E854E362E18EE392E00E94CC
:10913000085B85EE91E19983888381E0DF91CF918F
:109140001F910F910895AF92BF92CF92DF92EF924D
:10915000FF920F931F93CF93DF93EC018B015A0182
:109160008091410A9091420AA091430AB091440A29
:1091700081FD08C08091620280FD04C081FF55C05E
:109180001D9B53C0F801C384D484E584F684A4E60F
:10919000B0E0A70196010E942D93672F782F892FA9
:1091A000992724E630E040E050E00E94C1927F938E
:1091B0006F93CD2CDE2CEF2CFF24DF92CF92F801A1
:1091C00086811F928F9385811F928F9388818F70E4
:1091D0001F928F9389811F928F93F50181811F9236
:1091E0008F9380811F928F932296DF93CF9387EC8A
:1091F00096E09F938F930E94789980917D02EDB7BE
:10920000FEB774960FB6F894FEBF0FBEEDBF88236D
:1092100061F01F928F9380EE91E09F938F930E9455
:109220008A990F900F900F900F90DF91CF911F911F
:109230000F91FF90EF90DF90CF90BF90AF90089587
:109240008436910514F19F938F938BE097E09F9361
:109250008F930E9478998091D42F9091D52FA091CF
:10926000D62FB091D72F0196A11DB11D8093D42F79
:109270009093D52FA093D62FB093D72F0F900F9008
:109280000F900F9081E090E0089580E090E00895C5
:109290002F923F924F925F926F927F928F929F9206
:1092A000AF92BF92CF92DF92EF92FF920F931F93F4
:1092B000CF93DF93CDB7DEB7C859D1090FB6F89475
:1092C000DEBF0FBECDBFC057DF4F99838883C05923
:1092D000D0408A01633871F487E79AE0C856DF4FBF
:1092E0006883C859D0400E944B59C856DF4F6881E7
:1092F000C859D040C057DF4FA881B981C059D0406C
:109300002D913C912D37B1E13B0709F4D8C340F4CE
:109310002115310581F0213B3F4009F41AC40EC4E8
:109320002F3841E1340709F4EAC32639314111F4F9
:109330000C94815603C444EF52E061E870E087E783
:109340009AE00E94315981EB9FE0B0C3E3E0F0E086
:10935000EC0FFD1FE20FF31F1082C9010E9420498C
:10936000892B89F720E030E040E050E0C357DF4F21
:109370006881CD58D040627070E080E090E0A0E05D
:109380000E94F99409F097C6C557DF4F2881CB5842
:10939000D040287030E040E050E060E070E080E0D5
:1093A00090E0A0E00E94F994A1F127E04AE250E0A9
:1093B0006BE270E089E290E00E94836383E994E3CA
:1093C0000E94F165BC01882777FD8095982F0E9447
:1093D000DB8F20E030E048EC52E40E943C8F9F930A
:1093E0008F937F936F938FE397E09F938F931F9259
:1093F00087E78F93CE018E0D9F1D03969F938F93CA
:109400000E94DB99E80EF91E0FB6F894DEBF0FBE7E
:10941000CDBFC557DF4F2881CB58D040207130E0F9
:1094200040E050E060E070E080E090E0A0E00E946A
:10943000F994F1F126E04AE250E06BE270E089E253
:1094400090E00E94836381E090E00E944E0D809343
:109450003C0A86E09CE10E94F165BC01882777FD0B
:109460008095982F0E94DB8F20E030E048EC52E49A
:109470000E943C8F9F938F937F936F9389E497E033
:109480009F938F931F9287E78F93C7010296E1E026
:10949000F0E0EC0FFD1F8E0F9F1F9F938F930E9494
:1094A000DB99E80EF91E0FB6F894DEBF0FBECDBFF4
:1094B000272D30E040E050E060E070E080E090E098
:1094C000A0E00E94F99401F10E940A0D9F938F93EE
:1094D0007F936F9384E597E09F938F931F9287E725
:1094E0008F93C701029641E050E04C0F5D1F840F3F
:1094F000951F9F938F930E94DB99E80EF91E0FB67C
:10950000F894DEBF0FBECDBFC557DF4F2881CB58C3
:10951000D040207430E040E050E060E070E080E057
:1095200090E0A0E00E94F99431F18091CF2F8F93C9
:109530008091CE2F8F938091CD2F8F938091CC2FC0
:109540008F9382E697E09F938F931F9287E78F9385
:10955000C7010296A1E0B0E0AC0FBD1F8A0F9B1FB0
:109560009F938F930E94DB99E80EF91E0FB6F89433
:10957000DEBF0FBECDBFC557DF4F2881CB58D040CF
:10958000207830E040E050E060E070E080E090E083
:10959000A0E00E94F99441F1F8948091793490917F
:1095A0007A34A0917B34B0917C347894BF93AF939C
:1095B0009F938F9380E797E09F938F931F9287E706
:1095C0008F93C701029621E030E02C0F3D1F820FE0
:1095D000931F9F938F930E94DB99E80EF91E0FB69D
:1095E000F894DEBF0FBECDBF20E0C457DF4F3881F7
:1095F000CC58D040317040E050E060E070E080E056
:1096000090E0A0E00E94F99409F067C520E0C457FB
:10961000DF4F3881CC58D040327040E050E060E0FD
:1096200070E080E090E0A0E00E94F99409F0C8C5E5
:1096300020E0C457DF4F3881CC58D040347040E030
:1096400050E060E070E080E090E0A0E00E94F994DB
:1096500009F0E7C520E0C457DF4F3881CC58D0402F
:10966000387040E050E060E070E080E090E0A0E022
:109670000E94F99409F004C620E0C457DF4F3881F6
:10968000CC58D040307140E050E060E070E080E0C5
:1096900090E0A0E00E94F99409F065C620E0C4576C
:1096A000DF4F3881CC58D040307240E050E060E06D
:1096B00070E080E090E0A0E00E94F99409F083C699
:1096C00020E030E040E050E0C357DF4F6881CD58E4
:1096D000D040647070E080E090E0A0E00E94F994D7
:1096E00009F09FC620E0CB56DF4F3881C559D040E6
:1096F00040E050E060E070E080E090E0A0E00E9498
:10970000F99409F0FBC620E0CA56DF4F3881C659EC
:10971000D04040E050E060E070E080E090E0A0E009
:109720000E94F99409F018C7502F5170D52E20E0EF
:1097300030E0452F50E060E070E080E090E0A0E095
:109740000E94F99409F036C720E030E0402F4270C3
:1097500050E060E070E080E090E0A0E00E94F994CA
:1097600009F05BC720E030E0C657DF4F4881CA5898
:10977000D04050E060E070E080E090E0A0E00E9427
:10978000F99409F07DC720E030E0402F487050E0A8
:1097900060E070E080E090E0A0E00E94F99409F0C1
:1097A00099C720E030E0402F407150E060E070E069
:1097B00080E090E0A0E00E94F99409F0BBC720E0AF
:1097C00030E0402F407250E060E070E080E090E0D8
:1097D000A0E00E94F99409F0DDC720E030E0402FBE
:1097E000407450E060E070E080E090E0A0E00E9413
:1097F000F99411F00C94FB53F02FF078AF2E20E089
:1098000030E04F2F50E060E070E080E090E0A0E0BA
:109810000E94F99411F00C942E54212F2170B22E35
:1098200020E030E040E05B2D60E070E080E090E020
:10983000A0E00E94F99411F00C943B5420E030E039
:109840004A2D50E060E070E080E090E0A0E00E94EF
:10985000F99411F00C94495420E030E040E05B2D85
:1098600060E070E080E090E0A0E00E94F99411F0E8
:109870000C947E5420E030E040E0512F527060E0C4
:1098800070E080E090E0A0E00E94F99411F00C9468
:10989000B35420E030E040E0512F547060E070E0BD
:1098A00080E090E0A0E00E94F99411F00C94E6545E
:1098B00020E030E040E0512F507160E070E080E047
:1098C00090E0A0E00E94F99411F00C94195520E06A
:1098D00030E040E0512F507260E070E080E090E0B6
:1098E000A0E00E94F99411F00C94585520E030E06B
:1098F00040E0512F507460E070E080E090E0A0E024
:109900000E94F99411F00C94975520E030E040E06B
:10991000512F587060E070E080E090E0A0E00E947D
:10992000F99411F00C94D65520E030E040E05C2D25
:1099300060E070E080E090E0A0E00E94F99411F017
:109940000C94075620E030E04D2D50E060E070E0D0
:1099500080E090E0A0E00E94F99411F00C9443564E
:10996000C557DF4F2881CB58D040C457DF4F3881CF
:10997000CC58D040A801C357DF4F6881CD58D040A4
:10998000CE56DF4F7881C259D040CD56DF4F888107
:10999000C359D040CC56DF4F9881C459D040A0E085
:1099A0000E94F99411F00C944E56809160028061EF
:1099B000898380916B0A8A83FE01EE0DFF1D13825D
:1099C0008091410A9091420AA091430AB091440AC1
:1099D00087010D5F1F4F80FF0CC01F930F9380E026
:1099E00099E09F938F930E9478990F900F900F901A
:1099F0000F90B801CE0101960E947A6280916202B6
:109A000082FF0AC029E730E3A801BE016F5F7F4FE4
:109A10008BE692E00E940F678091410A9091420A82
:109A2000A091430AB091440A82FD73980E94A66EE9
:109A300087E79AE00E944D598091620290916302FB
:109A4000A0916402B091650290FF40C03FEFE31A1D
:109A5000F30A0E94A26FD82E89E10E94BA6F40914A
:109A6000620250916302609164027091650250FF3E
:109A700029C0739880916B0A8F5F80936B0A8A83E9
:109A8000B7016F5F7F4FCE0101960E947A6287E730
:109A90009AE00E944D5940E050E065E880918812BC
:109AA000909189120E94085B8DE791E1C057DF4FCA
:109AB000A881B981C059D0408D939C933CC0E12CC2
:109AC000F12CCDCF8D2D0E94BA6F739A80913E0AF2
:109AD00090913F0A892B11F00E945E6E80916B0A73
:109AE0008F5F80936B0A8091410A9091420AA09106
:109AF000430AB091440A82FF26CC739A24CC83E6B1
:109B00009AE00E94AE5D892BB1F00E94A66E809112
:109B1000620287FD2B9860E470E083E69AE00E9481
:109B2000875D86E991E1C057DF4FE881F981C0592F
:109B3000D0409183808381E00C949456C057DF4FCE
:109B4000A881B981C059D0401D921C9283E00C9429
:109B50009456623181F7C0906202D0906302E09027
:109B60006402F0906502D1FCEECBF8018081813077
:109B700091F50180F281E02D2081C557DF4F2883C8
:109B8000CB58D0403181C457DF4F3883CC58D040B8
:109B9000028113814481C357DF4F4883CD58D040A1
:109BA0005581CE56DF4F5883C259D0408681CD565D
:109BB000DF4F8883C359D0409781CC56DF4F9883BD
:109BC000C459D04020843184C257DF4F1982188293
:109BD000CE58D0406AC08230E9F4A381B481C25724
:109BE000DF4FB983A883CE58D040212C312CB1E06F
:109BF000C557DF4FB883CB58D040C457DF4F1882CA
:109C0000CC58D04000E010E8C357DF4F1882CD5841
:109C1000D0403CC08330F9F0843009F094CB212C43
:109C2000312CC257DF4F19821882CE58D040E5E060
:109C3000C557DF4FE883CB58D040C457DF4F188259
:109C4000CC58D04000E010E0F2E0C357DF4FF8837B
:109C5000CD58D0401BC0212C312CC257DF4F198268
:109C60001882CE58D04025E0C557DF4F2883CB5807
:109C7000D040C457DF4F1882CC58D04000E010E0ED
:109C800031E0C357DF4F3883CD58D040CE56DF4F39
:109C90001882C259D040CD56DF4F1882C359D040E8
:109CA000CC56DF4F1882C459D0408090CC2F909072
:109CB000CD2FA090CE2FB090CF2F40908A02509001
:109CC0008B0260908C0270908D022DEC3CEC4CE489
:109CD0005EE3C301B2010E94728E9B01AC01C5011B
:109CE000B4010E94FE9087FD0BC0E894E0F8C0929A
:109CF0006202D0926302E0926402F09265024AC06E
:109D0000A3019201C501B4010E94388F87FF42C0B0
:109D10008091D82F9091D92FA091DA2FB091DB2F7D
:109D20000196A11DB11D8093D82F9093D92FA09398
:109D3000DA2FB093DB2FE0FC06CB6894E0F8C092FA
:109D40006202D0926302E0926402F092650245E4FE
:109D5000C557DF4F4883CB58D04050E2C457DF4F40
:109D60005883CC58D04000E010E084E0C357DF4F68
:109D70008883CD58D040CE56DF4F1882C259D0408C
:109D8000CD56DF4F1882C359D040CC56DF4F1882D2
:109D9000C459D040902F9470C657DF4F9883CA584B
:109DA000D04020E030E0492F50E060E070E080E0FB
:109DB00090E0A0E00E94F99409F08C9AC557DF4F1B
:109DC000A881CB58D040A0727A2E2A2F30E040E0F4
:109DD00050E060E070E080E090E0A0E00E94F99444
:109DE00011F00E940A0DC457DF4FB881CC58D04003
:109DF000B074CB56DF4FB883C559D04020E03B2F1D
:109E000040E050E060E070E080E090E0A0E00E9480
:109E1000F99411F00E94FD20C457DF4FE881CC581F
:109E2000D040E078CA56DF4FE883C659D04020E0E2
:109E30003E2F40E050E060E070E080E090E0A0E085
:109E40000E94F99451F00E94A50C6093863470939F
:109E500087348093883490938934C557DF4F2881A5
:109E6000CB58D040217030E040E050E060E070E03E
:109E700080E090E0A0E00E94F994F1F084E99BE199
:109E80009F938F938FE197E09F938F931F9287E724
:109E90008F93CE0103969F938F930E94DB996C0161
:109EA0000E9420490FB6F894DEBF0FBECDBF892BAC
:109EB00009F049CA760102C0E12CF12CC557DF4FE9
:109EC0002881CB58D040227030E040E050E060E084
:109ED00070E080E090E0A0E00E94F994D1F1C70129
:109EE000029667E277E041E050E04C0F5D1F840F7F
:109EF000951F0E94DC9853E0E50EF11C43E9A42E67
:109F000044E3B42E5EEFC52E53E0D52E67E7962EC0
:109F1000D5018D915D011F928F93DF92CF921F9299
:109F20009F92C7010296E1E0F0E0EC0FFD1F8E0F5B
:109F30009F1F9F938F930E94DB99E80EF91E0FB627
:109F4000F894DEBF0FBECDBF3BE9A31634E3B306E2
:109F5000F9F6C557DF4F2881CB58D040247030E048
:109F600040E050E060E070E080E090E0A0E00E941F
:109F7000F99409F447C0C70102966BE277E041E02B
:109F800050E04C0F5D1F840F951F0E94DC9854E039
:109F9000E50EF11C4E018AE7880E911C80E1D40188
:109FA0001D928A95E9F728E0A40168E980EB0E94F8
:109FB000B0135401B8E0AB0EB11C2EEFC22E23E05B
:109FC000D22E37E7632EF40181914F011F928F93B8
:109FD000DF92CF921F926F92C701029621E030E08C
:109FE0002C0F3D1F820F931F9F938F930E94DB992D
:109FF000E80EF91E0FB6F894DEBF0FBECDBF8A146F
:10A000009B0409F7512F5078C52E20E030E040E046
:10A0100060E070E080E090E0A0E00E94F994E1F45C
:10A0200080913E0A90913F0A9F938F9380E397E03F
:10A030009F938F931F9287E78F93CE018E0D9F1D65
:10A0400003969F938F930E94DB99E80EF91E0FB63B
:10A05000F894DEBF0FBECDBF20E030E040E050E01E
:10A06000C357DF4F6881CD58D040617070E080E009
:10A0700090E0A0E00E94F99409F474C9E3E0F0E0F4
:10A08000EC0FFD1FEE0DFF1D80E28083ECEFFFE281
:10A09000808197012F5F3F4F7901882309F456C9CA
:10A0A0008081A1E0B0E0AC0FBD1FAE0DBF1D1296C8
:10A0B0008C933196EDCFCE018E0D9F1D67E377E037
:10A0C00003960E94DC9897E0E90EF11CC7010E94FC
:10A0D0002049892B09F037C957C92114310409F4E3
:10A0E00095CAF8944090793450907A3460907B34DB
:10A0F00070907C3478948091FE1B9091FF1BA0910E
:10A10000001CB091011CA3019201281B390B4A0BC2
:10A110005B0BCA01B9010E94D98F4B015C01B101EF
:10A1200080E090E00E94D98F9B01AC01C501B40191
:10A130000E943C8FB82ED92E9F938F937F936F935D
:10A140008BE797E09F938F931F9287E78F939E01F2
:10A150002E0D3F1D2D5F3F4F3F932F93C856DF4F6E
:10A160006883C859D040C956DF4F7883C759D0405B
:10A170000E94DB99E80EF91EC856DF4F6881C85966
:10A18000D040C956DF4F7881C759D040862F972FCE
:10A19000AB2DBD2D80938B3490938C34A0938D3454
:10A1A000B0938E344092FE1B5092FF1B6092001CB5
:10A1B0007092011C0FB6F894DEBF0FBECDBF26CA49
:10A1C0002114310409F434CAF8948091D51B90917C
:10A1D000D61BA091D71BB091D81B78949F938F93D7
:10A1E000809169028F93809168028F9388E897E04D
:10A1F0009F938F931F9287E78F93C7010296A1E0E9
:10A20000B0E0AC0FBD1F8A0F9B1F9F938F930E94DE
:10A21000DB99E80EF91E0FB6F894DEBF0FBECDBF76
:10A2200007CAF89480917D3490917E34A0917F3458
:10A23000B09180347894BF93AF939F938F9388E9C4
:10A2400097E09F938F931F9287E78F93C7010296A2
:10A2500021E030E02C0F3D1F820F931F9F938F93BF
:10A260000E94DB99E80EF91EC7010E9420490FB633
:10A27000F894DEBF0FBECDBF892B09F064C8EAC9D0
:10A280002114310409F4F8C9F89440907D345090B9
:10A290007E3460907F347090803478948091021C7A
:10A2A0009091031CA091041CB091051CA301920184
:10A2B000281B390B4A0B5B0BCA01B9010E94D98FCD
:10A2C0004B015C01B10180E090E00E94D98F9B01BD
:10A2D000AC01C501B4010E943C8FB82ED92E9F93CA
:10A2E0008F937F936F9383EA97E09F938F931F924F
:10A2F00087E78F939E012E0D3F1D2D5F3F4F3F93AC
:10A300002F93C856DF4F6883C859D040C956DF4FD6
:10A310007883C759D0400E94DB99E80EF91EC856D1
:10A32000DF4F6881C859D040C956DF4F7881C7597F
:10A33000D040862F972FAB2DBD2D80938F349093D7
:10A340009034A0939134B09392344092021C509276
:10A35000031C6092041C7092051C0FB6F894DEBFBB
:10A360000FBECDBF89C9232809F498C9F8948091FC
:10A37000D91B9091DA1BA091DB1BB091DC1B789468
:10A380009F938F93809167028F93809166028F9342
:10A3900080EB97E09F938F931F9287E78F93C7017E
:10A3A0000296A1E0B0E0AC0FBD1F8A0F9B1F9F93E8
:10A3B0008F930E94DB99E80EF91E0FB6F894DEBF6A
:10A3C0000FBECDBF6BC98091D02F9091D12FA0919E
:10A3D000D22FB091D32FBF93AF939F938F9380ECE5
:10A3E00097E09F938F931F9287E78F93C701029601
:10A3F00021E030E02C0F3D1F820F931F9F938F931E
:10A400000E94DB99E80EF91EC7010E9420490FB691
:10A41000F894DEBF0FBECDBF892B11F00C94A34979
:10A420004FC98091DB2F8F938091DA2F8F9380918A
:10A43000D92F8F938091D82F8F938091D72F8F937F
:10A440008091D62F8F938091D52F8F938091D42F89
:10A450008F938BEC97E09F938F931F9297E7D92E62
:10A46000DF92C7010296A1E0B0E0AC0FBD1F8A0FDA
:10A470009B1F9F938F930E94DB99E80EF91EC701E3
:10A480000E9420490FB6F894DEBF0FBECDBF892BC6
:10A4900011F00C94A3498091CA2B9091CB2B90FF83
:10A4A00021C98091DF2F8F938091DE2F8F93809130
:10A4B000DD2F8F938091DC2F8F938FEE97E09F930A
:10A4C0008F931F92DF92C701029621E030E02C0F9C
:10A4D0003D1F820F931F9F938F930E94DB99E80E7D
:10A4E000F91EC7010E9420490FB6F894DEBF0FBEC7
:10A4F000CDBF892B11F00C94A349F4C88091C127DA
:10A500008F938091C0278F938091BF278F938091E5
:10A51000BE278F9381E098E09F938F931F9287E7E8
:10A520008F93C7010296A1E0B0E0AC0FBD1F8A0F68
:10A530009B1F9F938F930E94DB99E80EF91EC70122
:10A540000E9420490FB6F894DEBF0FBECDBF892B05
:10A5500011F00C94A349D7C8809189348F938091CE
:10A5600088348F93809187348F93809186348F9332
:10A570008CE098E09F938F931F9287E78F93C7019A
:10A58000029621E030E02C0F3D1F820F931F9F9316
:10A590008F930E94DB99E80EF91EC7010E942049A3
:10A5A0000FB6F894DEBF0FBECDBF892B11F00C940F
:10A5B000A349BAC881E00E94560C209182023091D2
:10A5C000830240918402509185020E94BD919F9325
:10A5D0008F937F936F9389E198E09F938F931F925E
:10A5E00087E78F93C7010296A1E0B0E0AC0FBD1FD3
:10A5F0008A0F9B1F9F938F930E94DB99E80EF91E91
:10A60000C7010E9420490FB6F894DEBF0FBECDBF30
:10A61000892B11F00C94A34997C882E00E94560C34
:10A6200020917E0230917F02409180025091810200
:10A630000E94BD919F938F937F936F9386E298E0E2
:10A640009F938F931F9287E78F93C701029621E014
:10A6500030E02C0F3D1F820F931F9F938F930E941A
:10A66000DB99E80EF91EC7010E9420490FB6F89445
:10A67000DEBF0FBECDBF892B11F00C94A34972C869
:10A6800083E00E94560C9F938F937F936F9383E395
:10A6900098E09F938F931F9287E78F93C70102964D
:10A6A000A1E0B0E0AC0FBD1F8A0F9B1F9F938F935B
:10A6B0000E94DB99E80EF91E8C98C7010E94204980
:10A6C0000FB6F894DEBF0FBECDBF892B11F00C94EE
:10A6D000A34959C88091CA2B87FF63C821E042E192
:10A6E00061E080ED0E9442689F938F937F936F9308
:10A6F00080E498E09F938F931F9287E78F93C70121
:10A70000029621E030E02C0F3D1F820F931F9F9394
:10A710008F930E94DB99E80EF91EC7010E94204921
:10A720000FB6F894DEBF0FBECDBF892B11F00C948D
:10A73000A34937C88091CA2B87FF41C821E042E175
:10A7400062E080ED0E9442689F938F937F936F93A6
:10A750008EE498E09F938F931F9287E78F93C701B2
:10A760000296A1E0B0E0AC0FBD1F8A0F9B1F9F9324
:10A770008F930E94DB99E80EF91EC7010E942049C1
:10A780000FB6F894DEBF0FBECDBF892B11F00C942D
:10A79000A34915C88091CA2B87FF1FC821E042E159
:10A7A00063E080ED0E9442689F938F937F936F9345
:10A7B0008CE598E09F938F931F9287E78F93C70153
:10A7C000029621E030E02C0F3D1F820F931F9F93D4
:10A7D0008F930E94DB99E80EF91EC7010E94204961
:10A7E0000FB6F894DEBF0FBECDBF892B11F00C94CD
:10A7F000A3490C94ED4B8091CA2B87FD02C00C94A9
:10A80000FC4B21E042E164E080ED0E9442689F93AE
:10A810008F937F936F938AE698E09F938F931F9215
:10A8200087E78F93C7010296A1E0B0E0AC0FBD1F90
:10A830008A0F9B1F9F938F930E94DB99E80EF91E4E
:10A84000C7010E9420490FB6F894DEBF0FBECDBFEE
:10A85000892B11F00C94A3490C94FC4B8091CA2BCA
:10A8600082FD02C00C940D4C46E061E083E00E9442
:10A870006C150C940D4C8091CA2B82FD02C00C9477
:10A880001E4C21E046E061E083E00E946C150C94D0
:10A890001E4C8091CA2B82FD02C00C942C4C8091DE
:10A8A000AD1C8F938091AC1C8F938091AB1C8F93C8
:10A8B0008091AA1C8F9388E798E09F938F931F92B3
:10A8C00087E78F93C701029641E050E04C0F5D1F70
:10A8D000840F951F9F938F930E94DB99E80EF91EBA
:10A8E000C7010E9420490FB6F894DEBF0FBECDBF4E
:10A8F000892B11F00C94A3490C942C4C8091CA2BF9
:10A9000082FD02C00C943A4C8091B11C8F938091CF
:10A91000B01C8F938091AF1C8F938091AE1C8F934E
:10A9200080E898E09F938F931F9287E78F93C701EA
:10A930000296E1E0F0E0EC0FFD1F8E0F9F1F9F934A
:10A940008F930E94DB99E80EF91EC7010E942049EF
:10A950000FB6F894DEBF0FBECDBF892B11F00C945B
:10A96000A3490C943A4C8091CA2B9091CB2B90FD2B
:10A9700002C00C94494C80E090E00E9474209F93A8
:10A980008F937F936F938BE898E09F938F931F92A1
:10A9900087E78F93C701029641E050E04C0F5D1F9F
:10A9A000840F951F9F938F930E94DB99E80EF91EE9
:10A9B000C7010E9420490FB6F894DEBF0FBECDBF7D
:10A9C000892B11F00C94A3490C94494C8091CA2B0B
:10A9D0009091CB2B90FD02C00C94584C81E090E0FC
:10A9E0000E9474209F938F937F936F938BE998E0DD
:10A9F0009F938F931F9287E78F93C7010296E1E0A1
:10AA0000F0E0EC0FFD1F8E0F9F1F9F938F930E940E
:10AA1000DB99E80EF91EC7010E9420490FB6F89491
:10AA2000DEBF0FBECDBF892B11F00C94A3490C944F
:10AA3000584C8091CA2B9091CB2B90FD02C00C9466
:10AA4000674C81E090E00E9474204B015C0180E043
:10AA500090E00E9474209B01AC01C501B4010E94EA
:10AA6000751E9F938F937F936F938CEA98E09F93CB
:10AA70008F931F9287E78F93C701029641E050E0C2
:10AA80004C0F5D1F840F951F9F938F930E94DB993E
:10AA9000E80EF91EC7010E9420490FB6F894DEBFE8
:10AAA0000FBECDBF892B11F00C94A3490C94674CB9
:10AAB0008091CA2B9091CB2B90FD02C00C94764CC8
:10AAC00081E090E00E9474204B015C0180E090E006
:10AAD0000E9474209B01AC01C501B4010E94D61EE6
:10AAE0009F938F937F936F9387EB98E09F938F93C0
:10AAF0001F9287E78F93C7010296E1E0F0E0EC0F29
:10AB0000FD1F8E0F9F1F9F938F930E94DB99E80E6E
:10AB1000F91EC7010E9420490FB6F894DEBF0FBE90
:10AB2000CDBF892B11F00C94A3490C94764C8091E5
:10AB3000CA2B9091CB2B90FD02C00C94854C81E0E8
:10AB400090E00E9474204B015C0180E090E00E9444
:10AB500074209B01AC01C501B4010E94371F9F9373
:10AB60008F937F936F9385EC98E09F938F931F92C1
:10AB700087E78F93C701029641E050E04C0F5D1FBD
:10AB8000840F951F9F938F930E94DB99E80EF91E07
:10AB9000C7010E9420490FB6F894DEBF0FBECDBF9B
:10ABA000892B11F00C94A3490C94854C8091CA2BED
:10ABB0009091CB2B91FD02C00C94944C0E94C21931
:10ABC0009F938F937F936F9388ED98E09F938F93DC
:10ABD0001F9287E78F93C7010296E1E0F0E0EC0F48
:10ABE000FD1F8E0F9F1F9F938F930E94DB99E80E8E
:10ABF000F91EC7010E9420490FB6F894DEBF0FBEB0
:10AC0000CDBF892B11F00C94A3490C94944CC257DE
:10AC1000DF4FA881B981CE58D04016968C911697F7
:10AC20001F928F9315968C9115971F928F93139661
:10AC30008C9113971F928F9312968C911F928F93E2
:10AC400089EE98E09F938F931F9287E78F93C701B8
:10AC50000296E1E0F0E0EC0FFD1F8E0F9F1F9F9327
:10AC60008F930E94DB99E80EF91EC7010E942049CC
:10AC70000FB6F894DEBF0FBECDBF892B11F00C9438
:10AC8000A3490C94A24C779A8091410A9091420A70
:10AC9000A091430AB091440A92FD749A8091410AAE
:10ACA0009091420AA091430AB091440A82FD0CC0DF
:10ACB0008091620280FD08C081FD02C00C94D54CD9
:10ACC0001D9902C00C94D54C40E050E060E070E06B
:10ACD000CE0101960E94A40A2091B31C30E080911D
:10ACE000380A9091390A2817390710F40C94D54C7A
:10ACF00040E050E062E18CE092E00E94085B0C943E
:10AD0000D54C83E69AE00E94AE5D892B11F40C9439
:10AD10009B4D0E945E6E8091620287FD02C00C9482
:10AD2000A3492B9A0C94A349C856DF4F0FB6F89449
:10AD3000DEBF0FBECDBFDF91CF911F910F91FF906E
:10AD4000EF90DF90CF90BF90AF909F908F907F90CB
:10AD50006F905F904F903F902F9008950C9474598E
:10AD60006F927F928F929F92AF92BF92CF92DF921B
:10AD7000EF92FF920F931F93CF93DF93CDB7DEB780
:10AD800060970FB6F894DEBF0FBECDBF5B010E9487
:10AD9000A26FE82FF0E0EE0FFF1FE953F44E808121
:10ADA00091810196918380838091410A9091420A1A
:10ADB000A091430AB091440A81FD7498C090620248
:10ADC000D0906302E0906402F09065020E94CE6130
:10ADD0008C01FC018081982F92959F70913099F49D
:10ADE0008F7051F48091AB1B9091AC1B01969093A6
:10ADF000AC1B8093AB1B38C1B50183EA94E30E947E
:10AE0000EA58892B51F08091A91B9091AA1B0196B9
:10AE10009093AA1B8093A91B27C1D701C6012EE0DE
:10AE2000B695A795979587952A95D1F7F82FF17044
:10AE30006F2E82E89AE00E94F55B4C01009709F4BE
:10AE400048C0B501C40102960E94EA58892BE9F175
:10AE5000940147E65AE060E074E6C4010F960E9450
:10AE6000755EF8019181F4018481981321C0828577
:10AE70008F5F82878091A71B9091A81B019690936A
:10AE8000A81B8093A71B84E00E94EB62F40120853D
:10AE900030E02817390708F07BC184E00E94EB629C
:10AEA000F4018087F80180818F70F4018187DCC014
:10AEB000F401128684E00E94EB62F4018087F801BD
:10AEC00080818F70F401818764C1C4010E949D5C00
:10AED000B4CF84E092E00E948A5B4C01009709F4B1
:10AEE000C3C0B501C40102960E94E158F8018181F6
:10AEF0008150F401848380E091E0A0E0B0E083879A
:10AF00009487A587B687128684E00E94EB62F401DD
:10AF10008087F80180818F70F4018187B40182E815
:10AF20009AE00E94555C940147E65AE060E074E6BE
:10AF3000C4010F960E94755E77247394F801818195
:10AF4000F4018483F80180818F70F401878384E0A9
:10AF50000E94EB62F401858383E00E94EB62F401BE
:10AF6000868387818F3009F0712CF801C180F4014C
:10AF70008481C81AD12CE12CF12C76E0CC0CDD1C9C
:10AF8000EE1CFF1C7A95D1F72385348545855685BF
:10AF9000A0ECB0E00E942D93BB27A92F982F872FFC
:10AFA000C80ED91EEA1EFB1EC386D486E586F68629
:10AFB000A501B401C8010E94A40A2091B31C30E08D
:10AFC0008091380A9091390A2817390738F040E003
:10AFD00050E062E18CE092E00E94085B8091380AC8
:10AFE0009091390A029708F44BC08091CA2B86FFD2
:10AFF0002AC00E949167C80105960E945D67F8010A
:10B0000081811F928F93F40186811F928F93858196
:10B010001F928F9381E199E09F938F931F9280E11C
:10B020008F93CE0101967C01FF928F930E94DB9952
:10B0300082E00E947767C7010E945D670FB6F894AF
:10B04000DEBF0FBECDBF8091620290916302A091DE
:10B050006402B091650297FD50C08091380A9091CA
:10B06000390A029708F47EC08091410A9091420A01
:10B07000A091430AB091440A81FF8DC0749A8BC09D
:10B080008091620290916302A0916402B091650286
:10B0900096FFABCF662009F4A8CFF8012081322FAC
:10B0A0003F70832F90E00297F4F08FEF830F207FA3
:10B0B000822B808387E79AE00E94AE568091A51B81
:10B0C0009091A61B01969093A61B8093A51B80913F
:10B0D000410A9091420AA091430AB091440A96FF16
:10B0E00084CF739882CF8091AB1B9091AC1B01965B
:10B0F0009093AC1B8093AB1B78CF84E99BE12091AC
:10B10000941B222309F4A9CF9F938F9384E299E0A3
:10B110009F938F93CE0101967C01FF928F930E94A3
:10B12000189A6C01B701C80102960E94FD980F9011
:10B130000F900F900F900F900F90009709F48DCF04
:10B1400096012F5F3F4F280F391FA9012F5F3F4FF7
:10B15000FA0180818032C9F362E186E192E00E94C7
:10B16000085B7BCF772009F47FCF82E08093E52FC7
:10B170001092E72F1092E62F9092E92F8092E82FFD
:10B1800045EE5FE262E18EE392E00E94085B6CCFE5
:10B19000612C712CD3CE60960FB6F894DEBF0FBE33
:10B1A000CDBFDF91CF911F910F91FF90EF90DF9076
:10B1B000CF90BF90AF909F908F907F906F900895A9
:10B1C0000895FB012081FC012083FB012181FC010A
:10B1D00021830895FC019081DB018C91981309C0B3
:10B1E00081E090E0318111962C91321721F080E0BE
:10B1F000089580E090E00895BC0183EA94E30C9404
:10B20000E158DC011996ED91FC911A970280F381C7
:10B21000E02D309709F0099408950F931F93CF9371
:10B22000DF9300D0CDB7DEB78C0188E10E94FE62CB
:10B23000BC01CE0101960E94E158D8011996ED910A
:10B24000FC911A970190F081E02DBE016F5F7F4F56
:10B25000C80109950F900F90DF91CF911F910F9129
:10B260000895EF92FF920F931F93CF93DF93EC011A
:10B270008B017A014EE053E00E945A59FA86E98622
:10B2800062E173E0C801DF91CF911F910F91FF90B0
:10B29000EF900C94B3590C947259CF93DF93EC0157
:10B2A00063EA74E388E10E94F462CE01DF91CF91FA
:10B2B0000C947459EF92FF920F931F93CF93DF93E7
:10B2C000EC018B017A010E948F59F886EF8266E1CA
:10B2D00073E0C801DF91CF911F910F91FF90EF9024
:10B2E0000C94B3590C9497590C941C74DC01179668
:10B2F000ED91FC9118970190F081E02D0994DC010B
:10B300001796ED91FC9118970280F381E02D30970C
:10B3100009F00994089586E892E10C94F15BFC0130
:10B3200073836283BC0186E892E10C94555CBC0196
:10B3300086E892E10C943A5CCF93DF93EC0186E8C7
:10B3400092E10E94F55B009749F0FC012281338174
:10B350002C173D0729F00E949D5CF5CF80E090E01E
:10B36000DF91CF9108950F931F93CF93DF938B01BC
:10B370000E949C59EC01009731F01D830C83C80199
:10B380000E944D768E83DF91CF911F910F9108958A
:10B390001F93CF93DF93EC01162FEC81FD81309743
:10B3A000D1F0909389128093881282E08887CE0131
:10B3B00006960995992787FD90950297029710F0B8
:10B3C000133839F4BE01CE01DF91CF911F910C9457
:10B3D000F55981E08887DF91CF911F910895FC0195
:10B3E000208520FD0C94C8590895CF92DF92EF92EA
:10B3F000FF920F931F93CF93DF93EC016B01E090CB
:10B400008812F090891200918A1210918B12F80123
:10B41000EC17FD0739F0309709F44AC00190F0812C
:10B42000E02DF6CF209709F443C08885882309F1E1
:10B4300018860115110561F0C017D10729F0AE017A
:10B4400067E8C8010E94EF59F80100811181F1CF2E
:10B45000EC81FD81309769F0CC15DD0551F0D0937A
:10B460008912C093881240E050E063E8CE0106964E
:10B470000995E0918A12F0918B12CE17DF0769F4DB
:10B480008881998190938B1280938A120DC080815C
:10B4900091818C179D0721F0FC013097C1F704C002
:10B4A0008881998191838083F0928912E092881239
:10B4B000DF91CF911F910F91FF90EF90DF90CF9090
:10B4C00008951F93CF93DF9310929412C0918A1224
:10B4D000D0918B1211E0209779F08985882341F073
:10B4E0001887198640E050E062E8CE010E94C859F2
:10B4F0000990D881C02DEFCFDF91CF911F91089592
:10B500008091371391E0980F9093371308956091CD
:10B510008812709189120C94F5598AE88093371338
:10B52000109235131092361310928B1210928A12C9
:10B5300010928912109288120895809194128111AC
:10B540000E94615A70913613772309F451C0E0913B
:10B5500035132E2F30E085E0E89FF0011124EB56E3
:10B56000FD4E6081609393124181528150939212FB
:10B5700040939112838194819093901280938F12C3
:10B580002F5F3F4F2F7133272093351371507093E6
:10B590003613009731F580918A1290918B12909317
:10B5A0008E1280938D1280918D1290918E12892B24
:10B5B000F9F08091941281110E94615A4091911288
:10B5C000509192126091931280918D1290918E12EF
:10B5D0000E94EF59E0918D12F0918E12808191813D
:10B5E000DECF613819F421E0FC0120870E94EF5979
:10B5F000809194122091361390E0820F911D08954E
:10B60000809194122091361390E0820F911D08953D
:10B61000209136132032B9F0E0913513E20FEF712B
:10B62000E0938C1235E0E39FF0011124EB56FD4EC0
:10B63000608352834183948383832F5F20933613E7
:10B6400080E090E0089581E090E00895CF93DF934B
:10B65000C0918812D09189120E94EF59D09389121B
:10B66000C0938812DF91CF910895AB0130918A1277
:10B6700020918B12E32FF22FE817F907B1F03097E2
:10B6800021F00190F081E02DF7CF009771F0FC01DF
:10B690003083218390938B1280938A1221E020873C
:10B6A0001782168261E80C94265B0895009749F092
:10B6B000FC0120852150223020F421E021872093B5
:10B6C0009412089521E030E0FC018085811102C0D0
:10B6D00020E030E0C9010895CF93DF93EC014A8167
:10B6E0005B8160E070E08C819D810E94CC982A8112
:10B6F0003B8188819981289FA001299F500D389F07
:10B70000500D112460E070E08E819F81DF91CF9118
:10B710000C94CC98FC018281938120E030E02817C2
:10B720003907D1F0A481B581A20FB31F4C9141110B
:10B7300010C081E08C9380819181289FA001299F76
:10B74000500D389F500D112486819781840F951FCD
:10B7500008952F5F3F4FE3CF80E090E00895FC0114
:10B76000268137814281538180E090E084179507DC
:10B77000C9F02617370781F4A481B581A80FB91F36
:10B780002C91121614F421502C930480F581E02D95
:10B79000E80FF91F80810895A081B1812A0F3B1F16
:10B7A0000196E4CF8FEF0895FC0186819781681799
:10B7B0007907A0F0A081B18142815381A49F9001BB
:10B7C000A59F300DB49F300D1124280F391F81E043
:10B7D00090E06217730720F080E0089580E090E029
:10B7E0000895FC01118210820895FC0180819181ED
:10B7F0000895FB0120813181FC013183208308956C
:10B80000DC01ED91FC91309731F0808191810097BE
:10B8100029F0FC01FACF80E090E00895CF0108956F
:10B82000DC01ED91FC9111973097A9F020813181D5
:10B83000232B21F41D921C92CF010895A081B18188
:10B840008D919C911197892B11F0FD01F7CF1182F9
:10B850001082CD01089580E090E00895DC01ED9123
:10B86000FC911197309721F0208131812D933C93E9
:10B87000CF010895DC01ED91FC913097A9F0A0E093
:10B88000B0E020813181E617F70741F4109709F401
:10B89000DC012D933C93118210820895211531050E
:10B8A00019F0DF01F901EDCF08950F931F93CF93A6
:10B8B000DF938C01EB010E943A5C19821882C80167
:10B8C0000E94005C009711F4F80101C0FC01D183D3
:10B8D000C083DF91CF911F910F9108950F931F9314
:10B8E000CF93DF93EC018B010E943A5C88819981B0
:10B8F000F8019183808319830883DF91CF911F9191
:10B900000F910895DC01ED91FC9180E090E030977B
:10B9100029F001960190F081E02DF9CF0895FB0107
:10B92000309719F4BA010C946E5C80819181DA0130
:10B930008D939C93518340830895009721F0FC01DF
:10B9400080819181089580E090E0089580913A137C
:10B9500090913B13892B29F41092391310923813CC
:10B9600008950E94A96BE0913A13F0913B13228154
:10B97000338140815181240F351F281B390B0480EE
:10B98000F581E02D309769F04281538160817181AA
:10B99000460F571F481B590B4217530780F79A0150
:10B9A000EECF280F391F30933913209338130895A1
:10B9B00080E992E00C94565BEF92FF920F931F93F5
:10B9C000CF93DF938C01FC0180819181009799F0E6
:10B9D0008A359105D9F0F8011182108283E068C0A0
:10B9E000868197818417950709F049C00480F58105
:10B9F000E02D3097A9F710923B1310923A138AE585
:10BA000090E0F8019183808381E052C0673891F122
:10BA10006238A9F7C0913A13D0913B13E12CF12C75
:10BA2000209769F3CE010E941E7A892BF1F0AE01B6
:10BA300068E88E819F810E94085B892BA1F41F8298
:10BA40001E828C819D81E114F10421F0F701958320
:10BA5000848304C090933B1380933A131D821C820D
:10BA60000E94A65CD7CF0E94D85C7E010C80DD814D
:10BA7000C02DD6CFE0913A13F0913B13BACFF0939B
:10BA80003B13E0933A13A481B581109709F4B7CF23
:10BA900016968D919C9117978417950711F0FD01CB
:10BAA000F2CF14968D919C91159795838483EBCF5B
:10BAB000DF91CF911F910F91FF90EF900895CF9359
:10BAC000DF93EC010E94D85C8E819F8130913A1304
:10BAD00020913B13892B59F0E32FF22F309739F047
:10BAE000EC17FD0781F00480F581E02DF7CF809100
:10BAF0008812909189129F838E833C832D83D093EB
:10BB00003B13C0933A13DF91CF910C94A65CCF9373
:10BB1000DF93EC010E94FE79CE01DF91CF910C946E
:10BB20005F5DCF93DF93EC010E940A7ACE01DF9133
:10BB3000CF910C945F5DCF93DF93EC010E94147A58
:10BB4000CE01DF91CF910C945F5DFC0120813181AA
:10BB5000260F371F318320830C94A65C21E030E050
:10BB6000FC0186819781892B11F020E030E0C9012A
:10BB70000895FC012281338180819181820F931F7E
:10BB80000895FC0180819181089581E090E02091E9
:10BB90003A1330913B13232B11F480E090E0089589
:10BBA00080913A1390913B13892B29F0809138139F
:10BBB00090913913089580E090E00895CF93DF933A
:10BBC000EC01E0913A13F0913B138E179F0769F453
:10BBD0008C819D8190933B1380933A130DC0848197
:10BBE00095818C179D0721F0FC013097C1F706C0A5
:10BBF0008C819D81958384830E94A65C1D821C821A
:10BC00001F821E82DF91CF910895EF92FF920F93D2
:10BC10001F93CF93DF938C017A01FC018081918186
:10BC2000009741F08B34910501F1F80111821082E7
:10BC300083E048C08DE393E10E94F55BEC0120971F
:10BC400051F06C817D81CE0102960E94875D099042
:10BC5000D881C02DF4CF81E080933C138BE490E039
:10BC6000F8019183808381E02DC06838E1F78DE38E
:10BC700093E10E94F55BEC01209781F3CE010296DF
:10BC8000E816F906D9F4BE018DE393E10E943A5C0F
:10BC9000E0908812F09089128A859B859093891292
:10BCA00080938812EC85FD85309719F08E859F85ED
:10BCB0000995F0928912E0928812D0CF0990D8812C
:10BCC000C02DDACFDF91CF911F910F91FF90EF90B0
:10BCD000089510923C138DE393E10E94F15B60E0C4
:10BCE00070E08AE992E00C94355B0F931F93CF9339
:10BCF000DF93EC0100918812109189121B870A874B
:10BD00005D874C873F872E8780913C13882379F08D
:10BD10008AE992E09093891280938812CE0102966C
:10BD20000E94875D109389120093881202C07D8360
:10BD30006C83BE018DE393E10E943A5CBE018DE30A
:10BD400093E1DF91CF911F910F910C94555C0F936C
:10BD50001F93CF93DF93EC0180913C13882391F0E4
:10BD600000918812109189128AE992E090938912C9
:10BD700080938812CE0102960E94915D10938912E1
:10BD800000938812BE018DE393E10E943A5CBE01EC
:10BD90008DE393E1DF91CF911F910F910C94555C4E
:10BDA0000F931F93CF93DF93EC0180913C13882373
:10BDB00091F000918812109189128AE992E0909393
:10BDC000891280938812CE0102960E949B5D109387
:10BDD000891200938812BE018DE393E10E943A5CC0
:10BDE000BE018DE393E1DF91CF911F910F910C94F0
:10BDF000555CCF93DF93EC0180913C13882329F0AD
:10BE0000CE0102960E94DE5D04C01F821E8219864A
:10BE10001886BE018DE393E1DF91CF910C943A5CDB
:10BE2000CF93DF93EC0180913C13882331F0CE0156
:10BE30000296DF91CF910C94AE5D8DE393E10E9469
:10BE4000F55B009739F08C179D0739F0FC01808174
:10BE50009181F7CF81E090E002C080E090E0DF9137
:10BE6000CF9108952F923F924F925F926F927F925F
:10BE70008F929F92AF92BF92CF92DF92EF92FF92FA
:10BE80000F931F93CF93DF93CDB7DEB7E8970FB62D
:10BE9000F894DEBF0FBECDBFEAEDF6E3208131811D
:10BEA00042815381E6EDF6E3508041803280238069
:10BEB000E2EDF6E38081898391819A83A281AB834D
:10BEC0006380EEECF6E3B081BC8381818D83928147
:10BED0009E83A381AF83EAECF6E3B081B8878181CA
:10BEE000898792819A87A381AB87E6ECF6E3B081DC
:10BEF000BC8781818D8792819E87A381AF87E2EC89
:10BF0000F6E3B081B88B8181898B92819A8BA38172
:10BF1000AB8BEEEBF6E3B081BC8B81818D8B928194
:10BF20009E8BA381AF8BEAEBF6E3B081B88F818162
:10BF3000898F92819A8FA381AB8FE6EBF6E3B08174
:10BF4000BC8F81818D8F92819E8FA381AF8FE2EB19
:10BF5000F6E3B081B8A3818189A392819AA3A381DA
:10BF6000ABA3EEEAF6E3B081BCA381818DA39281FD
:10BF70009EA3A381AFA3EAEAF6E3B081B8A78181CB
:10BF800089A792819AA7A381ABA7E6EAF6E3B081DD
:10BF9000BCA781818DA792819EA7A381AFA7E2EA6A
:10BFA000F6E3B081B8AB818189AB92819AAB7380A3
:10BFB000EEE9F6E3B080A18092808380EAE9F6E3BF
:10BFC000F080E180D280C380E6E9F6E3A081AFABE8
:10BFD000B181B8AF128103812BAB3CAB4DAB5EABF3
:10BFE0000E94D76B5EA95F934DA94F933CA93F93E5
:10BFF0002BA92F932F923F924F925F926F922B819A
:10C000002F932A812F9329812F932F812F932E8174
:10C010002F932D812F932C812F932B852F932A855E
:10C020002F9329852F9328852F932F852F932E8546
:10C030002F932D852F932C852F932B892F932A892E
:10C040002F9329892F9328892F932F892F932E8916
:10C050002F932D892F932C892F932B8D2F932A8DFE
:10C060002F93298D2F93288D2F932F8D2F932E8DE6
:10C070002F932D8D2F932C8D2F932BA12F932AA1AE
:10C080002F9329A12F9328A12F932FA12F932EA176
:10C090002F932DA12F932CA12F932BA52F932AA55E
:10C0A0002F9329A52F9328A52F932FA52F932EA546
:10C0B0002F932DA52F932CA52F937F922AA92F93F1
:10C0C00029A92F9328A92F938F929F92AF92BF9265
:10C0D000CF92DF92EF92FF920F931F9328AD2F9391
:10C0E0002FA92F939F938F937F936F93A4EAB4E329
:10C0F0008C911F928F93E3EAF4E380811F928F93D8
:10C100008DE191E19F938F930E948A99EAE0F7E392
:10C110002081318142815381E6E0F7E35080418004
:10C1200032802380EAEFF6E3908081807280638022
:10C13000E6EFF6E38081898391819A83A281AB83C4
:10C14000B381BC83E2EFF6E380818D8391819E838E
:10C15000A281AF83B381B887EEEEF6E38081898751
:10C1600091819A87A281AB87B381BC87EAEEF6E31F
:10C1700080818D8791819E87A281AF87B381B88BA3
:10C18000E6EEF6E38081898B91819A8BB280A38061
:10C19000E2EEF6E3F080E180D280C380EEEDF6E3DC
:10C1A000A081AB8BB181BC8B128103810FB6F89457
:10C1B000DEBF0FBECDBF2BAB3CAB4DAB5EAB0E9429
:10C1C000D76B5EA95F934DA94F933CA93F932BA9D1
:10C1D0002F932F923F924F925F926F927F928F9206
:10C1E0009F922C812F932B812F932A812F9329812A
:10C1F0002F9328852F932F812F932E812F932D817D
:10C200002F932C852F932B852F932A852F93298568
:10C210002F9328892F932F852F932E852F932D854C
:10C220002F93AF92BF922A892F9329892F93CF9270
:10C23000DF92EF92FF920F931F932C892F932B89FC
:10C240002F939F938F937F936F93A4EAB4E38C9182
:10C250001F928F93E3EAF4E380811F928F938EEA1B
:10C2600090E19F938F930E948A990FB6F894DEBF56
:10C270000FBECDBFE8960FB6F894DEBF0FBECDBFA0
:10C28000DF91CF911F910F91FF90EF90DF90CF90B2
:10C29000BF90AF909F908F907F906F905F904F90E6
:10C2A0003F902F90089580E38093F3130895CF93E8
:10C2B000DF936091F31370E0C0E3D0E0C61BD70BAF
:10C2C0006F5B7C4EAE010E94C398CE01DF91CF918F
:10C2D0000895CF92DF92EF92FF920F931F93CF9327
:10C2E000DF937C01C090F613D090F7136091F313A5
:10C2F00070E0E601E096C61BD70BC138D105D8F433
:10C3000000E310E0061B170B6F5B7C4EA8010E9438
:10C31000C39860913F13709140138091F4139091F2
:10C32000F513680F791FA601C701800F911F0E94A6
:10C33000C398CE0102C080E090E0DF91CF911F91C1
:10C340000F91FF90EF90DF90CF9008959091F313AD
:10C35000980F9093F31308954091F6135091F713AB
:10C360004817590798F02091F4133091F513280FCE
:10C37000391F3093F5132093F413481B590B509336
:10C38000F7134093F61381E090E0089580E090E089
:10C3900008959093F7138093F61308958091F41302
:10C3A0009091F5138F589C4E08958091F31390E06F
:10C3B0008F5B9C4E089581E090E020913F13309177
:10C3C00040132157334111F480E090E008950E941A
:10C3D000DB61892B61F060913F13709140134091B4
:10C3E000F6135091F71381E793E10C94C3982091D1
:10C3F000F4133091F51321153105B9F08091F6133E
:10C400009091F713C096E1E7F3E1AF014154534136
:10C410004817590734F4DF01A20FB31F4C91419321
:10C42000F4CF1092F5131092F413089580913F13F6
:10C430009091401308958091F6139091F713089509
:10C440009091F31380E3891B089520E38091F31307
:10C45000281B8091F6139091F713820F911D089578
:10C460001F93CF93DF93EC011091F313812F90E092
:10C470008C179D076CF00E9425628C0F9D1F8138E0
:10C48000910530F41C1B1093F31381E090E002C07F
:10C4900080E090E0DF91CF911F910895CF93DF93DB
:10C4A000EDEAF4E31192119284E3ED3DF807D1F740
:10C4B000C5EAD4E36CE073E0CE010E94E158229615
:10C4C00084E3CD3AD807B1F7DF91CF910895109268
:10C4D000F5131092F4131092F7131092F61380E3F1
:10C4E0008093F31381E793E19093401380933F137C
:10C4F0000C944E62EF92FF920F931F93CF93DF93B2
:10C5000000D0CDB7DEB78C0169837A830E94676261
:10C510006981E62E7A81F72E81E8E816F10418F099
:10C5200080E8E82EF12CA701B80180913F1390918B
:10C5300040130E94C398F092F713E092F613C701DC
:10C540000F900F90DF91CF911F910F91FF90EF907F
:10C5500008950F931F93CF93DF938C01EB010E94FB
:10C5600067621093401300933F13D093F713C09367
:10C57000F613DF91CF911F910F91089520E3EDEA1B
:10C58000F4E3DC0101900D922A95E1F788E0E5EAF9
:10C59000F4E3DB0101900D928A95E1F7089520E321
:10C5A000FC01ADEAB4E301900D922A95E1F788E031
:10C5B000FB01A5EAB4E301900D928A95E1F7089595
:10C5C000E82FF0E0EE0FFF1FE355FB4C7183608313
:10C5D00081E090E00895E82FF0E0EE0FFF1FE355B3
:10C5E000FB4C80819181089590E0880F991F8B58B2
:10C5F0009B4C0E94E15881E090E0089590E0880F04
:10C60000991F8B589B4C08958115910511F0019746
:10C61000F1F70895E091E034F091E1349081809158
:10C62000DF3489230895E091DD34F091DE34808198
:10C630009091DF34892B8083E091E234F091E334F0
:10C6400080819091DF34892B80830895E091DD34DF
:10C65000F091DE3490818091DF348095892380834E
:10C66000E091E234F091E33490818091DF34809561
:10C670008923808308951F93CF93DF93E091DD3466
:10C68000F091DE3490818091DF348095892380831E
:10C69000E091E234F091E33480819091DF34892B92
:10C6A00080838FEB93E00E9404631FB7F894E091BE
:10C6B000E234F091E33490818091DF3480958923D6
:10C6C000808383E890E00E940463E091E034F0917D
:10C6D000E134D081C091DF341FBF78948BE393E0C5
:10C6E0000E940463E091E034F091E1349081809104
:10C6F000DF34982319F08D2F8C2301C081E0DF9166
:10C70000CF911F9108955093E3344093E234709396
:10C71000DE346093DD349093E1348093E03481E043
:10C7200001C0880F2A95EAF78093DF340C943B63AD
:10C73000CF93DF93C82FDFB7F894E091E234F09104
:10C74000E33480819091DF34892B808383E090E013
:10C750000E940463CC2351F0E091E234F091E33481
:10C7600080819091DF3490959823908387E190E0C9
:10C770000E940463E091E034F091E1348081909173
:10C78000DF34892309F4C0E089E590E00E94046366
:10C79000E091E234F091E33480819091DF34909520
:10C7A00098239083DFBF8BE390E00E9404638C2F7B
:10C7B000DF91CF910895CF93DF93C82FD8E08C2FCE
:10C7C00081700E949863C6958111C068D150B9F7F5
:10C7D0008C2FDF91CF9108958FEF0C94DB63DF9264
:10C7E000EF92FF920F931F93CF93DF93E82EEB010D
:10C7F0000E943B6381112FC080EF0E94DB63F12C0C
:10C8000010E488EFD82ED10E81E00E949863082FA3
:10C8100081E00E949863882319F0002361F01DC015
:10C82000011109C01E1528F0888180FF04C0E1169F
:10C8300011F0F12E01E0802F0E9498639881969567
:10C8400001119068988311501D11DECF21961111AE
:10C85000D8CF8F2D03C08FEF01C08EEFDF91CF9126
:10C860001F910F91FF90EF90DF900895FF920F932B
:10C870001F93CF93DF93F82EEB010E943B63209729
:10C8800069F085E50E94DB638E01085F1F4F899187
:10C890000E94DB63C017D107D1F703C08CEC0E9464
:10C8A000DB638F2DDF91CF911F910F91FF900C943F
:10C8B000DB630F931F93CF93DF93DB01EC91119612
:10C8C0009C911197F0E0F92B803181F4BF016E7FCC
:10C8D000E3E0660F771FEA95E1F716969C911697AD
:10C8E000ECE0F0E0E91BF109E60FF71FF7FF07C0E6
:10C8F00091E0EA019883F195E195F10902C0EA011E
:10C900001882883279F414968C91982F907690360C
:10C9100049F086FF02C0EE7F05C085FF02C0EC7FB4
:10C9200001C0E87FCF0144E0969587954A95E1F7ED
:10C93000D9018C93EF70E801E88380E0DF91CF911B
:10C940001F910F9108950F931F93CF93DF93EC01E5
:10C950008B01B80188810E94EF63888381508D3FED
:10C9600030F4F8018081883211F0803191F7DF9145
:10C97000CF911F910F910895CF93DF93EC010E9407
:10C980003B63BE0184EB0E94366481E00E949863A1
:10C99000C82F0E943B6381E0C11101C080E0DF919C
:10C9A000CF9108951F93CF93DF9300D0CDB7DEB71B
:10C9B000182F69837A830E943B630E940A6369810E
:10C9C0007A81882341F084E40E943664113029F092
:10C9D0000E94136302C082E001C080E00F900F90BC
:10C9E000DF91CF911F9108954F925F926F927F9246
:10C9F0008F929F92AF92BF92CF92DF92EF92FF926F
:10CA00000F931F93CF93DF93CDB7DEB729970FB660
:10CA1000F894DEBF0FBECDBF6C015B014A018901F6
:10CA20000E943B63B6018EEB0E943664CE010196F4
:10CA30007C013E019AE0690E711C27010E94EC63A3
:10CA4000F70181937F01E615F705C1F769E070E012
:10CA5000C2010E948F7E811109C09401A501B2011B
:10CA6000F60180810E94596480E001C083E029962C
:10CA70000FB6F894DEBF0FBECDBFDF91CF911F91EF
:10CA80000F91FF90EF90DF90CF90BF90AF909F906D
:10CA90008F907F906F905F904F9008955F926F920C
:10CAA0007F928F929F92AF92BF92CF92DF92EF923E
:10CAB000FF920F931F93CF93DF93CDB7DEB72997E4
:10CAC0000FB6F894DEBF0FBECDBF582E6B015A01D2
:10CAD000890160E070E08EEB0E943664CE01019621
:10CAE0007C014E019AE0890E911C37010E94EC6393
:10CAF000F70181937F01E815F905C1F769E070E05E
:10CB0000C3010E948F7E811108C09501A601B30167
:10CB1000852D0E94596480E001C083E029960FB6FC
:10CB2000F894DEBF0FBECDBFDF91CF911F910F9163
:10CB3000FF90EF90DF90CF90BF90AF909F908F903D
:10CB40007F906F905F9008950F931F93CF93DF9323
:10CB5000CDB7DEB728970FB6F894DEBF0FBECDBFB6
:10CB6000182F062F98E0E8E1F3E0DE01119601901E
:10CB70000D929A95E1F7242F332727FD309541E751
:10CB800052E0249FC001259F900D349F900D1124E9
:10CB900064E670E00E94AD92CB0144E6049F800DF4
:10CBA000911D1124FE013196AE01475F5F4F6191E7
:10CBB00070E02617370711F4019603C0E417F50754
:10CBC000B1F7112319F091958195910928960FB627
:10CBD000F894DEBF0FBECDBFDF91CF911F910F91B3
:10CBE0000895EF92FF920F931F93CF93DF93CDB7EA
:10CBF000DEB72B970FB6F894DEBF0FBECDBFF82E71
:10CC0000E92E682F792F88E08F0D0E94D264882347
:10CC100019F084E391E243C066E471E48FE090E0B0
:10CC20000E945C668E01075F1F4F9801AE01465F50
:10CC30005F4FBE01655F7F4F8F2D9E2D0E94F46474
:10CC40008111E7CF88E0E8E1F3E0DE011196019081
:10CC50000D928A95E1F7498521E732E0429FC001B4
:10CC6000439F900D112464E670E00E94AD928A8586
:10CC700094E6899F600D711D1124FE01319681910A
:10CC8000481303C06F5F7F4F03C0E017F107B9F788
:10CC90008B85882319F0719561957109CB012B96CD
:10CCA0000FB6F894DEBF0FBECDBFDF91CF911F91BD
:10CCB0000F91FF90EF900895DC01CB018115910554
:10CCC000A105B10529F081509040A040B040D9F7AE
:10CCD00008959B01AC011092B90060E072E18AE70F
:10CCE00090E00E94C19220513109410951095695A5
:10CCF0004795379527952093B800089594EA909327
:10CD0000BC0040EA56E861E070E09091BC0097FDFD
:10CD10000BC0415051096109710941155105610567
:10CD2000710599F781E008959091B900987F983046
:10CD300011F09031B9F78093BB0084E88093BC0078
:10CD400080EA96E8A1E0B0E02091BC0027FD08C091
:10CD50000197A109B1090097A105B105A9F7E2CF93
:10CD60008091B900887F883111F08034D9F680E055
:10CD7000089524EA34E844E92093BC009091BC0073
:10CD800097FFFCCF9091B900987F983011F09031C7
:10CD900099F78093BB003093BC009091BC0097FF43
:10CDA000FCCF9091B900987F903211F0983539F40A
:10CDB0004093BC009091BC0094FDFCCFDDCF089562
:10CDC0000C947E6684E98093BC008091BC0084FD55
:10CDD000FCCF08958093BB0084E88093BC008091D1
:10CDE000BC0087FFFCCF9091B900987F81E098321A
:10CDF00009F480E0089584EC8093BC008091BC002D
:10CE000087FFFCCF8091BB00089584E88093BC002D
:10CE10008091BC0087FFFCCF8091BB000895E0E1CA
:10CE2000DC01FD91CD01F0933F01E150C9F7809104
:10CE30003C018F7D80933C0180913C01877F8093F2
:10CE40003C01FB0180E1919190933E018150D9F723
:10CE500080913C01806880933C0180913D0180FF7E
:10CE6000FCCF4051510980913C01806280933C018C
:10CE700080913C01877F80933C01141615069CF439
:10CE8000FB0180E1919190933E018150D9F780910F
:10CE90003C01806880933C0180913D0180FFFCCF84
:10CEA00040515109EACFF90180E190913E019193FF
:10CEB0008150D9F781E090E008950F931F93CF93AD
:10CEC000DF93EC018CE70E94B9668CE70E94EA666A
:10CED0008E01005F1F4F89910E94EA66C017D1073B
:10CEE000D1F7DF91CF911F910F910C94E2668130C1
:10CEF00019F440E050E002C040EC50E060E070E027
:10CF00008CE790E00C949913813019F44EE050E0D6
:10CF100002C048E050E060E070E08CE790E00C94E4
:10CF2000991341E050E060E070E08CE790E00E94EF
:10CF300099136AE67AE080E090E00C945C6648E33E
:10CF400050E060E070E08CE790E00E94991349E3C4
:10CF500050E060E070E08CE790E00E94991344E1BB
:10CF600050E060E070E08CE790E00E94991348E7A1
:10CF700050E060E070E08CE790E00E9499134EE58D
:10CF800050E060E070E08CE790E00E9499134DE67D
:10CF900050E060E070E08CE790E00E9499136CE153
:10CFA0007AE186E090E00E945C664CE050E060E050
:10CFB00070E08CE790E00E94991341E050E060E05F
:10CFC00070E08CE790E00E94991346E050E060E04A
:10CFD00070E08CE790E00E9499136AE67AE080E0C6
:10CFE00090E00C945C66CF93DF93CDB7DEB7A29749
:10CFF0000FB6F894DEBF0FBECDBF81E1E8EBF9E0DC
:10D00000DE01529601900D928A95E1F781E1E9ECFB
:10D01000F9E0DE01119601900D928A95E1F70E94E8
:10D020009F67CE0142960E945D6782E00E9477670B
:10D030006AE67AE080E090E00E945C66CE010196AC
:10D040000E945D6760E17EEA88E290E00E945C6693
:10D0500080E00E94846760E17EEA88E290E00E94BE
:10D060005C664EE050E060E070E08CE790E00E948B
:10D070009913A2960FB6F894DEBF0FBECDBFDF9115
:10D08000CF910895CF92DF92EF92FF920F931F936B
:10D09000CF93DF9300D01F92CDB7DEB7F82E042FC9
:10D0A000122F213031F0223031F0243031F028308D
:10D0B00031F090E005C091E003C092E001C093E040
:10D0C0000C3059F00E3011F4946007C0003111F4A7
:10D0D000986003C0023109F49C60613059F06230FD
:10D0E00011F4906207C0633011F4906403C064309F
:10D0F00009F490669068692F70E023E030E0AE019B
:10D100004F5F5F4F8F2D90E00E94B01369E07AE18E
:10D1100080E090E00E945C668F2D8160F82E0E9476
:10D120007E660E94FB6689830E94FB668A830231C9
:10D1300019F40E94FB668B830E94FB6687FDF1CF8A
:10D140000E9405670E94E26669E07AE180E090E073
:10D150000E945C668F2D0E947E660E94FB6689831A
:10D160000E94FB668A83023119F40E9405678B8353
:10D170000E9405670E94E26639812A81023149F5E1
:10D18000832F90E0A0E0B0E04B817727662731FF46
:10D190000EC030E0322F2227620F731F811D911DB8
:10D1A000640F711D811D911D8C6F9F6F0BC030E04E
:10D1B000322F2227620F731F811D911D640F711D75
:10D1C000811D911D0E94DB8F20E83FEF4FEF57E458
:10D1D00020C0632F70E0762F6627620F711D8827AD
:10D1E00077FD8095982F0E94DB8F0C3029F420E08A
:10D1F00030EE4FEF54E40DC00E3029F420E038EF4C
:10D200004FEF55E406C0003131F420E03EEF4FEF20
:10D2100056E40E943C8F2FE632E143E050E40E9446
:10D22000BD916B017C01612F70E080E090E00E9475
:10D23000DB8F9B01AC01C701B6010E943C8F0F90B0
:10D240000F900F90DF91CF911F910F91FF90EF9072
:10D25000DF90CF900895E6E4F1E080812081908115
:10D260003081829586958695837022952F70822BCA
:10D27000832B92959F70892B08950F931F93CF93C3
:10D28000DF9300D0CDB7DEB746E06CE080E00E94CF
:10D290006D6C89E18093C4001092C50082E0809398
:10D2A000C00080E00E94FA6C0E94996B84B784B73A
:10D2B00084B784B784B7E4E6FDE322E432E4318343
:10D2C00020833A968DB79EB70A97E817F907B8F307
:10D2D0008AED99E09F938F938AE692E19F938F93D3
:10D2E0000E948A990E94D27A0E948D5A60E070E072
:10D2F00080E992E00E94355B0E94695EE091200324
:10D30000F091210309950E942B6990E00E940E7B09
:10D31000CE0101960E94CE6A0F900F900F900F9051
:10D32000882341F08AE492E19F938F930E948A9927
:10D330000F900F90CE0101960E94FC580E94DC6A6B
:10D340008C010E94D86AAE014F5F5F4FB8010E9406
:10D35000C46F0E94486A0E94A56F0E94E06A0E9402
:10D36000FE708DE392E19F938F930E948A998A8148
:10D370001F928F9309E312E11F930F930E948A99E2
:10D3800089811F928F931F930F930E948A9987E33D
:10D3900092E19F938F930E948A990E94127BE09161
:10D3A0005D03F0915E030995E0914F03F091500306
:10D3B0000995E0913603F091370309950E940571B4
:10D3C000182F0E94A26F1F921F931F928F9380911C
:10D3D0005C038F9380915B038F9380914E038F93B7
:10D3E00080914D038F938CE192E19F938F930E94E4
:10D3F0008A99E0916703F09168030FB6F894DEBF55
:10D400000FBECDBF309791F00995BC0180E890E048
:10D410000E9499927F936F9389E092E19F938F93FB
:10D420000E948A990F900F900F900F9087E092E1E1
:10D430009F938F930E948A9960E070E086EE92E05D
:10D440000E94355B8AEF92E00E94E2798FEF91E1D2
:10D450009F938F930E948A990F900F900F900F9037
:10D460000F900F90DF91CF911F910F9108957F93AF
:10D470006F939F938F9389EF91E19F938F930E9476
:10D480008A990F900F900F900F900F900F90089522
:10D490001F93CF93DF93CDB7DEB7A0970FB6F89465
:10D4A000DEBF0FBECDBF83E690E00E94F69A182F34
:10D4B000282F35EF380F303108F0982F9095291725
:10D4C00009F461C085E892E19F938F930E948A9945
:10D4D000EAECF2E10F900F90DE01119684918D93AA
:10D4E000319682E1E23DF807C9F7F89448E050E050
:10D4F0006FE770E0CE0101960E94FC9AECEBF2E13E
:10D50000DE01119684918D93319682E1EA3CF80711
:10D51000C9F74EE050E061E770E0CE0101960E944D
:10D52000FC9AE2EBF2E1DE01119684918D93319643
:10D5300082E1EC3BF807C9F74AE050E067E670E0AB
:10D54000CE0101960E94FC9A6DEC7BEA81E690E0A8
:10D550000E94149B60E070E08FE590E00E94149BB5
:10D5600060E08EE590E00E94069B60E070E085E65A
:10D5700090E00E94149B1AE16AE175EE83E690E068
:10D580000E94149B7894812FA0960FB6F894DEBF6A
:10D590000FBECDBFDF91CF911F910895F89442E067
:10D5A00050E06FE770E00E94DE9A789480E0089582
:10D5B00081E690E00C94F69A8FE590E00C94F69A50
:10D5C0008EE590E00C94EE9A4091F2345091F33451
:10D5D0006091F4347091F53490E0A0E0B0E0480F31
:10D5E000591F6A1F7B1F4093F2345093F3346093AA
:10D5F000F4347093F5344091EE345091EF346091EF
:10D60000F0347091F134480F591F6A1F7B1F40930B
:10D61000EE345093EF346093F0347093F1342091F2
:10D6200092362223A1F04091EA345091EB3460917C
:10D63000EC347091ED34480F591F6A1F7B1F4093E3
:10D64000EA345093EB346093EC347093ED340895E6
:10D650001F920F920FB60F9211240BB60F922F93B9
:10D660003F934F935F936F937F938F939F93AF936A
:10D67000BF93EF93FF938091FA139091FB13019660
:10D680009093FB138093FA138091F9138F5F80932B
:10D69000F9138038A9F41092F9138091F234909123
:10D6A000F334A091F434B091F5340196A11DB11D6D
:10D6B0008093F2349093F334A093F434B093F53420
:10D6C000809192368823E1F08091F8138F5F8093E8
:10D6D000F8138038A9F41092F8138091EA349091ED
:10D6E000EB34A091EC34B091ED340196A11DB11D45
:10D6F0008093EA349093EB34A093EC34B093ED3400
:10D700000E94C55D892B11F00E94D85CFF91EF91BA
:10D71000BF91AF919F918F917F916F915F914F9149
:10D720003F912F910F900BBE0F900FBE0F901F9047
:10D730001895F8941092B60016BC83EF87BD82E06E
:10D7400084BD94E095BD95B395BB80936E007894AD
:10D7500008958091FA139091FB132091FA13309160
:10D76000FB1382179307A9F70895009751F022E35E
:10D7700030E000002150310921153105D1F7019722
:10D78000F4CF08950F931F93CF93DF93EC010E9482
:10D79000A96B8C010E94A96B801B910B8C179D07B4
:10D7A000C8F3DF91CF911F910F91089508950F93C2
:10D7B0001F936091F2347091F3348091F43490911E
:10D7C000F5340091F2341091F3342091F434309117
:10D7D000F534601771078207930759F71F910F916E
:10D7E00008951F920F920FB60F9211241092BC024F
:10D7F0000F900FBE0F901F9018951F920F920FB6AB
:10D800000F9211240BB60F922F933F934F935F9378
:10D810006F937F938F939F93AF93BF93EF93FF93F8
:10D82000E091B202F091B3028081E091BD02F091EB
:10D83000BE02309709F00995FF91EF91BF91AF912A
:10D840009F918F917F916F915F914F913F912F9118
:10D850000F900BBE0F900FBE0F901F9018951F9248
:10D860000F920FB60F9211241092C9020F900FBEA3
:10D870000F901F9018951F920F920FB60F921124C0
:10D880000BB60F922F933F934F935F936F937F93BA
:10D890008F939F93AF93BF93EF93FF93E091BF025A
:10D8A000F091C0028081E091CA02F091CB023097E2
:10D8B00009F00995FF91EF91BF91AF919F918F91E1
:10D8C0007F916F915F914F913F912F910F900BBE80
:10D8D0000F900FBE0F901F9018959DE0899FF0014B
:10D8E0001124EE54FD4FA281B3811C92A481B58115
:10D8F0006C93A681B78188ED8C93A085B1854C93FC
:10D9000012861486138608959DE0899FF0011124E4
:10D91000EE54FD4F81E08287A081B1816C933A96ED
:10D9200080818111FDCF08951F93CF93DF93182F2E
:10D93000EB01FE018491882339F0FE016491812F6F
:10D940000E94846C2196F5CFDF91CF911F910895AD
:10D950001F93CF93DF93182FEB018881882369F001
:10D960008A3021F46DE0812F0E94846C69916D30C2
:10D97000A1F3812F0E94846CF0CFDF91CF911F9192
:10D980000895CF93DF93CDB7DEB79E01285F3F4F59
:10D990004E815F8160E470E08CEF93E10E94479AD2
:10D9A0006CEF73E18D810E94A86CDF91CF91089597
:10D9B000CF93C82F8A3031F46DE080913C140E94DF
:10D9C000846C02C08D3029F06C2F80913C140E9431
:10D9D000846C80E090E0CF9108959DE0899FF001F4
:10D9E0001124EE54FD4F748763870895682F80E0FB
:10D9F0000C94846C80933C1484EA92E090935F3D95
:10DA000080935E3D089584B7877F84BF88E10FB619
:10DA1000F89480936000109260000FBE08952FE08C
:10DA200088E190E00FB6F894A895809360000FBE4F
:10DA3000209360000895A895089588E10FB6F894A2
:10DA400080936000109260000FBE0895F89428E063
:10DA500088E190E00FB6F894A895809360000FBE1F
:10DA600020936000FFCF8091FD348091FD3490E0E1
:10DA7000089540E06FE181E491E00C949A72E9E34B
:10DA8000F1E0808180818D7F80838DE090E001973F
:10DA9000F1F723E040E06FE182E491E00E94A4729C
:10DAA00083E090E00197F1F708959091390191FD9D
:10DAB0000AC0282F803108F02FE040E06FE085E4B5
:10DAC00091E00C94A47208958091390181FD0EC0FB
:10DAD00040E06FE181E491E00E949A72282F2F7E4E
:10DAE00081E090E0213021F080E0089580E090E036
:10DAF00008958091390181FD10C040E06FE181E41B
:10DB000091E00E949A728F3131F0982F9F7E915050
:10DB100081E0923018F480E0089581E008950E9439
:10DB2000796D8823E1F30895CF93DF93C82F0E9486
:10DB30008F6D0E94396DD82FC81789F1C83019F43C
:10DB40000E943F6D25C0C93121F4863189F429E056
:10DB500005C0C63169F4893159F426E040E06FE12F
:10DB600082E491E00E94A472E3E0F0E03197F1F7E3
:10DB70002C2F40E06FE182E491E00E94A472D83043
:10DB800019F4E9E6F1E002C0E3E0F0E03197F1F7E3
:10DB90000E94396D8C1719F083E490E002C080E494
:10DBA00090E0DF91CF9108950E948F6D1092923690
:10DBB0000E943F6D8091390182608093390180918C
:10DBC00015378823D9F18091940090919500409168
:10DBD00026375091273784179507A0F48091F236A5
:10DBE0009091F336A091F436B091F5368C57914E62
:10DBF000AF4FBF4F8093F2369093F336A093F43635
:10DC0000B093F5362091940030919500241B350B8C
:10DC10008091F2369091F336A091F436B091F536BA
:10DC2000820F931FA11DB11D8093F2369093F3369E
:10DC3000A093F436B093F5361092153780911737CC
:10DC40008823D9F1809194009091950040912A37D2
:10DC500050912B3784179507A0F48091FA36909154
:10DC6000FB36A091FC36B091FD368C57914EAF4FEC
:10DC7000BF4F8093FA369093FB36A093FC36B09357
:10DC8000FD362091940030919500241B350B809136
:10DC9000FA369091FB36A091FC36B091FD36820F9A
:10DCA000931FA11DB11D8093FA369093FB36A0936C
:10DCB000FC36B093FD361092173708958091923656
:10DCC000882381F08091C014811104C00E94796D75
:10DCD000811106C081E08093BE1481E090E0089538
:10DCE0000E94D46D80E090E008958091940090911E
:10DCF000950090932B3780932A3721E02093173794
:10DD00008091390181FD08C08091390181FD1AC0DF
:10DD100086E10E94946D16C0209391368091940004
:10DD2000909195009093273780932637209315374D
:10DD3000809139018D7F80933901809191368111D5
:10DD4000FCCFE2CF81E080939236089580919236A5
:10DD500081110AC08091C014882321F081E0809352
:10DD6000BF1402C00E94756E81E090E008951F9379
:10DD7000CF93DF931F92CDB7DEB78FB789838091A2
:10DD8000C014811126C0F89480919236882351F0F6
:10DD90008091390181FD1BC00E94796D8823B9F003
:10DDA00080E003C00E94A66E81E02091470191E0CF
:10DDB0002E3008F090E0192F119581110E945E6EAF
:10DDC000107429F089818FBF81E090E004C08981BF
:10DDD0008FBF80E090E00F90DF91CF911F91089569
:10DDE0008091BF14882321F00E94756E1092BF1499
:10DDF0008091BE14882321F00E94D46D1092BE142D
:10DE00001092C01408950F931F93AB0121E020934B
:10DE1000C0140091D6361091D7362091D836309163
:10DE2000D9360F5F1F4F2F4F3F4F0093D6361093B9
:10DE3000D7362093D8363093D93622E0260F27FFE5
:10DE40000CC080918F3690919036019690939036C9
:10DE500080938F360FEF1FEF07C0BC018DE394E175
:10DE60000E94C39800E010E00E94F06EC8011F916C
:10DE70000F9108958093C21408950E94396D8230E5
:10DE800011F0823111F480E0089581E00895089541
:10DE90008FEF80934E0122E044E060EF8CE691E04A
:10DEA0000E94A47225E041E06EE08CE290E00E94C6
:10DEB000A47280E880936F018091460180936D0188
:10DEC00021E045E060E284E491E00C94A4728DEFDF
:10DED00093E00197F1F70E9490721092063510922C
:10DEE000883510920A361092053510920435E9E310
:10DEF000F1E080818E7F808380818D7F80838DE0C3
:10DF000090E00197F1F780818160808323E040E019
:10DF10006FE182E491E00E94A4728DEF93E001979B
:10DF2000F1F780915D0180915E010E94486F60E091
:10DF300070E08CEC92E00E94355B0E94756E81E08F
:10DF400090E008958091C1140895CF93DF931F92BC
:10DF5000CDB7DEB789830E948F6D89818093C1140C
:10DF6000282F40E06FE188E491E00F90DF91CF919E
:10DF70000C94A4720E94A56F8091390181FD03C0A9
:10DF800086E00C94946D0895FA0180936201909359
:10DF9000630160936001709361013097C1F08081EB
:10DFA00080936B01818180936A01828180936901F2
:10DFB0008381809368018481809367018581809348
:10DFC000660186818093650187818093640108954D
:10DFD0008CEC92E00E94565B81E08093FD3480914E
:10DFE000FE349091FF3401969093FF348093FE3479
:10DFF00081E090E008958091053592E8899FF001D5
:10E000001124EA5FFA4C10828F5F833018F48093FA
:10E01000053502C010920535E091053582E8E89F8C
:10E02000F0011124EA5FFA4C808181110C94E86FB1
:10E030001092FD3408951F93CF93DF9320910535FF
:10E0400012E8129F90011124D901AA5FBA4C4C9199
:10E05000411103C00E94FB6F93C05091390151FDE3
:10E060008FC050919236552309F48AC047FF16C0DD
:10E070000E94FB6F8091C6369091C736A091C8363A
:10E08000B091C9360196A11DB11D8093C6369093FB
:10E09000C736A093C836B093C93672C04330B0F4C7
:10E0A0000E94FB6F8091C2369091C336A091C43616
:10E0B000B091C5360196A11DB11D8093C2369093D3
:10E0C000C336A093C436B093C5365AC050E0EA01B7
:10E0D00022976C177D07B0F40E94FB6F8091BE36CB
:10E0E0009091BF36A091C036B091C1360196A11D66
:10E0F000B11D8093BE369093BF36A093C036B093C7
:10E10000C1363EC0B901695F7A4C0E94C398E09164
:10E1100005351E9FF0011124EA57FA4C8081809347
:10E12000F6340E94FB6F809147018093F734909101
:10E13000FC34992311F0891710F48093FC3460911A
:10E14000F73470E084E00E94E0626091F63470E0A1
:10E1500083E00E94E0624091DA365091DB366091B4
:10E16000DC367091DD364F5F5F4F6F4F7F4F4093CE
:10E17000DA365093DB366093DC367093DD3602C0BE
:10E18000C0E0D0E0CE01DF91CF911F910895CF93F1
:10E19000DF93EC01888199810097E9F08730954001
:10E1A00021F01982188283E026C06238C1F41092EF
:10E1B000FD340E9467620E94CE6160E870E00E94B8
:10E1C0001B70181619066CF40E94C961E091610376
:10E1D000F0916203099587E095E09983888381E057
:10E1E0000AC08091FA349091FB3401969093FB34ED
:10E1F0008093FA34F0CFDF91CF91089591E090931E
:10E20000C0140E94556D0C94F06E8091390181FD0F
:10E2100006C040E06FE085E491E00C949A7280E1E2
:10E2200008950F931F93CF93DF93182F21E020932E
:10E23000C014009192368091390181FF16C08091FF
:10E2400094009091950090932737809326372093E0
:10E25000153720939136809139018D7F8093390154
:10E26000809191368111FCCF00E00E948F6D8091EA
:10E270009236882309F43FC0809117378823D9F15B
:10E280008091940090919500E0912A37F0912B377E
:10E290008E179F07A0F44091FA365091FB3660919B
:10E2A000FC367091FD364C57514E6F4F7F4F409367
:10E2B000FA365093FB366093FC367093FD3620910E
:10E2C0009400309195002E1B3F0B4091FA365091EF
:10E2D000FB366091FC367091FD36420F531F611D75
:10E2E000711D4093FA365093FB366093FC36709361
:10E2F000FD36109217378091390181FD03C089E105
:10E300000E94946D86E00E94EB62892B51F00E947E
:10E310000571C82F86E00E94EB6281500E94556D06
:10E3200002C0C0E0D0E0209194003091950030937D
:10E3300029372093283781E080931637F89480910D
:10E340003901826080933901809139018D7F8093FA
:10E35000390162E0610F8DE394E10E94D3727894F9
:10E3600020918C3630918D362F5F3F4F30938D3614
:10E3700020938C360E948F6D45E060EE82E491E040
:10E380000E949A72182F86E00E94EB62892B19F086
:10E390008C2F0E94556D002319F00E94756E02C0EB
:10E3A0000E94D46D809116378823D9F18091940012
:10E3B00090919500E0912837F09129378E179F07AB
:10E3C000A0F44091F6365091F7366091F83670918E
:10E3D000F9364C57514E6F4F7F4F4093F63650935E
:10E3E000F7366093F8367093F936209194003091A7
:10E3F00095002E1B3F0B4091F6365091F7366091F9
:10E40000F8367091F936420F531F611D711D40930C
:10E41000F6365093F7366093F8367093F9361092CB
:10E42000163780919236882361F0209194003091C4
:10E43000950030932B3720932A3781E0809317374C
:10E4400007C023E040E06FE182E491E00E94A47203
:10E450000E94F06E1130E9F01330A9F48091CE36AD
:10E460009091CF36A091D036B091D1360196A11DB2
:10E47000B11D8093CE369093CF36A093D036B09313
:10E48000D13612E009C0153031F0173029F411E00F
:10E4900003C010E001C013E0812F90E0DF91CF9125
:10E4A0001F910F910895CF93DF93EB010E94036FAB
:10E4B000009729F4CE010E941171009751F020912C
:10E4C0008F36309190362F5F3F4F309390362093A8
:10E4D0008F36DF91CF910895CF93DF93809192365D
:10E4E000811104C00E94A66ED1E001C0D0E00E945C
:10E4F000396D863111F0813119F4C091470109C09D
:10E5000040E06FE186E491E00E949A72C82FCC0F40
:10E51000C80FD1110E945E6E8C2FDF91CF910895AC
:10E520001092C4141092C314EFE6F0E08081806270
:10E5300080830895FC018081862390E002C0959538
:10E5400087954A95E2F70895F894FC015081362F9B
:10E5500030955323042E01C0220F0A94EAF7262394
:10E56000522B50837894089540917B01FC01419394
:10E57000A0E8B1E050E8540F9D012F5F3F4F6C9130
:10E580006193521711F0D901F7CF4150E42FF0E019
:10E59000E058FE4F2181FC01E058FF4F2083319667
:10E5A00021E02083089560938001E1E8F1E0615863
:10E5B0009F012F5F3F4FDC014D91CD0140836217DA
:10E5C00011F0F901F5CF08951F920F920FB60F9237
:10E5D00011240BB60F922F933F934F935F936F933A
:10E5E0007F938F939F93AF93BF93EF93FF9380910C
:10E5F00047018093F7348091043522E8829FC0015F
:10E6000011248A5F9A4C0E94B472809104358F5F06
:10E61000833018F48093043502C0109204350E94B0
:10E62000E86FFF91EF91BF91AF919F918F917F9193
:10E630006F915F914F913F912F910F900BBE0F9073
:10E640000FBE0F901F9018951F920F920FB60F924A
:10E6500011240F900FBE0F901F9018951F920F92CC
:10E660000FB60F9211240F900FBE0F901F901895A8
:10E670001F920F920FB60F9211240F900FBE0F90A2
:10E680001F9018951F920F920FB60F92112410929F
:10E6900091360F900FBE0F901F9018951F920F92FA
:10E6A0000FB60F921124109291360F900FBE0F905B
:10E6B0001F9018951F920F920FB60F9211248F93EF
:10E6C00081E08093FD348F910F900FBE0F901F90CB
:10E6D00018951F920F920FB60F9211241092913637
:10E6E0000F900FBE0F901F9018951F920F920FB6AC
:10E6F0000F9211248F939F938091C3149091C4140F
:10E7000001969093C4148093C3149F918F910F909E
:10E710000FBE0F901F901895CF92DF92EF92FF924D
:10E720000F931F93CF93DF937C018B016A0185ECDC
:10E7300094E10E94F55BEC01009751F0EC81FD81C2
:10E74000309711F0C8010995CE010E949D5CF3CF6E
:10E75000A601B801C701DF91CF911F910F91FF90E2
:10E76000EF90DF90CF900C947F590F931F93CF932E
:10E77000DF9300D0CDB7DEB780919A3690919B366B
:10E78000A0919C36B0919D360196A11DB11D80933C
:10E790009A3690939B36A0939C36B0939D360E94F8
:10E7A0001F768C0185EC94E10E94F55B009779F06F
:10E7B000DC011296ED91FC911397309729F0898333
:10E7C0009A8309959A8189810E949D5CEFCF0115FA
:10E7D000110549F0C8010F900F90DF91CF911F9163
:10E7E0000F910C9476590F900F90DF91CF911F915C
:10E7F0000F9108950E94127B0E9467620E944674E6
:10E800008DE493E090939536809394360E941D7624
:10E810002FEF31E040E05EE160E074E082E090E004
:10E820000C94E675BC0185EC94E10C94555CBC013C
:10E8300085EC94E10C943A5CCF93DF93EC0140912A
:10E8400096365091973660919836709199364F5F11
:10E850005F4F6F4F7F4F409396365093973660933C
:10E860009836709399360E943276009761F00E9434
:10E87000E761E0915103F0915203BE018CE893E708
:10E88000099581E090E0DF91CF9108958BEC94E1C0
:10E890000C94F15B0F93CF93DF93EC017B836A833E
:10E8A00018865F834E83BC018BEC94E10E94555C1B
:10E8B000E091C714F091C814309749F04C815D8104
:10E8C00001E020E030E068858A819B810995DF9135
:10E8D000CF910F910895BC018BEC94E10C943A5CBC
:10E8E0000F93DC0118961C921897E091C714F091D1
:10E8F000C814309759F000E020E030E040E050E0EC
:10E9000060E012968D919C91139709950F9108954F
:10E910000F93DC01AB0114962D913C91159781E08A
:10E9200018968C93189715967C936E931497E09194
:10E93000C714F091C814309739F000E061E01296E6
:10E940008D919C91139709950F9108950F93DC0178
:10E95000E091C714F091C814309771F014964D915E
:10E960005C91159701E09A0118966C911897129690
:10E970008D919C91139709950F910895E091C91479
:10E98000F091CA14309709F0099408959093CA142D
:10E990008093C91408959093C8148093C714089560
:10E9A0008BEC94E10C94F55BEF92FF920F931F9325
:10E9B000CF93DF938C01EB017A018BEC94E10E9401
:10E9C000F55B0097D9F0DC0112962D913C911397DD
:10E9D0002C173D0781F41696ED91FC91179730970F
:10E9E00069F09701AE01B801DF91CF911F910F91AE
:10E9F000FF90EF9009940E949D5CE3CFDF91CF914F
:10EA00001F910F91FF90EF9008950895CF93DF939A
:10EA1000CEEFD4E16881798120E030E045E255E72E
:10EA200088EE94E10E94755E0E94107B6881798176
:10EA30000E94999220E030E049E355E7BC0188ED5F
:10EA400094E1DF91CF910C94755E8091FE149091CA
:10EA5000FF142091FC143091FD14880F991F281782
:10EA6000390708F4C9019093FF148093FE140C94A5
:10EA70000675CF93DF930E9467620E94CE61EC011E
:10EA8000198218820E94D07428813981009719F167
:10EA9000FC0140854423F9F0FC0142815381F901D6
:10EAA000EE0FFF1FEE0FFF1FEC0FFD1F538342837E
:10EAB000FC01448155812F5F3F4FF901EE0FFF1F8D
:10EAC000EE0FFF1FEC0FFD1F518340833983288316
:10EAD0000E949D5CD9CFC901880F991F880F991F8B
:10EAE00002960E94C96188819981892B31F08DEC51
:10EAF00094E1DF91CF910C944D59DF91CF9108951E
:10EB0000AF92BF92CF92DF92EF92FF920F931F933B
:10EB1000CF93DF9300D0CDB7DEB76B010E94CE61FB
:10EB2000FC01008111811A8309830C30110518F44E
:10EB3000E12CF12C0DC01F930F9388EF99E09F9368
:10EB40008F930E9478990F900F900F900F9021C093
:10EB5000E016F106F1F00E94CE61F701EE0FFF1F03
:10EB6000EE0FFF1FE80FF91FA280B3800E94CE6155
:10EB7000FFEFEF1AFF0AF701EE0FFF1FEE0FFF1F67
:10EB8000E80FF91F40815181B501C6010E94D4747C
:10EB9000DFCF0F900F90DF91CF911F910F91FF90DA
:10EBA000EF90DF90CF90BF90AF9008950F9301301A
:10EBB00059F48091F8149091F9149093FF14809374
:10EBC000FE140F910C9406750F910895EF92FF9229
:10EBD0000F931F93CF93DF938B01EA0179014AE3EF
:10EBE00053E0BC018DEC94E10E9431591093F9146B
:10EBF0000093F814D093FB14C093FA14F092FD1410
:10EC0000E092FC1486ED95E7DF91CF911F910F9173
:10EC1000FF90EF900C94CB7488EE94E10E94F95E23
:10EC200088ED94E10E94F95E8DEC94E10C944B59CF
:10EC30008091FE149091FF1408950C948B59CF93FA
:10EC4000DF93E0913E03F0913F030995EC010097BB
:10EC500029F06A817B8181E00E94E062CE01DF9130
:10EC6000CF9108950F931F93CF93DF93EC01E09121
:10EC70004003F091410309958C016A817B8181E019
:10EC80000E94E06281E090E0012B11F480E090E0CE
:10EC9000DF91CF911F910F910895E0914203F09180
:10ECA0004303099420E030E00296FC013297408152
:10ECB000442331F0FC0131974081240F311DF4CF02
:10ECC000C9010895FC01208130E0322F2227818183
:10ECD000282B02C0220F331F6A95E2F7832F992752
:10ECE000FA01EC5BFC4F208130E08223932328E083
:10ECF00030E0241B350B02C0969587952A95E2F7E4
:10ED000008956F927F928F929F92AF92BF92CF920F
:10ED1000DF92EF92FF920F931F93CF93DF938C01BB
:10ED2000EB016A0179012830310524F4A901B6010B
:10ED3000CE014AC0590123E0B594A7942A95E1F782
:10ED40004115510521F04801612C712C03C0D801F7
:10ED5000FB0120C048E050E0B601CE01860D971DB2
:10ED60000E946276F40181934F01FFEF6F1A7F0AD0
:10ED70006A147B047CF3C501B7FE02C080E090E01A
:10ED8000A701477055274115510511F1080F191FAB
:10ED9000B60118C0CF018C1B9D0B8A159B051CF476
:10EDA00081918D93F7CFC501B7FE02C080E090E05E
:10EDB000A701477055274115510551F0080F191F3C
:10EDC00060E070E08C0F9D1F0E946276F8018083E6
:10EDD000DF91CF911F910F91FF90EF90DF90CF9037
:10EDE000BF90AF909F908F907F906F9008958F927B
:10EDF0009F92AF92BF92CF92DF92EF92FF920F93CA
:10EE00001F93CF93DF9300D0CDB7DEB70E94CE61C2
:10EE10008C0182E090E00E94AC61892B19F480E0C3
:10EE200090E05DC0F801818190E0982F88272081D3
:10EE3000820F911D0E949C597C01009781F30E94D2
:10EE4000CE614C01F7012681822F869586958695A5
:10EE500090E0422F477021E030E011F420E030E0F4
:10EE6000820F931F0E94AC61892BC9F2F7010481C4
:10EE70001581C12CD12CF8018081882379F1F8010A
:10EE8000A180B12CB60133E0759567953A95E1F70D
:10EE9000A60147705527680D791D883168F09501E6
:10EEA000CE0101960E948176BE016F5F7F4FF8010F
:10EEB00080810E94F4620DC01A8219829501CE01F0
:10EEC00001960E94817669817A81F80180810E9491
:10EED000E062CA0CDB1C0E5F1F4FCDCFC7010F9045
:10EEE0000F90DF91CF911F910F91FF90EF90DF90E6
:10EEF000CF90BF90AF909F908F900895DC0150E02D
:10EF0000E0E1F0E0E61BF70BE21BF30B02C0440F5D
:10EF1000551FEA95E2F78C91852B8C9311968C9175
:10EF20001197842B11968C9308956F927F928F92F4
:10EF30009F92AF92BF92CF92DF92EF92FF920F9388
:10EF40001F93CF93DF938C016B01EA017901283085
:10EF500031051CF44881C8015CC0390153E0759447
:10EF600067945A95E1F76115710521F04E01A12CC6
:10EF7000B12C03C0D801FE0127C0F40141914F011B
:10EF800028E030E0B601C8018A0D9B1D0E947E7703
:10EF9000FFEFAF1ABF0AA614B7047CF3C30177FED4
:10EFA00002C080E090E097012770332721153105DA
:10EFB00009F43FC0C80FD91F488150E0B601621B59
:10EFC000730B685F7F4F1CC0CF018C1B9D0B861598
:10EFD00097051CF481918D93F7CFC30177FE02C092
:10EFE00080E090E09701277033272115310509F162
:10EFF000C80FD91F488150E068E070E0621B730BB6
:10F0000002C0559547956A95E2F760E070E0800F81
:10F01000911FDF91CF911F910F91FF90EF90DF90A3
:10F02000CF90BF90AF909F908F907F906F900C94F7
:10F030007E77DF91CF911F910F91FF90EF90DF903E
:10F04000CF90BF90AF909F908F907F906F900895DA
:10F050006F927F928F929F92AF92BF92CF92DF92E8
:10F06000EF92FF920F931F93CF93DF9300D0CDB712
:10F07000DEB78C01FC018681E82EE694E694E694E6
:10F08000F12C282F277081E090E011F480E090E0CF
:10F09000E80EF91EC70102960E943062009709F43B
:10F0A00045C00E94D561F8012281FC012083F8014E
:10F0B0002381FC0121830E94D56102965C01A70196
:10F0C00060E070E00E94CC98F80104811581E12C89
:10F0D000F12CF8018081882339F1F8018180912C8D
:10F0E000670163E0D594C7946A95E1F73701F7E0CB
:10F0F0006F227724CA0CDB1C883128F00E94FE6244
:10F100009401AC0108C00E94EB629A838983940148
:10F11000AE014F5F5F4FB301C6010E949577E80CC7
:10F12000F91C0E5F1F4FD5CF81E090E00F900F903C
:10F13000DF91CF911F910F91FF90EF90DF90CF90D3
:10F14000BF90AF909F908F907F906F900895E091C7
:10F150005F03F09160030994E0913803F091390363
:10F160000994E0916303F09164030994E0916503CD
:10F17000F0916603099480E090E008950895E0918D
:10F180003003F0913103099480E090E008950F93EB
:10F190001F93CF93DF93CDB7DEB7E0970FB6F89408
:10F1A000DEBF0FBECDBF0E941B628C010E94CE61EC
:10F1B000AE014F5F5F4F602F0E949780882309F454
:10F1C00046C088A99801281B3109C9010E94AC6179
:10F1D000892BE9F12E8121110CC0BE016A5E7F4F9F
:10F1E00088E10E94F462E0915303F0915403099581
:10F1F0002EC08A859B858D3C3BEA930711F00196D2
:10F2000031F5223019F088E090E002C082E090E011
:10F2100001979C012F5F3F4F12161306F4F6E1E0B1
:10F22000F0E0EC0FFD1FE80FF91F23852F3F81F35E
:10F23000BE01645F7F4F89E10E94F46289E10E9410
:10F24000FE6263EA74E30E94EA58892B31F6E09685
:10F250000FB6F894DEBF0FBECDBFDF91CF911F91E7
:10F260000F910895AF92BF92CF92DF92EF92FF92EB
:10F270000F931F93CF93DF93CDB7DEB7E0970FB611
:10F28000F894DEBF0FBECDBF8C016B01CE0101969D
:10F290007C0180E3F70111928A95E9F781E0898387
:10F2A0008CE00E94EB628C831D821F82809102158C
:10F2B00091E0980F90930215898783E0B82EB88665
:10F2C0008DEC9BEA9B878A8789E10E94FE626CE055
:10F2D00073E00E94EA58892B31F082E08E838FEF31
:10F2E0008C878D8709C089E10E94FE62BC01CE0136
:10F2F0000C960E94E158BE828DEC9BEA9D8B8C8B14
:10F3000063EA74E3CE0146960E94E1580E94CE6102
:10F310009FA78EA70E941B6288ABC7010E94907FA7
:10F32000B82E90E00E943062892B31F10E94D561A5
:10F33000BC014B2DC7010E94AE7FE0902603F090E8
:10F3400027030E9425625C010E94D561B501F70187
:10F3500009950115110581F0009739F0019761F4C5
:10F3600041E050E064E070E004C041E050E060E063
:10F3700070E0C601F8010995E0960FB6F894DEBF7B
:10F380000FBECDBFDF91CF911F910F91FF90EF90F6
:10F39000DF90CF90BF90AF9008950E94107B809334
:10F3A0000215E0913003F09131030994892B29F083
:10F3B000E0913003F091310304C0E0913203F09109
:10F3C00033030994CF93DF93EC01899199910097CE
:10F3D00029F060E070E00E94355BF7CFDF91CF91BC
:10F3E0000895CF93DF93EC0189919991009719F0DB
:10F3F0000E94875AF9CFDF91CF910895CF93DF9381
:10F40000EC017B836A830E94A96B99838883DF91D7
:10F41000CF910895FC018081918122813381820FF7
:10F42000931F918380830895CF93DF93EC010E9413
:10F43000A96B99838883DF91CF910895CF93DF9350
:10F44000EC010E94A96B28813981821B930B9C01DE
:10F450002F5F3F4F81E090E04A815B814217530765
:10F4600010F080E090E0DF91CF910895CF93DF938B
:10F47000FC01C281D38180819181C80FD91F0E9474
:10F48000A96B9E01281B390BC901DF91CF9108950B
:10F49000CF93DF93ECE1F7E3CEEDD6E3A0E1B7E362
:10F4A0001192119219921992199219921D9287E351
:10F4B000E433F807A9F7DF91CF910895CF93DF9355
:10F4C000FC01E05FF84C40819C01220F331F220FAA
:10F4D000331F442301F1A0919400B0919500FC01E9
:10F4E000EE0FFF1FE45EF84C80819181AD01481B57
:10F4F000590BCA01E901C252D94C488159816A812C
:10F500007B81480F591F611D711D488359836A8390
:10F510007B83B183A083F901E252F94C6081718150
:10F5200082819381DF91CF91089560E070E0CB01FB
:10F530000895FC01EE0FFF1FEE0FFF1FE252F94C82
:10F5400040835183628373830895CF93DF9320E1D7
:10F5500037E3CEEDD6E3ECE1F7E3D9018D919D01E0
:10F560008823B9F040919400509195008081918159
:10F57000BA01681B790B88819981AA81BB81860FAA
:10F58000971FA11DB11D88839983AA83BB835183D3
:10F59000408324963296B7E32C313B07F1F6DF9196
:10F5A000CF9108950C941F7F0F931F93FC01CB0103
:10F5B00040910315509104153383228315830483EE
:10F5C00071836083F0930415E0930315452B11F4C8
:10F5D0000E94397F80E090E01F910F910895809103
:10F5E0000315909104150097C1F010920415109224
:10F5F0000315DC0114966D917C9115971296ED918F
:10F60000FC9113970995E0910315F091041530973B
:10F6100021F0808191810C94397F08950C94569546
:10F620000C9452958EED92E00E946C5B86ED92E018
:10F630000C946C5BCF93DF930E94DB61892BA9F064
:10F6400086ED92E00E948A5BEC01009721F10E9416
:10F650001B62998388830E9416629B838A83CE01F2
:10F6600004960E9457618CAB14C08EED92E00E940C
:10F670008A5BEC01009779F002960E946961998398
:10F680008883BE016E547F4FCE018E579F4F0E94DC
:10F69000BE62CE0102C080E090E0DF91CF9108957C
:10F6A000BC016E547F4F8E579F4F0C94BE62CF9318
:10F6B000DF93EC01BC018EED92E00E94D45BBE01B1
:10F6C000892B19F08EED92E009C086ED92E00E9440
:10F6D000D45B892B39F0BE0186ED92E0DF91CF91AA
:10F6E0000C94AF5BDF91CF9108950F931F93CF934D
:10F6F000DF93EC01BC018EED92E00E94D45B892B7C
:10F7000091F0FE0161917191CF010E947A62BE0178
:10F710006E547F4FCE018E579F4FDF91CF911F9137
:10F720000F910C94CF62BE0186ED92E00E94D45BF3
:10F73000892BD1F00E946762688179818A819B81DF
:10F740000E947A628CA990E00E9430620CA910E0BD
:10F750000E94D561BE016C5F7F4FA801DF91CF9100
:10F760001F910F910C94C398DF91CF911F910F912E
:10F770000895CF93DF93EC01BC018EED92E00E94DF
:10F78000D45B892B19F0CE0102960CC0BE0186ED28
:10F7900092E00E94D45B892B19F08A819B8102C080
:10F7A00080E090E0DF91CF910895FC01808191810C
:10F7B0000895860F911D860F911D8E579F4F0895B6
:10F7C000860F911D860F911D8E579F4FFC018081E2
:10F7D00091810895089582E69BE10E94AE5D892B98
:10F7E00021F082E69BE10C949B5D0895E0914E1B15
:10F7F000F0914F1B309709F0099480E00895EF9243
:10F80000FF920F931F93CF93DF937C01EA01FC01DA
:10F8100080819181009741F08C30934071F1F70124
:10F820001182108283E0F2C080E024E0829FF00128
:10F830001124E05BF44E118210828F5F8430A8F3B4
:10F8400080934D1B80918812909189129093611B37
:10F850008093601B0E94805A8093343760E470E08C
:10F8600082E69BE10E94875D0E940C828CE093E01F
:10F87000F7019183808381E0C9C06230D9F480911F
:10F88000353790913637892B89F38091463786300A
:10F8900029F480915E3781FD0E94EB7B81E00E941C
:10F8A00049838091353790913637892BF9F20E9440
:10F8B0000F7EDCCF633060F5611114C02097B1F288
:10F8C000D093433CC093423C83E00E9449838091A3
:10F8D000353790913637892B11F00E94F67B0E94C4
:10F8E000EB7BC4CF613011F6209709F4BFCFD093E2
:10F8F0003F3CC0933E3C85E00E9449838091353770
:10F9000090913637892B09F4B1CF0E94F67BAECFA8
:10F910006738E9F510924C1B00E51BE180914C1B08
:10F920008430B8F4F801828193818C179D0749F4E3
:10F93000808191810E941683F801118210821382C6
:10F9400012820C5F1F4F80914C1B8F5F80934C1B6A
:10F95000E5CFEDE5FCE3838194818C179D0719F4D5
:10F96000148213821082B0962CE3ED3DF20799F7D2
:10F97000EAEDFCE3818592858C179D0711F41582D1
:10F9800014823D968DE3EC35F807A1F76FCF683808
:10F9900009F06CCFC256DB4109F068CF82E69BE1EB
:10F9A0000E94AE5D892B09F461CF10924C1BE0914F
:10F9B0004C1BE43008F05ACF20E2E29FF001112402
:10F9C000EC5BF34C818D8823D9F082E69BE10E94A9
:10F9D0009B5D80914C1BE0E28E9FC00111248C5BEB
:10F9E000934C9093433C8093423C82E00E94498335
:10F9F0008091353790913637892B11F00E94F67B34
:10FA000080914C1B8F5F80934C1BD1CFDF91CF91A6
:10FA10001F910F91FF90EF90089590934F1B80934B
:10FA20004E1B0895209188123091891260E0E0E524
:10FA3000FBE1643098F4408151814817590759F42B
:10FA4000428153814217530731F460934B1B11825B
:10FA500010820C94168334966F5FEBCF60934B1B30
:10FA6000089540E0E0E5FBE14430A8F451E0540F94
:10FA700020813181232B61F440934A1B9183808341
:10FA80002091881230918912338322830C94308321
:10FA90003496452FE9CF40934A1B08952091881250
:10FAA00030918912FC01358F248F778F668F0895EE
:10FAB0002091881230918912FC0132872187748746
:10FAC00063870895CF93DF93EA010E94B98200977C
:10FAD00049F02091881230918912FC0132872187E8
:10FAE000D487C387DF91CF9108950F931F93CF934E
:10FAF000DF9300D000D0CDB7DEB78C01AB018FEF24
:10FB000089838A838B838C83B801CE0101960E94FE
:10FB1000627D009719F0FC01158304830F900F900C
:10FB20000F900F90DF91CF911F910F91089540E0BA
:10FB300050E062E086EE92E00E94265B109236373B
:10FB4000109235370895AC0161E086EE92E00C9496
:10FB5000085BAC0160E086EE92E00C94085B0F93CA
:10FB60001F93CF93DF938A010E943882EC010097A4
:10FB700059F080918812909189129D8F8C8F1F8FE0
:10FB80000E8FCE010E94A97DCE01DF91CF911F91F2
:10FB90000F910895CF93DF93A091423CB091433CE5
:10FBA000109719F0ED016C9605C0C0913E3CD091C4
:10FBB0003F3C299680913D3C86FF22C01092491B14
:10FBC00040E0E0E5FBE14430B8F420813181149657
:10FBD0008D919C9115972817390759F4828193814B
:10FBE000009739F04093491B998388831B821A82BE
:10FBF00005C034964F5FE7CF4093491B0E94EB7BD3
:10FC000088819981009741F04A815B816091343706
:10FC1000DF91CF910C94265BDF91CF9108950F93E4
:10FC20001F93CF93DF9380914637863009F071C0E0
:10FC300080913537909136378115954009F069C02C
:10FC4000C4E9D2E0D0933637C093353702E0009351
:10FC50003F3714E9109340371092623710926137A2
:10FC60000E940682809590959093623780936137C9
:10FC700010924837109247370E94F58180959095F1
:10FC800090934837809347370E94F67BD09336375E
:10FC9000C093353700933F3710934037A091403CD5
:10FCA000B091413CFD01E459FD4F8CE692E001909A
:10FCB0000D920197E1F76CE672E085E597E30E940B
:10FCC000B481809139378093553780913A3780934A
:10FCD000563780913B378093573780913C378093DC
:10FCE000583710926237109261370E9406828095D1
:10FCF00090959093623780936137109248371092B5
:10FD000047370E94F581809590959093483780936E
:10FD10004737DF91CF911F910F910C94F67BFC0137
:10FD2000680F791F80E048E1E617F70781F021911D
:10FD300098E0322F3827532F517030FD8427869555
:10FD4000513009F480682695915099F7EDCF0895C8
:10FD50001F920F920FB60F9211240BB60F922F9392
:10FD60003F934F935F936F937F938F939F93AF9343
:10FD7000BF93EF93FF93809194009091950090939F
:10FD800021378093203781E0809312378091710072
:10FD9000807D809371000E94EF7A809112378823D2
:10FDA000D9F1809194009091950040912037509125
:10FDB000213784179507A0F48091E6369091E736B5
:10FDC000A091E836B091E9368C57914EAF4FBF4FB6
:10FDD0008093E6369093E736A093E836B093E93601
:10FDE0002091940030919500241B350B8091E636CC
:10FDF0009091E736A091E836B091E936820F931FD3
:10FE0000A11DB11D8093E6369093E736A093E836A6
:10FE1000B093E93610921237FF91EF91BF91AF91F5
:10FE20009F918F917F916F915F914F913F912F9112
:10FE30000F900BBE0F900FBE0F901F9018959FB79D
:10FE4000F894E1E7F0E08081807D808388B38F6261
:10FE500088BB10929000E1E9F0E0108210929200CD
:10FE600010929500109294008081856080839FBFDE
:10FE700008952FB7F894909399008093980088B3D1
:10FE80008F6288BBE1E7F0E08081826080832FBFD2
:10FE90000895CF93DF93FC01DB0185E0EB0119921C
:10FEA0008A95E9F78581837011F082E08C938781D0
:10FEB000837021F082E012968C9312978581837073
:10FEC00081F08781837069F02389348981859285E7
:10FED0002817390731F481E0848312961C92129717
:10FEE00001C0148285818370823021F0833021F03B
:10FEF00080E003C082E001C088E011968C931197E6
:10FF000087818370823021F0833021F080E003C04C
:10FF100082E001C088E013968C93DF91CF91089521
:10FF2000CF93DF9300D000D01F92CDB7DEB7BE01D4
:10FF30006F5F7F4F0E94497F89819A81890F8D5F12
:10FF40009B81890F9C81890F9D81890F0F900F9054
:10FF50000F900F900F90DF91CF9108954F925F9285
:10FF60006F927F928F929F92AF92BF92CF92DF92C9
:10FF7000EF92FF920F931F93CF93DF9300D000D0A7
:10FF800000D0CDB7DEB78C017B01BE016F5F7F4F24
:10FF90004E830E94497FB981AA815B804C808B2F60
:10FFA00090E003962A2F30E0820F931F850D911D5C
:10FFB000642D70E0860F971F5D81850F911D4E8126
:10FFC00050E0481759070CF49AC0F801818180FB72
:10FFD000662460F8712C43E0660C771C4A95E1F7C3
:10FFE000828180FB882480F8912C54E0880C991C35
:10FFF0005A95E1F7862880818770882A838180FB63
:020000021000EC
:10000000AA24A0F8B12C85E0AA0CBB1C8A95E1F7C4
:100010008A28848180FBCC24C0F8D12C96E0CC0CBB
:10002000DD1C9A95E1F78C28F7018082F801458163
:100030004370F4E04F9FA0011124F8018681837082
:10004000F0E18F9FC0011124482BF8018781F0E473
:100050008F9FC0011124482BF7014183F80180854F
:10006000F7018283B23059F4F8018185F701838367
:10007000F8018285F701848395E0C92E02C083E0F0
:10008000C82EB0E080E090E0200F311FDB2EDC0CAA
:100090000197BA1761F0A901480F591FFA01B384FB
:1000A000A7014D0D511DFA01B082BF5FEFCF9D2D0D
:1000B000F2E05F120EC0D701AD0DB11DF8018389CA
:1000C0008C9381E08D0DD701A80FB11D9E5F8489AF
:1000D0008C9340E020E030E0060F171F842F890F3B
:1000E00021503109441561F0D801A20FB31F559674
:1000F0005C91D701A80FB11D5C934F5FEFCF80E0FB
:1001000026960FB6F894DEBF0FBECDBFDF91CF911C
:100110001F910F91FF90EF90DF90CF90BF90AF9025
:100120009F908F907F906F905F904F900895BF92B7
:10013000CF92DF92EF92FF920F931F93CF93DF93B3
:100140007C01D62EEA0182E0861708F0B1C0F701E3
:10015000808186FBBB24B0F89181292F26952695B6
:100160002370C92EC294C694C69453E0C522382F7A
:100170003770388383FB332730F9398384FB332787
:1001800030F93A8385FB882780F98B83BC822D83E5
:10019000892F829583708E83CF82828188872223E4
:1001A00089F13381848190E0982F8827830F911DF6
:1001B0009A87898787010B5F1F4F223071F46CE0AB
:1001C00073E0CE010B960E94E158F70186818B8780
:1001D00085818C870E5F1F4F20C02330F1F4F7011B
:1001E0003D9680E090E03E2F2F2F4291DE01A80F38
:1001F000B91F1B964C93019688309105B1F7032FD8
:10020000122F0BC087010D5F1F4F6CE073E0CE0112
:100210000B960E94E1581A861986CC20B9F1B110CC
:100220000DC0F8012081818190E0982F8827820FEE
:10023000911D9C8B8B8B0E5F1F4F04C089859A8507
:100240009C8B8B8BF2E0CF120EC06CE073E0CE0182
:1002500045960E94E158F80181818D8B80818E8BBB
:100260000E5F1F4F1BC0F3E0CF1218C0085F1F4F77
:10027000F80180E090E02291DE01A80FB91F5596A9
:100280002C93019688309105B1F708C06CE073E0BB
:10029000CE0145960E94E1581C8A1B8AC8018E191E
:1002A0009F092D2D281B2FA71EA70DA7D81608F4D0
:1002B00080E0DF91CF911F910F91FF90EF90DF9041
:1002C000CF90BF900895FB0141505109460F571F31
:1002D000E417F50778F4208130E0322F222761817E
:1002E000260F311D820F931F8217930708F4019682
:1002F0003296EECFE417F50751F4208130E0322F2B
:100300002227820F931F8217930708F401960895FE
:10031000CF93DF93C0914037D0E0649720913F376F
:1003200030E0322F2227C20FD31F48E050E069E4AB
:1003300077E39E01280F311DC9010E946381AE0140
:1003400061E577E30E946381009721F09827892770
:10035000982702C08FEF9FEFDF91CF910895909380
:100360007B1B80937A1B0895FC015381560F509399
:100370003C37872F99274281480F40933B37A18113
:10038000A0933A37E081E0933937242F30E02817E3
:10039000390748F481E08A0F80933A37811103C00E
:1003A000EF5FE0933937852F90E07727861797071F
:1003B00088F44F5F40933B3741110CC080913A372E
:1003C0008F5F80933A37811105C0809139378F5FF5
:1003D000809339370895AB01BC0180E090E00E9422
:1003E0006381982789279827089544E150E06DE3B9
:1003F00077E380E090E00E946381009721F09827E6
:100400008927982708958FEF9FEF089586E00C9431
:10041000888181E10C94888180E0E82FF0E0EE0F84
:10042000FF1FEC53F34C118210828F5F8430A8F3CE
:1004300080E090E2899FF0011124EC5BF34C118E77
:100440008F5F8430B0F380E094E09093751B8093CD
:10045000741B80E09DE0989FF0011124E652F34C5C
:10046000158214828F5F8A30B0F38093731B0895D6
:10047000CF932091741B3091751B2F5F3F4F211537
:100480004DE7340710F020E030E1522F432FE4E431
:10049000FCE3C0E0C43059F0A18DAA2329F0A48167
:1004A000B581A417B50749F3CF5FB096F3CF30936A
:1004B000751B2093741B1092731B20E0E0E0F0E0AA
:1004C0002430E8F430E2239FD0011124AC5BB34C1C
:1004D00059963C915997311104C02093731BFD012B
:1004E00010C0373041F4309739F05A964C915A97F2
:1004F000328D341708F0DF012F5FFD01E1CF20932B
:10050000731B309799F122E0218F2091761B24876D
:100510002091771B25872091781B26872091791BB6
:10052000278728ED34E0338B228B358B248B21E019
:1005300030E0318B208B138E228F23E0208F168AA0
:1005400020E1278B2091741B3091751B32272327C4
:1005500032273583248377836683DC014D915D9157
:100560006D917C914083518362837383CF01CF91DE
:100570000895CF93DF932091741B3091751B2F5FEB
:100580003F4F21154DE7340710F020E030E1522FA6
:10059000432FEEEDFCE3C0E0CA3041F0A081B18111
:1005A000CF5F3D96A417B507B9F7E9CF3093751B18
:1005B0002093741B40E05DE04A30A0F4A1E0A40F5A
:1005C000549FF0011124E652F34C24813581232BF2
:1005D00039F44093731B309741F480E090E023C0DE
:1005E0004A2FEACF4093731BF8CF2091741B3091B0
:1005F000751B32272327322735832483778366832D
:10060000009729F4108211821282138209C0EC0132
:1006100088819981AA81BB8180839183A283B383DE
:1006200080E48087CF01DF91CF91089540E044308E
:10063000A0F4E42FF0E051E0540FEE0FFF1FEC5355
:10064000F34C208131812817390729F44093731B1B
:10065000118210820895452FEACF4093731B0895AD
:1006600040E0443098F4E42FF0E051E0540FEE0FF6
:10067000FF1FEC53F34C20813181232B29F440934D
:10068000731B918380830895452FEBCF4093731B99
:100690000895AF92BF92CF92DF92EF92FF920F93A5
:1006A0001F93CF93DF93C091423CD091433C843061
:1006B00009F4DCC125E637E33093413C2093403C0C
:1006C0003093383720933737833059F4898D8F70C2
:1006D000833009F06BC088899989892B09F0DFC6BE
:1006E0007FC0823009F080C08091791B8F5F80933A
:1006F000791B811113C08091781B8F5F8093781BC9
:1007000081110CC08091771B8F5F8093771B8111C3
:1007100005C08091761B8F5F8093761B10923637D1
:10072000109235371092D93C1092D83C298D822FE7
:100730008D7F853041F48A8D8F5F8A8F843109F0F7
:10074000AEC6198EACC6222309F4A9C68889998938
:10075000892B09F441C08A8D9FEF980F9A8F8111E0
:100760009EC68B8D883031F09FEF920F923048F407
:10077000853039F4198E80E880933D3C0E94CA7D13
:1007800047C5853038F493E0082E01C0990F0A94CC
:10079000EAF701C090E39A8F8F5F8B8F822F8F7063
:1007A0008330A1F048F4813009F44FC3823009F05E
:1007B00076C610925E374CC3863009F4C8C48830C0
:1007C00009F4C5C4843009F06AC6C1C484E08093CA
:1007D0003D3C0E94CA7D4EC52F70233009F05FC694
:1007E00088E080933D3C09C5853019F5E0913E3C99
:1007F000F0913F3C84819581892B09F450C6109279
:10080000433C1092423C89E597E39093413C8093AE
:10081000403C90933837809337371092D93C1092F0
:10082000D83C109236371092353788E080933D3CA3
:100830001BC180913D37853409F031C600913F37A7
:1008400010E0102F002780914037080F111D809174
:100850003537909136378017910708F420C61093EA
:10086000363700933537809143378F7309F017C6B9
:1008700080914437811113C68091D43C9091D53C2E
:10088000C0916903D0916A038C179D0759F4409178
:10089000D63C5091D73C20916B0330916C034217AA
:1008A0005307A1F020914D3730914E372817390763
:1008B00009F0F5C520914F37309150378091D63CE3
:1008C0009091D73C2817390709F0E9C50E94F581B6
:1008D000019609F0E4C580914637863009F429C1B4
:1008E0008131E9F1813009F0DAC5809151378830E2
:1008F00009F0D5C5109251378091533790915437F4
:10090000873F3FEF930710F0099601C00896909338
:100910005437809353378091493790914A37A0914B
:100920004B37B0914C3780934D3790934E37A0930F
:100930004F37B09350378091D43C9091D53CA091E3
:10094000D63CB091D73C8093493790934A37A093D7
:100950004B37B0934C3780E4809345377DC50C51BD
:100960001109109336370093353789E597E3909353
:10097000413C8093403C8091573790915837892B68
:1009800029F00E940982019609F089C52091533708
:10099000309154372115310509F481C58AED9CE366
:1009A00090933F3C80933E3CA0905137B09052379B
:1009B00040916B0350916C0360916D0370916E03D5
:1009C000A0916F03B09170030091493710914A379D
:1009D000E0904B37F0904C37E0913E3CF0913F3C3B
:1009E0008DE3EC35F80708F05AC5848195810097AE
:1009F00021F12817390709F586819781009719F0A9
:100A0000A816B906D1F4808191818C179D0729F42D
:100A1000C280D380C416D506B1F08617970729F493
:100A2000C280D380CA16DB0671F00817190729F4B3
:100A300082819381E816F90631F03D96F0933F3CB0
:100A4000E0933E3CC9CF1092433C1092423C82E07E
:100A500080933D3C89E597E390933837809337370F
:100A60001092D93C1092D83C0E94CA7D8091D83C0B
:100A70009091D93C009709F412C59C01245E3F4F28
:100A8000309336372093353730933F3720934037B4
:100A9000E0913E3CF0913F3C20852093453721E199
:100AA000209346370896982789279827909356379A
:100AB000809355371092583710925737848195811B
:100AC0009093523780935137868197819093543712
:100AD000809353378091D43C9091D53CA091D63CE3
:100AE000B091D73C8093493790934A37A0934B37C6
:100AF000B0934C3780819181A281B38180934D372F
:100B000090934E37A0934F37B093503785E697E3D5
:100B10009093413C8093403C0E940982809590953F
:100B2000009711F48FEF9FEF9093583780935737CA
:100B300093C40E940682019609F0B1C48091533794
:100B400090915437009709F4AAC4209151373091FD
:100B500052372115310509F4A2C44091493750910B
:100B60004A3760914B3770914C37EDE5FCE3C4E4B4
:100B7000DCE3F080FF20A9F0AC81BD818A179B07E0
:100B800081F4AE81BF812A173B0759F4A881B9814E
:100B90004A175B0731F4AA81BB816A177B0709F406
:100BA0006FC1A096B096ACE3C43CDA0711F7209170
:100BB0005E372F732230D9F49093711B8093701B92
:100BC00040E0443090F4E42FF0E0EE0FFF1FEC53D0
:100BD000F34C208131814F5F8217930791F7109278
:100BE000731B20E0C0E0D0E07EC04093731B809177
:100BF0005E3782FD54C484E180935E3788E290E0E2
:100C0000909336378093353780E580935D378091B8
:100C1000583790915C37909358373091573790916F
:100C20005B379093573730935B37209156379091CD
:100C30005A379093563720935A379091553790935F
:100C4000731B4091593740935537909359378F5FB5
:100C500080935C3781110FC081E0830F80935B37F5
:100C6000811109C081E0820F80935A37811103C03E
:100C70009F5F90935937809151379091523790935D
:100C8000711B8093701B20915337309154373093F0
:100C90005237209351379093543780935337809134
:100CA000493790914A37A0914B37B0914C37809398
:100CB0004D3790934E37A0934F37B0935037809174
:100CC000D43C9091D53CA091D63CB091D73C809338
:100CD000493790934A37A0934B37B0934C37A1C311
:100CE000373089F02F5F2430C0F430E2239FC001F9
:100CF0001124FC01EC5BF34C318D3111F1CF2093C9
:100D0000731BEF010CC0209721F0428D3A8D3417F0
:100D100048F7EC01CC5BD34CE5CF2093731B2097B5
:100D200009F4BDC3D093433CC093423C83E08A8F17
:100D3000888F1E8A84E08F8B1B8E80915337909111
:100D400054379D838C8380915137909152379F8384
:100D50008E838091493790914A37A0914B37B0915B
:100D60004C3788839983AA83BB8381E0898F8091E4
:100D7000761B8C878091771B8D878091781B8E875F
:100D80008091791B8F8781E090E0998B888B80918F
:100D900058378B87809157378A8780915637898754
:100DA00080915537888781E090E00E94B38A8091D6
:100DB0005D37282F207F30E0213531050CF445C008
:100DC00082958F7090E00597880F991F880F991F63
:100DD0003091721B20E0E22FF0E0E817F9078CF564
:100DE000E35CF84C30A5311105C02093731B1092C1
:100DF000721B2BC0313011F42F5FEDCF3230E1F494
:100E000041A54430C9F42093731B3093721B82A513
:100E100090E0982F882723A5822B9093711B8093B5
:100E2000701B893DA4E09A0710F088ED94E09B8B3D
:100E30008A8B9D8B8C8B09C041A5442311F0240F14
:100E4000CACF2093731B3093721B80E180935E376F
:100E500080915E37826080935E3782E08093653751
:100E600084E0809366378093673788ED8093683796
:100E70008CE290E0909336378093353780E67EC2DF
:100E8000D093433CC093423C10923D3C90915E37DE
:100E900092FF03C0198E80E21AC280915D3782955D
:100EA0008F70880F880F8093731B081B11090451E2
:100EB000110910933637009335378F2D8F7082309C
:100EC00029F4892F8F73823139F41FC0813021F4C6
:100ED000892F8F738230C9F0012B19F4892F837009
:100EE000A1F020915537888528133EC220915637AE
:100EF0008985281339C2209157378A85281334C22F
:100F0000209158378B8528132FC294FF4AC06889D7
:100F100079896115710509F444C0CE010C960E94CF
:100F2000B481309159378091393738133AC02091C4
:100F30005A3780913A37281334C090915B378091AB
:100F40003B3798132EC080915C3740913C37841317
:100F500028C03C872D879E878F878B8D81111AC073
:100F60002E89888D9A8D891B922F969596959695A8
:100F7000891B280F2E8B87FD81959F89392F3695E8
:100F80003695931B980F9F8B822F86958695869515
:100F9000890F888F81E080933D3C888D8A8F198AE4
:100FA000188A498D842F8F7090E0FC013197E830CA
:100FB000F10508F074C2E057FF4F0C940293809142
:100FC0003D3C80FF14C083E0898F80E480933D3CEA
:100FD000198A188A8091353790913637009709F42D
:100FE00008C122E420933D3C0E94B38A02C1809153
:100FF0005E378F73823009F052C227CF80913D3C1B
:1010000080FF70C080915E378F73823109F06AC0B3
:1010100080915D37282F207F30E0213531050CF499
:1010200045C082958F7090E00597880F991F880FB3
:10103000991F3091721B20E0E22FF0E0E817F907CA
:101040008CF5E35CF84C30A5311105C02093731B7F
:101050001092721B2BC0313011F42F5FEDCF323064
:10106000E1F441A54430C9F42093731B3093721B03
:1010700082A590E0982F882723A5822B9093711B3F
:101080008093701B893D24E0920710F088ED94E076
:101090009B8B8A8B9D8B8C8B09C041A5442311F0BF
:1010A000240FCACF2093731B3093721B83E0898F68
:1010B0008091553788878091563789878091573737
:1010C0008A87809158378B8781E090E00E94B38AAD
:1010D00082E480933D3C198A188A10923637109228
:1010E000353787C080E280933D3C0E94CA7DE09105
:1010F000423CF091433C118E7ACD80915E3780FF67
:1011000028C044FD26C088899989892B09F0C7C168
:10111000809135379091363701960E94B38A20919D
:101120003D3C822F806180933D3C8091353790918A
:101130003637892B19F0226120933D3C0E94CA7DED
:1011400081E090E0998B888B88E0898F1B8E81E10C
:101150000CC185FF1CC08091633790E0982F8827D1
:1011600020916437822B2091403C3091413C280FE4
:10117000391F3093413C2093403C209135373091CA
:101180003637281B390B309336372093353780910B
:10119000353790913637009749F044FD07C02091CC
:1011A0003D3C226020933D3C0E94B38A80915F3792
:1011B00090E0982F882720916037820F911D90939F
:1011C000711B8093701B2C893D892817390710F0FB
:1011D000892B21F43093711B2093701B8091701B1D
:1011E0009091711B9B8B8A8B80913D3C837009F49D
:1011F00056C11092D93C1092D83C0E94CA7D809171
:101200003D3C85FF07C01092D93C1092D83C198E06
:1012100084E1ABC084FF0AC01092D93C1092D83C44
:1012200081E090E0998B888B84E08FCF2091D83C2F
:101230003091D93C21153105E1F080FF02C0198AB7
:10124000188A88899989009781F48A899B898217ED
:10125000930720F49093D93C8093D83C8091D83C5C
:101260009091D93C998B888B04C09093D93C809302
:10127000D83C1B8E80913737909138379093413C02
:101280008093403C8091D83C9091D93C892B59F077
:1012900088899989009739F088969093363780939A
:1012A000353788E10BC080913D3C81FFF8C088E272
:1012B00090E0909336378093353780E180935E37A6
:1012C0005CC080913D3C80FFEAC0198E80E1809334
:1012D0003D3C0E94CA7DE3C08091353790913637FE
:1012E000009711F00E94B38A90915E3780913D3C47
:1012F00090FF0BC080FF06C087E0898F1A8E198A85
:10130000188A19C086E0898F16C080FF1EC085E04C
:10131000898F198A188AC3C08091353790913637E2
:10132000009711F00E94B38A80915E3780FF0DC054
:1013300087E0898F1A8E81E090E00E94B38A80E175
:1013400080933D3C0E94CA7D0FC0809135379091BB
:101350003637892B49F4A3C080913D3C80FF9FC064
:1013600087E0898F1A8E9BC080E180935E3788E288
:1013700090E0909336378093353780E580935D37E2
:10138000888580935937898580935A378A858093D9
:101390005B378B8580935C378C85809355378D8543
:1013A000809356378E85809357378F858093583733
:1013B00086E0809346378C819D819093523780934D
:1013C00051378E819F81909354378093533780910A
:1013D000D43C9091D53CA091D63CB091D73C809321
:1013E000493790934A37A0934B37B0934C37888155
:1013F0009981AA81BB8180934D3790934E37A093FA
:101400004F37B0935037898D84FF05C010926037F5
:1014100010925F3706C084E080935F3788ED809339
:10142000603780E480934537809135379091363727
:1014300090933F3780934037109264371092633710
:1014400010926237109261370E94068280959095C3
:10145000909362378093613785E480933D37109293
:101460003E37109244371092433780917A1B909107
:101470007B1B019690937B1B80937A1B9093413743
:101480008093423710924837109247370E94F58177
:1014900080959095909348378093473704C0109279
:1014A00036371092353710923D3CDF91CF911F9126
:1014B0000F91FF90EF90DF90CF90BF90AF90089585
:1014C00098278927982708950E9408930895FC017A
:1014D00080913737909138372DE33CE3281B390B47
:1014E000AB01261737070CF4A9011416150654F49E
:1014F0005093D93C4093D83CE817F90719F0BF0145
:101500000C94C398089580E8809361001092610064
:101510000E943D690E949D5A0E941B6D8091E43497
:101520009091E534009729F001979093E5348093EA
:10153000E434C090E634D090E734E090E834F090A2
:10154000E9340E94D76BC616D706E806F90611F3F0
:101550000E94D76B6093E6347093E7348093E8344D
:101560009093E934D7CF2091423C3091433CBC0169
:10157000C90108960E94B481E091423CF091433C3D
:1015800080913937808780913A37818780913B37C6
:10159000828780913C37838708952F923F924F92A4
:1015A0005F926F927F928F929F92AF92BF92CF92F3
:1015B000DF92EF92FF920F931F93CF93DF93CDB7FC
:1015C000DEB763970FB6F894DEBF0FBECDBF7C01C8
:1015D0001B016A01FC0117821682838181FF66C3A9
:1015E000BE016F5F7F4F4B01F7019381F10193FDC6
:1015F000859193FF81911F01882309F453C385329C
:1016000039F493FD859193FF81911F01853239F45F
:10161000B70190E00E94469956016501E5CF10E0C0
:10162000512C20E02032A0F48B3269F030F480326B
:1016300059F0833269F420612CC08D3239F0803347
:1016400039F4216026C02260246023C0286021C0B4
:1016500027FD27C030ED380F3A3078F426FF06C05A
:10166000FAE01F9F300D1124132F13C06AE0569E1D
:10167000300D1124532E20620CC08E3221F426FD31
:1016800011C3206406C08C3611F4206802C088366D
:1016900041F4F10193FD859193FF81911F01811127
:1016A000C1CF9BEB980F933018F42061805E06C089
:1016B0009BE9980F933008F0AAC12F7E26FF16E011
:1016C0002F73722E853621F4F22FF0647F2E08C01E
:1016D000863621F4622F6068762E02C011111150F7
:1016E00077FE07C01C3348F444244394410E27E09E
:1016F0000BC0183030F4212F06C027E04CE3442EF5
:1017000003C027E017E0412C560174E0A70EB11C7E
:10171000F6016081718182819381042DA4010E9470
:10172000CB976C01098100FF02C003FF06C071FC6A
:1017300007C072FC08C0612C08C03DE2632E05C0E2
:101740002BE2622E02C090E2692E802F8C7099F1FC
:10175000662011F084E001C083E0851510F0512C63
:101760000BC0581A73FC08C0B70180E290E00E94D9
:1017700046995A94C9F7F3CF662029F0B701862D10
:1017800090E00E94469903FD03C006ED12E102C0FD
:1017900002ED12E1F72DF0717F2EF801849188237C
:1017A00009F476C271108052B70190E00E94469908
:1017B0000F5F1F4FF2CF77FE0FC04C0C04FF04C029
:1017C0008A81813309F44A94141474F5F8E0F4150D
:1017D00078F588E0482E2CC076FC2AC0812F90E056
:1017E0008C159D059CF06CEFC6166FEFD60674F055
:1017F000772D7068772E0AC0E2E0F0E0EC0FFD1F55
:10180000E10FF11D8081803319F411501111F4CFD3
:1018100077FE0EC044244394410E812F90E0C816F9
:10182000D9062CF41C1904C04424439401C010E0D0
:1018300077FE07C01C141D043CF496012F5F3F4F38
:1018400005C025E030E002C021E030E0662011F064
:101850002F5F3F4F112331F0412F50E04F5F5F4F1B
:10186000240F351F452D50E02417350714F4521A64
:1018700001C0512C872D897049F4552039F0B701EA
:1018800080E290E00E9446995A94F7CF662029F0B2
:10189000B701862D90E00E94469973FC09C055203F
:1018A00039F0B70180E390E00E9446995A94F7CF4F
:1018B00077FE5FC09C2D8D2DD7FE02C090E080E0AA
:1018C000692E782E40E050E0C601841991099D8769
:1018D0008C87960126193709280D391D812F90E034
:1018E000EE27FF27E81BF90BFF87EE87FFEF6F1648
:1018F0007F0669F4B7018EE290E02B8B3A8B488B20
:10190000598B0E944699598948893A892B89C6146E
:10191000D70454F06C857D85661577052CF4F901A4
:10192000E40FF51F818101C080E371E0671A71083F
:101930004F5F5F4FEE85FF856E167F066CF0B70137
:1019400090E02B8B3A8B488B598B0E9446992B89C0
:101950003A8948895989CACF6C147D0439F49A812F
:10196000963318F4953311F404FF81E3B70190E046
:101970004BC08A81813309F00F7EB70190E00E944D
:101980004699111105C074FE18C085E490E017C097
:10199000B7018EE290E00E94469982E0662463944B
:1019A000680EF401E80FF11D8081B70190E00E94FC
:1019B0004699115041F3862DF1CF85E690E0B701AD
:1019C0000E944699D7FC05C0C114D10439F404FF24
:1019D00005C0D194C194D1088DE201C08BE2B7015A
:1019E00090E00E94469980E36AE0C616D1042CF08C
:1019F0008F5FFAE0CF1AD108F7CFB70190E00E94CD
:101A00004699B701C601C0960E94469941C18336E6
:101A100031F0833779F0833509F058C021C0560181
:101A200072E0A70EB11CF6018081898301E010E00D
:101A3000640114C05601F2E0AF0EB11CF601C08083
:101A4000D18026FF03C0612F70E002C06FEF7FEFEF
:101A5000C6012B8B0E94F2988C012B892F7715C021
:101A60005601F2E0AF0EB11CF601C080D18026FF16
:101A700003C0612F70E002C06FEF7FEFC6012B8BB8
:101A80000E94B4988C012B892068722E23FD1AC005
:101A9000852D90E008171907A8F4B70180E290E0BF
:101AA0000E9446995A94F4CFF60177FC859177FE0F
:101AB00081916F01B70190E00E94469951105A94AC
:101AC000015011090115110579F7E2C0843611F0B2
:101AD000893651F5560127FF09C0F4E0AF0EB11C5D
:101AE000F60160817181828193810AC0F2E0AF0EBC
:101AF000B11CF60160817181882777FD8095982F50
:101B0000022F0F7697FF08C090958095709561958C
:101B10007F4F8F4F9F4F00682AE030E0A4010E9462
:101B2000809AC82EC8183EC0022F853721F40F7E38
:101B30002AE030E01DC0097F8F3691F018F4883517
:101B400059F0B0C0803719F0883711F0ABC0006190
:101B500004FF09C0046007C024FF08C0066006C077
:101B600028E030E005C020E130E002C020E132E0B2
:101B7000560107FF09C0F4E0AF0EB11CF601608109
:101B800071818281938108C0F2E0AF0EB11CF60131
:101B90006081718180E090E0A4010E94809AC82E4B
:101BA000C8180F7706FF0BC0202F2E7FC11650F4E8
:101BB00004FF0AC002FD08C0202F2E7E05C0DC2CC9
:101BC000202F03C0DC2C01C0D12E24FF0DC0FE014C
:101BD000EC0DF11D8081803311F4297E09C022FFB4
:101BE00006C0D394D39404C0822F867809F0D3948E
:101BF00023FD13C020FF06C01C2DD51418F4150DAD
:101C00001D19D52CD51468F4B70180E290E02B8B18
